:10000000004000207D600000BD600000BF60000077
:1000100000000000000000000000000000000000E0
:10002000000000000000000000000000C1600000AF
:100030000000000000000000C3600000C560000078
:10004000C760000055470000F9640000C760000069
:10005000C760000000000000C7600000C76000002B
:10006000C7600000C9670000C7600000C7600000EB
:10007000C7600000C7600000C7600000C7600000E4
:10008000C760000061690000C7600000C760000031
:10009000C7600000C7600000C7600000C7600000C4
:1000A000C7600000C7600000000000000000000002
:1000B0000000000000000000000000000000000040
:1000C00010B5064C2378002B07D1054B002B02D02E
:1000D000044800E000BF0123237010BD500200203F
:1000E0000000000030D10000044B10B5002B03D0FD
:1000F0000349044800E000BF10BDC04600000000F6
:100100005402002030D10000164B002B00D1144BBC
:100110009D46402292029A1A924600218B460F4633
:100120001348144A121A0AF0C3F90F4B002B00D0DF
:1001300098470E4B002B00D0984700200021040068
:100140000D000D48002802D00C4800E000BF0AF066
:100150006FF92000290006F0EDF90AF043F9C046D6
:100160000000080000400020000000000000000027
:1001700050020020A82F0020000000000000000016
:100180000123034010D104280CD90268120909D0B8
:10019000531E9B001A1DC1180979002902D0013392
:1001A0009342F8D1180070470023FBE70378002B37
:1001B00003D05AB2002A01DB013070473F2293433B
:1001C000C03B59424B41C01803789343802BF4D174
:1001D0000130F9E710B500240378002B01D120008D
:1001E00010BDFFF7E3FF0134F6E770B5002204000D
:1001F0000D00411C092002F00DFF002806D001234C
:100200006200134343600023A34200DB70BD9A00E9
:10021000A958821891600133F6E770B5012803DC14
:100220001C2000F093FE70BD01230D6811201D42BB
:10023000F7D04868184206D1042804D90F23026871
:100240001340042B01D00E20EBE702F04DFD6D10A2
:100250000400002D03DDFFF7BDFFA84206DA1220DF
:10026000DFE72000FFF7A2FF0400013D012DF8D1D8
:1002700020787F2809DDDF280BDCF8233F22DB0014
:10028000800118406378134018430123400018434D
:10029000C9E7EF280BDCFC22637812019B011340B5
:1002A0003F220007000C0343A0781040ECE7F7283A
:1002B00012DCFC22637892021B031340E0228004CC
:1002C000520310403F221843E3781340FC220343BB
:1002D000A07812018001E8E701204042D5E7F0B59F
:1002E000070085B00D001C20012F06DD4C6801239E
:1002F00022001A40019203D10D2000F027FE54E0A5
:10030000022F02D08A681A42F6D001232E681E42BC
:1003100000D07EE0042E00D87BE01C41002C00DCE5
:100320001C000F2332681340092B29D173685B101E
:100330000193022F05D0AB68019A5B109A4200DD51
:100340000193019B01221F1B0137FB43DB171F4059
:10035000791C092002F05EFE061E09D001237F00F1
:100360001F4303002A68083347600199A14202DA5B
:10037000300005B0F0BD0134A100515802C3F4E7CC
:10038000042B46D1300002F0AFFCFFF723FF0290B0
:10039000022F04D0AB685B10984200DD0293029BF1
:1003A0009C4204DD002002F0A1FE0600E0E73000E0
:1003B00002F09AFC0700019B9C4222DC300001976E
:1003C00002F092FC03903800FFF7F0FE029B01342C
:1003D0000700A342F7DA019BC71A380002F086FE35
:1003E000061EC5D002F080FC0400286802F07CFCE8
:1003F000039A019B991A41183A0020000AF03CF830
:10040000B6E73800FFF7D2FE019B070001330193E6
:10041000D1E7212071E7F8B54D680F00EB0706D44E
:10042000042D04D90F232E683340092B03D00B2051
:1004300000F08CFDF8BD6B6836095C10731EA3429A
:100440000FD80321200007F0EFFE6421642803DCAD
:100450000100032800DA03212800891902F00AFEAE
:1004600005002B6800201B09013B9C42E2D23A6840
:10047000A31C9B005A510123013464001C436C608F
:10048000D8E7F0B585B0012803DC1C2000F05EFD44
:1004900029E001254F682A00022806D08B682B42EC
:1004A00003D05D10002D00DC15000124274200D090
:1004B00074E0042F00D871E00F223B680E681340EF
:1004C000042B25D1264205D1042E03D933681340CD
:1004D000042B01D00E20D9E73800FFF751FEA842C7
:1004E00003DA0120404205B0F0BD380002F0FCFB09
:1004F0000700300002F0F8FB013D010078190AF016
:1005000076FB0028EDD0C01B013040002043EAE715
:10051000092B43D17B685B1000939D42E1DC3000E6
:1005200020402ED1042E2BD90F22336820001340F7
:10053000042B26D1300002F0D7FB0F2325000290B8
:100540000393631C01939B00F858864202D1640018
:100550002800DBE728420ED104280CD90368039A4F
:100560001340042B07D102F0BFFB010002980AF0F0
:1005700011FB0028EBD0019C009B9C42E1DDB0E721
:100580002000431C9A00BA58B24202D14000012414
:10059000BCE71800009B9842F3DDA2E7212075E735
:1005A00010B502F085FB43000120184310BD000088
:1005B00010B57F2902DC0170013010BD1A4B994241
:1005C0000CDC40238A115B42134303703F230B4032
:1005D00080214942194341700230EEE7134B9942A2
:1005E00010DC20230A135B4213433F248022037054
:1005F0008B1152422340214013430A4343708270BF
:100600000330DAE70A4B9942D7DCF0230370603BF2
:100610004370113B8A11FF3B1A4382703F22114005
:100620001943C1700430C8E7FF070000FFFF000056
:10063000FF0F0100F0B50D0085B0002803DC1C2081
:1006400000F084FC0DE009680122080010400AD087
:1006500002AC11412000FFF7ABFF011B200002F0AC
:1006600051FD04001AE004293FD90F230C682340F0
:10067000092B3AD14B685B10019303239C46019BE5
:100680009A420EDD02F032FD041E07D02E680125CD
:1006900002F02AFB2F00019B9D421DDD200005B0CA
:1006A000F0BD01329300CC580123234001D10D202D
:1006B000C6E764107F2C0DDD0D4E0223B44209DD28
:1006C0000C4E6346B44205DD00270B4EE30FA642F5
:1006D0007B419B00C018D2E70135AB00F15839428D
:1006E000E5D04910FFF764FFD5E72120A8E7C04611
:1006F000FF070000FFFF0000FF0F010010B504001E
:100700000120084010D104290DD90F230A68134095
:10071000042B08D1080002F0E7FA010020000AF0DB
:1007200039FA4342584110BD0020FCE7F7B50F00ED
:10073000012803DC1C2000F009FCFEBD01264D68E9
:100740002E4006D1042D04D90F222B681A40092A05
:1007500001D00B20EFE76A681B095410A34200D8B0
:100760005C1E39681E48FFF7C9FF0123019000286D
:1007700013D139681B48FFF7C1FF002811D0002CA6
:100780000DD00123621C013C9C4092005351234335
:100790006B6004E00136B200AB50B442FADA0020DC
:1007A000CBE73B680D20DA07C5D55B10002B11DDC8
:1007B0009C420FDB9B00A200291DEB188918043313
:1007C000994209D10123013C9C40AA181C43536063
:1007D0006C60E4E71220AEE758681860EFE7C046A7
:1007E0000BBB00000FBB0000002310B50C000B700A
:1007F000C30705D50D49421020000AF09DF908E015
:100800000B49002802D0042804D10A4920000AF02C
:10081000B3F910BD0428FCD90F2302681340042B40
:10082000F7D102F061FA04490200E5E768C300006D
:1008300014BB00001ABB00001FBB0000F0B593B052
:100840000390030002911C20012B1DDD029B01255A
:100850001B681C002C4000D0A8E0042B00D8A5E0A9
:100860001A680F231A40092A48D10194019A029963
:1008700092008A5816002E4005D1042A03D9106828
:100880001840092804D0222000F060FB07002CE06B
:1008900052685210A418019A013201920199039AE8
:1008A0008A42E3D1611C012202F0B4FB071E01D190
:1008B00000271AE064002543456005000835029AC8
:1008C000B300D1584B680A685B1012099A4200D8ED
:1008D000531E002293420BDCDA43D21713409B00D5
:1008E000ED18019B01369E42E9DB380013B0F0BDE4
:1008F00090000C18A46801322C50EBE7042A55D163
:100900002F0026001D00029AB300D058384237D17C
:10091000042835D903682B40042BB4D1FFF730FCF1
:10092000039B01362418B342EDD1200002F0DEFB18
:10093000071EBDD0039B029D9B00EB18041D029374
:1009400001232E681E4222D1042E20D90F223368A3
:100950001340042B0DD13000FFF712FC0190300042
:1009600002F0C2F9019A0100200009F085FD019B07
:10097000E418029B0435AB42E2D100232370B4E7B4
:1009800005A9FFF731FF05A80AF016F9C8E705A980
:100990003000FFF729FF05A80AF00EF90600020053
:1009A00005A9200009F068FDA419E2E7212000F064
:1009B000CDFA7DE7F0B50D0095B0002806DC1C20CF
:1009C00000F0C4FA0400200015B0F0BD0C6801214D
:1009D00023000B40009306D1042C04D922680F3366
:1009E0001A40092A01D00B20EAE7626852100392EC
:1009F000002A03DC009802F079FBE3E73F4A01920A
:100A000001280BD06868084208D1042806D902687A
:100A10001340042B02D102F067F9019001980AF00B
:100A2000CBF806000F27039B0834013B04935E4379
:100A3000039B02909B001B19059301232068184219
:100A400051D104284FD903683B40042B52D1FFF702
:100A500097FB059B04343618A342EED1300002F018
:100A600045FB041EAFD02B680593029B002B03D0DF
:100A7000686802F039F90190200002F035F90500AC
:100A8000009B059A9B00D3189F68380002F02CF950
:100A9000012306001F4201D1042F04D807A9380002
:100AA000FFF7A2FE07AE30000AF086F8070002004A
:100AB0003100280009F0E0FC029BED19002B0AD060
:100AC000049B009A934206DD2800029A019909F0DE
:100AD000D3FC029BED18009B01330093009A039B0B
:100AE0009342CDD16FE707A9FFF77EFE07A80AF072
:100AF00063F8AEE702F0F8F8F9E7C0466FBE000011
:100B000010B50024A04207DD0B6801341C4003D05F
:100B10005C10E343DB171C40611C0122092002F03A
:100B200079FA002803D0012364001C43446010BDFF
:100B30000B6870B518000125284032D1042B30D93C
:100B40000F241A6849681440092C16D15C681209F0
:100B50002C41A24200D8541E844205DC02200132FE
:100B6000904206DB00200FE085005D19A96001308E
:100B7000F2E7840019510130F2E7032C11D1294228
:100B800003D1132000F0E2F970BD4910FF29F8D815
:100B90001209043392009A189A42E3D9197001336A
:100BA000FAE70B2000F0D2F9DCE700000123F7B5EB
:100BB00000264D680F002B400093B3420DD11E005C
:100BC000042D0AD90F222B681A40092A0FD16A680E
:100BD0001B095610B34200D85E1E3968CB0713D5E7
:100BE0004C10002C01DDA64219DA12202EE0042A56
:100BF00004D12800FFF7C4FA0600EEE7009E032A9E
:100C0000EBD11E09B600E8E72E48FFF777FD002874
:100C100014D009F02DFF310007F0ECFB4C1C009BB9
:100C2000002B4CD1042D4AD92A680F331340092BCD
:100C300010D10134A40064592000FEBD3968224857
:100C4000FFF75CFD34000028E9D1113000F07EF997
:100C50000400F1E7042B2AD1280002F045F8060031
:100C6000FFF7B8FAA042C0DB012C1ADC280002F022
:100C70003BF800903000FFF799FA851B280002F03E
:100C800035FA041ED8D002F02FF80190786802F0EF
:100C90002BF8009B2A00F11A4118019809F0ECFB8F
:100CA000CAE73000FFF782FA013C0600DCE7032BBD
:100CB00005D12C19E478023B64001C43BCE70B20EF
:100CC000C4E7C04604BB00000FBB0000F7B54C688A
:100CD0000F000120210001402AD1042C28D90F2225
:100CE0002368BE681A40092A13D162681B0955108F
:100CF0000191AB4200D85D1E39682848FFF7FEFC21
:100D0000002829D00F2322681340092B19D1012371
:100D100013E0032A0CD1064203D1132000F016F988
:100D2000FEBD72100192FF2AF7D81D09AD00E3E75E
:100D30000B20F3E701339A00A6509D42FADA002017
:100D4000EEE7032BFBD1230001331A1BAA42F6DC8A
:100D50006A461279DA70F7E73968CB0706D5491089
:100D6000002901DD8D4209DA1220D7E70C48FFF790
:100D7000C5FC2900002801D11130CFE70F232268DC
:100D80001340092B03D1013189000E51D7E7032B02
:100D9000D5D16B461B796418E370D0E70BBB00001C
:100DA0000FBB000010B501240868204216D10428AA
:100DB00014D90F2203681A40092A01D1406810BDD6
:100DC000032A03D11809C0002043F8E7042A05D1FB
:100DD00001F08AFFFFF7FEF94000F5E70B2000F075
:100DE000B5F8ECE710B5034A0A21034803F0BCFD4F
:100DF00010BDC046B4BA0000ACBA00000200012029
:100E0000104001D0501070470D22014B1A70FAE7C4
:100E100090020020F0B585B00393019002912C4E12
:100E20002C4B002A02D002223270013A00251A60AF
:100E30001B68F554019B9D4201DB05B0F0BD029A91
:100E4000AB00D058234B1C68C8239B0037191C1BD0
:100E50000123184206D0204A43102100380009F02F
:100E600039FE09E01D4A002802D004281BD11C4A83
:100E70002100380009F02EFE300009F09DFE154AD1
:100E8000039B1060002B0CD0019B013BAB4208DDA3
:100E9000144B984205D8431C136020223254002280
:100EA000F2540135C6E704280FD90F230268134016
:100EB000042B04D101F018FF0B4A0300CDE7092BE6
:100EC00004D14368094A5B10C7E70123084AC4E715
:100ED00091020020B405002068C3000014BB00008C
:100EE0001ABB00001F0300005FC9000084BD0000A2
:100EF00093BD00000123020010B51A4015D104284B
:100F000001D9026812090B4011D1042901D90B68DB
:100F10001B090024934206D104309B000431C318FE
:100F2000984206D30124200010BD0022EBE70023E5
:100F3000EFE704780A78002C01D1002AF2D00130C2
:100F400001319442ECD00024EDE70000014B187011
:100F5000002070479002002070B501F0D5FC094CCC
:100F60000100251D1F22280009F02DFE280009F090
:100F700023FE042304308008000118432060200071
:100F800070BDC0466C020020C368F0B59D00836848
:100F900089B05D190300183306930369069A9F0010
:100FA000069B0290DF19436901939B00D3180393BA
:100FB000CD4B1B78002B26D17F222B68CB491C12EE
:100FC00013409B005B58043501929F46029B587862
:100FD00004F0A6F80023029A137027E0C24B1B7896
:100FE000002B10D12B68019A1C121340BF4A9B00A2
:100FF0009B580435E9E7069B3A1DD11ABA4BD8290C
:1010000028DD1A221A70029BB74C9B682178019345
:10101000EA1A029B92109B7812021A43029B58789C
:1010200004F086F80023029A23701370029B069A3C
:101030009B680193ED1A029BAD10DD60069BFE1AC2
:10104000029BB6101E61039B9B1A029A9B10536170
:1010500009B0F0BD1B783C60002B01D01700D2E72F
:101060002B6801991C120B40A0499B005B5817008C
:101070000435AAE7069B3A1DD11A9B4BD82902DDFD
:101080001A221A70BFE728681B78291D3860002BC8
:1010900002D017000D00B6E76B6801991C120B40D7
:1010A00092499B005B58170008358EE7069B3A1D56
:1010B000D11A8D4BD82902DD1A221A70A3E7A40099
:1010C0001B782C193C60002B01D017009BE72B6884
:1010D00001991C120B4085499B005B581700043591
:1010E00073E7069B3A1DD11A7F4BD82902DD1A22DD
:1010F0001A7088E77E49A40061581B783960002B7C
:1011000001D017007FE72B6801991C120B4077492B
:101110009B005B581700043557E7043F744B3A684F
:10112000A400E250704B1B78002B00D06BE72B68BB
:10113000019A1C1213406D4A9B009B58043544E7EA
:101140006B4BA400E058FFF759FE043F06003868D7
:10115000FFF754FE36180120654B76000643E65033
:10116000614B1B78002B00D04DE72B68019A1C12B5
:1011700013405E4A9B009B58043526E7069B3A1DA8
:10118000D11A594BD82902DD1A221A703BE706986A
:10119000039C0121A04202D221000C3909681B786E
:1011A0003960002B01D017002DE72B6801991C1224
:1011B0000B404E499B005B581700043505E7069B22
:1011C0003A1DD11A484BD82902DD1A221A701AE7A3
:1011D0000699039881420FD203000C3B1B684549D6
:1011E0005B106418E41AA40023583B603E4B1B7844
:1011F000002B05D0170006E7182119700023F4E72B
:101200002B6801991C120B4038499B005B58170052
:101210000435DAE6069B039A934219D213000C3B7D
:101220001B68344A043FA4185B10E31A039A396818
:101230009B0099502C4B1B78002B00D0E3E62B68C9
:10124000019A1C121340294A9B009B580435BCE6A6
:101250001822254B1A70EDE7069B039A93422DD274
:10126000244B3E1FE31814000C3C04932368049A9B
:101270005B10D31A039A9B009858FFF7BFFD0790A5
:101280003068FFF7BBFD2468049B64101C1B079BA0
:10129000A4001F1801207F00039B0743E75037007D
:1012A000114B1B78002B00D0ADE62B68019A1C1265
:1012B00013400E4A9B009B58043586E618220A4BC1
:1012C0001A70EDE7069B3A1DD11A074BD82902DDAB
:1012D0001A221A7097E60399A40061581B783960A6
:1012E000002B09D017008EE69002002084BB00007E
:1012F000502D0020FDFFFF3F2B6801991C120B4071
:10130000D7499B005B58170004355EE6043F039BFA
:101310003A68A400E250D34B1B78002B00D072E651
:101320002B68019A1C121340CD4A9B009B58043530
:101330004BE6039BA4001C192368043F38685E1029
:10134000FFF75CFD36180120C64B76001B7806437C
:101350002660002B00D056E62B68019A1C12134021
:10136000BF4A9B009B5804352FE6069BA4003F1BF9
:10137000BC4CBB420CD82378002B00D043E62B6832
:10138000019A1C121340B64A9B009B5804351CE678
:10139000B54801F099FC2378002B00D033E62B6888
:1013A000019A1C121340AE4A9B009B5804350CE670
:1013B000A300ED18002C00DA38E6AA4B1B78002BAE
:1013C00000D020E62B68019A1C121340A44A9B000F
:1013D0009B580435F9E5043F3B68042B04D1A30076
:1013E000ED18002C00DA21E69E4B1B78002B00D074
:1013F00009E62B68019A1C121340994A9B009B58DE
:101400000435E2E5043F3B68042B06D0A200AD188A
:10141000002C02DA002B00D108E6924B1B78002B3F
:1014200000D0F0E52B68019A1C1213408C4A9B00F7
:101430009B580435C9E53A1F13685B10013B002B2C
:1014400006DD01215B00A4000B432D191360EDE5BF
:10145000844B17001B78002B00D0D4E52B68019A31
:101460001C1213407E4A9B009B580435ADE53A00A0
:10147000069B0C32D31AD82B03DD1A22794B1A7033
:10148000C1E5FF2361005B001940FE3BFF3B1943B0
:101490003960029906988968241204916D1A02999C
:1014A000AD1089782D020D4303999D40091A8910CA
:1014B00099401D430B43BB60029B7D609C70E4B26E
:1014C0006A4BE4000392E358029A9360654A1278EB
:1014D000002A03D008331D00039F94E51D00019AE4
:1014E0009B680C351C1213405D4A9B009B58039F60
:1014F0006BE53B1F1C68039A069B93422DD10A2083
:10150000E3070CD4042C13D90F2322681340042BB7
:1015100011D1200001F0E8FB09F04EFB06306430E9
:1015200003F0B2FA00280FD1043D069B03937DE53A
:101530000720042CF3D02000431E9841FA23404298
:10154000FF3318400730EAE7029B2100587803F088
:1015500001FE0023029A1370E7E7039B039A0C3BFA
:101560001B6802995B109B00D31A0C3B1C601F1D6B
:101570001300083B1B685A108A70D2B23B49D20054
:101580005B0055589B0A029A9B009560ED18039BDF
:10159000069A043B1B685B109B00D3180393314BE6
:1015A0001B78002B00D02EE52B68019A1C121340EB
:1015B0002B4A9B009B58043507E53B1F1868FFF733
:1015C0001DFCA40006003F1B1E2827DC00280DDCA4
:1015D000244B1B78002B00D015E52B68019A1C12B8
:1015E00013401F4A9B009B580435EEE401F07AF942
:1015F000033E361801F076F91D4B801B9842F9D84E
:10160000184B1B78002B00D0FDE42B68019A1C12AC
:101610001340134A9B009B580435D6E40123029AD9
:10162000137001F05FF9029B0A3886195E60FDE4D1
:101630003B1F1868FFF7E2FBA40006003F1B0028D1
:1016400018DC084B1B78002B00D0DCE42B68019AD7
:101650001C121340024A9B009B580435B5E4C04657
:1016600084BB000090020020A5BD0000582500208A
:101670003F420F00CA4B984203DD1D22C94B1A702E
:10168000C1E40123029A137001F02CF9FA239B00A4
:101690005E43029B0A3E30185860C7E4A300FF1A5D
:1016A000002320001A003900FFF7B4FBBE4EBF4CE8
:1016B0003168200001F026FDBD4B31681860200024
:1016C00003F0FCFB3168200003F04BFD3168200083
:1016D00001F0B4FDB34B1B78002B00D093E42B68D2
:1016E000019A1C121340B34A9B009B5804356CE4CA
:1016F000AC4BA4001B783F1B002B00D083E42B686D
:10170000019A1C121340AB4A9B009B5804355CE4C1
:10171000029803F01DFAA34B1B78002B00D072E453
:101720002B68019A1C121340A24A9B009B58043557
:101730004BE43B1F1B68002B3ED13B000C3B1B685E
:10174000DA072CD5390001225B1058000839024312
:101750000A60002B44DD012259001143381F01604B
:101760003900083909681141CB1A39000C39096868
:10177000114224D09B189340A4001343039AA35012
:10178000884B1B78002B00D03DE42B68019A1C127B
:101790001340884A9B009B580435FFF716FC042B26
:1017A00006D90F2219680A40092A01D15B68C9E7E6
:1017B00019227C4B1A7026E45B10013BC9E704290F
:1017C00009D90F2208680240092A04D102339B007C
:1017D0005B58A400D2E71922724B1A70FFF713FC72
:1017E0000435CDE7A300069AFB189B1AD82B13DC0F
:1017F0000122631E002C14DC6A4B1B78002B01D0E5
:10180000FFF701FC2B68019A1C121340694A9B00E8
:101810009B580435FFF7D9FB1A22624B1A70FFF769
:10182000F2FB3A601C000437E3E7069A3B1D9B1A63
:101830005C4ED82B03DD1A233370FFF7E4FB069BC5
:10184000039AA40093422AD23B1F1868FFF7D6FAE6
:10185000011E21DD039B0C3B1A68521082421BDBE8
:101860009007801A544B4018C018039B8000C25840
:101870003B1B1A604B4B3F1B1B780437002B01D0DE
:10188000FFF7C1FB2B68019A1C121340494A9B00C9
:101890009B580435FFF799FB20233370EAE71823A0
:1018A000FBE7434BA4001A683B1B1F001A603D4B2B
:1018B00004371B78002B01D0FFF7A5FB2B68019A9A
:1018C0001C1213403B4A9B009B580435FFF77DFBDD
:1018D000A3009C46FE1A002C17DC1C22314B1A7008
:1018E000002333606346FF1A2E4B04371B78002B0E
:1018F00001D0FFF788FB2B68019A1C1213402D4A78
:101900009B009B580435FFF760FB002033685A109A
:101910008300F15801230B4003D10D21214A11709E
:10192000DFE749108A4200DD0A0001308442EFDC23
:10193000012352001343D4E7A3009C46FE1A002C57
:1019400017DC1C22174B1A70002333606346FF1A02
:10195000144B04371B78002B01D0FFF754FB2B6886
:10196000019A1C121340134A9B009B580435FFF741
:101970002CFB002033685A108300F15801230B40E0
:1019800003D10D21074A1170DFE749108A4200DABE
:101990000A0001308442EFDC012352001343D4E7F4
:1019A00080EE360090020020B40500209102002055
:1019B0000800002084BB0000FCFFFF3F3B00083B09
:1019C0001868FFF71BFA3B1F06001868FFF716FAA6
:1019D0000023864200DA0433A4003A1B1700136088
:1019E000E34B04371B78002B01D0FFF70CFB2B686F
:1019F000019A1C121340DF4A9B009B580435FFF7E5
:101A0000E4FA3B00083B1868FFF7F8F93B1F0600B3
:101A10001868FFF7F3F9F30FC217B0425341A4005F
:101A20003A1B17009B001360D14B04371B78002B27
:101A300001D0FFF7E8FA2B68019A1C121340CD4A37
:101A40009B009B580435FFF7C0FA3B00083B186821
:101A50003B1F1968A600BE1B0423814202D0042844
:101A600002D80023336016E001231842F9D10F2376
:101A700002681A40042AF4D1033A1142F1D1042930
:101A8000EFD90A681340042BEBD1FFF733FA431E5A
:101A9000984180003060B64BA4001B783F1B043790
:101AA000002B01D0FFF7AFFA2B68019A1C121340EC
:101AB000B04A9B009B580435FFF787FA3B00083B70
:101AC00018683B1F1968A600BE1B0023814202D084
:101AD000042802D80423336016E001231842F9D108
:101AE0000F2302681A40042AF4D1033A1142F1D1BB
:101AF0000429EFD90A681340042BEBD1FFF7FAF958
:101B00004342584180003060994BA4001B783F1B32
:101B10000437002B01D0FFF776FA2B68019A1C12CC
:101B20001340944A9B009B580435FFF74EFA3B0044
:101B3000083B1868FFF762F93B1F06001868FFF7BB
:101B40005DF9F317C20F86425341A4003A1B1700F8
:101B50009B001360864B04371B78002B01D0FFF7E6
:101B600052FA2B68019A1C121340824A9B009B5820
:101B70000435FFF72AFA3B00083B1868FFF73EF9E7
:101B80003B1F06001868FFF739F90023864200DD85
:101B90000433A4003A1B17001360754B04371B78FD
:101BA000002B01D0FFF72FFA2B68019A1C1213406B
:101BB000704A9B009B580435FFF707FA3B1F1B68D0
:101BC000A400043B5A1E93413A1B17009B0013606C
:101BD000674B04371B78002B01D0FFF714FA2B68F2
:101BE000019A1C121340634A9B009B580435FFF76F
:101BF000ECF93B00083B1868FFF700F93B1F0600B3
:101C00001868FFF7FBF832180120A4003B1B1F00E7
:101C1000520002431A60564B04371B78002B01D048
:101C2000FFF7F1F92B68019A1C121340514A9B00EF
:101C30009B580435FFF7C9F93B00083B1868FFF7CC
:101C4000DDF83B1F06001868FFF7D8F8321A0120AC
:101C5000A4003B1B1F00520002431A60444B043790
:101C60001B78002B01D0FFF7CEF92B68019A1C12CC
:101C70001340404A9B009B580435FFF7A6F93B00F0
:101C8000083B1868FFF7BAF83B1F06001868FFF713
:101C9000B5F802000120A4003B1B1F007243520054
:101CA00002431A60324B04371B78002B01D0FFF738
:101CB000AAF92B68019A1C1213402E4A9B009B58CC
:101CC0000435FFF782F93B1F1868FFF797F8061EE7
:101CD00017D11F22264B1A70A4003B1B1F001E6049
:101CE000234B04371B78002B01D0FFF78CF92B68AE
:101CF000019A1C1213401F4A9B009B580435FFF7A2
:101D000064F93B00083B1868FFF778F8310006F0EB
:101D10008BFA012640000643DEE73B1F1868FFF7F9
:101D20006DF8061E17D11F22114B1A70A4003B1B21
:101D30001F001E600E4B04371B78002B01D0FFF7ED
:101D400062F92B68019A1C1213400A4A9B009B58A7
:101D50000435FFF73AF93B00083B1868FFF74EF8E7
:101D6000310006F047FB012649000E43DEE7C0467E
:101D70009002002084BB00003B1F1868FFF73EF86C
:101D8000C217801850400122A4003B1B1F004000D6
:101D900010431860F64B04371B78002B01D0FFF777
:101DA00032F92B68019A1C121340F24A9B009B588F
:101DB0000435FFF70AF9A300FE1A3068012C24D17C
:101DC000FFF71CF80494079008F052FE07990029C9
:101DD00000DC012106F00EFB049BA400C9180123BE
:101DE00049001943E24B3F1B1B7831600437002B3D
:101DF00001D0FFF708F92B68019A1C121340DD4A45
:101E00009B009B580435FFF7E0F8FEF7F7FF0490BE
:101E10007068FEF7F3FF049B0130C31A0793D3E702
:101E2000A300FE1A31002000049301F0A7F9049BDF
:101E30003060FF1ACE4B04371B78002B01D0FFF720
:101E4000E2F82B68019A1C121340CA4A9B009B5867
:101E50000435FFF7BAF83B00083B1868FEF7CEFFE1
:101E60003B1F06001868FEF7C9FF02000120A4000E
:101E70003B1B1F003240520002431A60BC4B043728
:101E80001B78002B01D0FFF7BEF82B68019A1C12BB
:101E90001340B84A9B009B580435FFF796F83B0067
:101EA000083B1868FEF7AAFF06003B1F1868FEF7FC
:101EB000A5FF320002430120A4003B1B1F0052007B
:101EC00002431A60AA4B04371B78002B01D0FFF79E
:101ED0009AF82B68019A1C121340A64A9B009B5843
:101EE0000435FFF772F83B00083B1868FEF786FFE1
:101EF00006003B1F1868FEF781FF320042400120B8
:101F0000A4003B1B1F00520002431A60984B043789
:101F10001B78002B01D0FFF776F82B68019A1C1272
:101F20001340944A9B009B580435FFF74EF83B1F23
:101F30001868FEF763FFC0430122A4003B1B1F008B
:101F40004000104318608A4B04371B78002B01D0E7
:101F5000FFF759F82B68019A1C121340854A9B0021
:101F60009B580435FFF731F83B00083B1868FEF733
:101F700045FF06003B1F1868FEF740FF3200824015
:101F800051000122A4003B1B1F000A431A60784B3A
:101F900004371B78002B01D0FFF735F82B68019A26
:101FA0001C121340734A9B009B580435FFF70DF831
:101FB0003B00083B1868FEF721FF06003B1F18682E
:101FC000FEF71CFF3200024151000122A4003B1B1E
:101FD0001F000A431A60664B04371B78002B01D0A0
:101FE000FFF711F82B68019A1C121340614A9B00FD
:101FF0009B580435FEF7E9FF3B000C3B1868FEF7E1
:10200000FDFE3B00083B06001868FEF7F7FEF117DF
:102010000200C317300006F03FFA3B1F0490059101
:102020001868FEF7EBFE02000498059906F0E8F93F
:1020300043000120A4003E1B370018434C4B306086
:102040001B780437002B01D0FEF7DDFF2B68019AC7
:102050001C121340474A9B009B580435FEF7B5FFFE
:10206000A300FE1A310020000493FEF749FD049BF3
:102070003060FF1A3E4B04371B78002B01D0FEF76F
:10208000C2FF2B68019A1C1213403A4A9B009B58CE
:102090000435FEF79AFFA300FF1A39002000FEF76F
:1020A00047FD334B1B78002B01D0FEF7ACFF2B68AC
:1020B000019A1C1213402F4A9B009B580435FEF7CF
:1020C00084FFA300FE1A310020000493FEF76EFD8A
:1020D000049B3060FF1A264B04371B78002B01D07D
:1020E000FEF791FF2B68019A1C121340214A9B00B6
:1020F0009B580435FEF769FFA300FF1A3900200042
:10210000FEF7E4FD1A4B1B78002B01D0FEF77BFF96
:102110002B68019A1C121340164A9B009B580435E9
:10212000FEF753FFA300FE1A310020000493FEF7D0
:1021300039FE049B3060FF1A0D4B04371B78002BCF
:1021400001D0FEF760FF2B68019A1C121340094A68
:102150009B009B580435FEF738FF069B3E1DF31A83
:10216000034CD82B08DD1A232370FEF74CFFC04622
:102170009002002084BB000000F0BEFB4300012061
:10218000184323783860002B02D03700FEF73BFF5E
:102190002B68019A1C121340F44A9B009B5837008D
:1021A0000435FEF712FF069B3E1DF31AF04CD82BA8
:1021B00003DD1A232370FEF726FF00F093FBED4B9F
:1021C000400018400123184323783860002B02D0C8
:1021D0003700FEF718FF2B68019A1C121340E34AE0
:1021E0009B009B5837000435FEF7EFFE0123A60045
:1021F000BE1B20001A003100FEF70CFEDE4C2068EA
:10220000643002F041FC002802D1043DFEF70EFFCD
:10221000029B21685A78D94802F0B1FF0123029A43
:102220003700137000F05EFBD54B22681B68063246
:1022300053431818029B5860FEF7F8FEA600BE1B19
:102240002000012300223100FEF7E4FDCA4C206883
:10225000643002F019FC0028D7D0C84802F086FD8F
:10226000DCE7A4003E1BFEF777FE3700C04B306072
:102270001B780437002B01D0FEF7C5FE2B68019AAE
:102280001C121340B94A9B009B580435FEF79DFE73
:10229000A4003E1B300000F05EFB3700B44B306002
:1022A0001B780437002B01D0FEF7ADFE2B68019A96
:1022B0001C121340AD4A9B009B580435FEF785FE67
:1022C000A4003E1B300000F048FB3700A84B3060F4
:1022D0001B780437002B01D0FEF795FE2B68019A7E
:1022E0001C121340A14A9B009B580435FEF76DFE5B
:1022F000A300FE1A31002000049300F031FB049B80
:102300003060FF1A9A4B04371B78002B01D0FEF780
:102310007AFE2B68019A1C121340944A9B009B582A
:102320000435FEF752FEA4003F1B380000F04AFBC4
:102330008F4B1B78002B01D0FEF765FE2B68019AAE
:102340001C121340894A9B009B580435FEF73DFE42
:10235000A300FE1A31002000049300F05BFB049BF5
:102360003060FF1A824B04371B78002B01D0FEF738
:102370004AFE2B68019A1C1213407C4A9B009B5812
:102380000435FEF722FEA4003F1B380000F084FB5A
:10239000774B1B78002B01D0FEF735FE2B68019A96
:1023A0001C121340714A9B009B580435FEF70DFE2A
:1023B0000121200000F058FB6D4B1B78002B01D051
:1023C000FEF721FE2B68019A1C121340674A9B00FE
:1023D0009B580435FEF7F9FD0021200000F044FB76
:1023E000634B1B78002B01D0FEF70DFE2B68019A82
:1023F0001C1213405D4A9B009B580435FEF7E5FD17
:10240000A4003E1B300000F069FB3700584B3060E1
:102410001B780437002B01D0FEF7F5FD2B68019ADD
:102420001C121340514A9B009B580435FEF7CDFD0A
:10243000A4003E1B300000F065FB37004C4B3060C1
:102440001B780437002B01D0FEF7DDFD2B68019AC5
:102450001C121340454A9B009B580435FEF7B5FDFE
:10246000A4003F1B380000F027FB414B1B78002BDA
:1024700001D0FEF7C8FD2B68019A1C1213403B4A9D
:102480009B009B580435FEF7A0FDA4003F1B3800BD
:1024900003F090F9364B1B78002B01D0FEF7B3FD0B
:1024A0002B68019A1C121340304A9B009B5804353C
:1024B000FEF78BFDA4003E1B300003F00DFA370041
:1024C0002B4B30601B780437002B01D0FEF79BFDAF
:1024D0002B68019A1C121340244A9B009B58043518
:1024E000FEF773FDA4003F1B380003F013F9204BE7
:1024F0001B78002B01D0FEF786FD2B68019A1C1279
:1025000013401A4A9B009B580435FEF75EFDA40059
:102510003E1B300003F014F93700154B30601B7878
:102520000437002B01D0FEF76EFD2B68019A1C12B8
:1025300013400E4A9B009B580435FEF746FDA3004E
:10254000FF1A3900200001F01BF9094B1B78002B02
:1025500001D0FEF758FD2B68019A1C121340034A64
:102560009B009B580435FEF730FDC04684BB00003D
:1025700090020020FEFFFF7FB405002091020020A2
:1025800004000020A300FF1A3900200000F080FFA3
:102590009F4B1B78002B01D0FEF735FD2B68019A6D
:1025A0001C1213409B4A9B009B580435FEF70DFDFF
:1025B000A300FF1A3900200000F07AFF944B1B782B
:1025C000002B01D0FEF71FFD2B68019A1C1213404F
:1025D000904A9B009B580435FEF7F7FCA300FF1AB6
:1025E0003900200000F08CFF894B1B78002B01D0B4
:1025F000FEF709FD2B68019A1C121340854A9B00C7
:102600009B580435FEF7E1FCA300FE1A31002000C0
:10261000049303F006FA049B3060FF1A7C4B0437E6
:102620001B78002B01D0FEF7EEFC2B68019A1C12E0
:102630001340784A9B009B580435FEF7C6FCA30064
:10264000FE1A31002000049303F0F3F9049B30607C
:10265000FF1A6F4B04371B78002B01D0FEF7D3FC19
:102660002B68019A1C1213406A4A9B009B58043540
:10267000FEF7ABFCA300FE1A31002000049303F028
:10268000E0F9049B3060FF1A614B04371B78002B84
:1026900001D0FEF7B8FC2B68019A1C1213405D4A6A
:1026A0009B009B580435FEF790FCA300FE1A3100F6
:1026B0002000049302F0E6FF049B3060FF1A544BA5
:1026C00004371B78002B01D0FEF79DFC2B68019A84
:1026D0001C1213404F4A9B009B580435FEF775FCB3
:1026E000A300FF1A3900200000F0D2FF484B1B78EE
:1026F000002B01D0FEF787FC2B68019A1C121340B7
:10270000444A9B009B580435FEF75FFCA300FF1A68
:102710003900200000F01CFF3D4B1B78002B01D03E
:10272000FEF771FC2B68019A1C121340394A9B007A
:102730009B580435FEF749FCA300FE1A3100200027
:10274000049300F073FE049B3060FF1A304B043793
:102750001B78002B01D0FEF756FC2B68019A1C1247
:1027600013402C4A9B009B580435FEF72EFCA30017
:10277000FF1A3900200000F0E9FF254B1B78002BE1
:1027800001D0FEF740FC2B68019A1C121340214A2D
:102790009B009B580435FEF718FC069B029AFB1A17
:1027A0009B101361A300FF1A3900200002F0F0F81B
:1027B000174B1B78002B01D0FEF725FC2B68019AE4
:1027C0001C121340134A9B009B580435FEF7FDFB77
:1027D000069B029AFB1A9B101361A300FE1A31009C
:1027E0002000049302F0D4F8049B3060FF1A084BD9
:1027F00004371B78002B01D0FEF705FC2B68019AEB
:102800001C121340034A9B009B580435FEF7DDFB66
:102810009002002084BB00000023F7B55A1E0192ED
:10282000002B07DA00F0C2FF02F0A6FB02F006FD63
:102830001923019300263000194B1968B14212DDAB
:10284000184B1A6801328A420FDAF0241A601D68A8
:10285000154F6C43E35D002B1FD0E419022B06D10A
:102860002000FEF791FB019BD8E70022EDE7012B4A
:102870000DD1002801D100F035F8F0226A43BB18D1
:102880005B680A49C31A8B4201D80223BB54F02368
:102890005D43054BEB5C022BE2D00136CCE7C04632
:1028A000B805002000000020F81B00203F420F0068
:1028B00000207047002070470020704700207047BC
:1028C00001220020054B06491A615850043103309B
:1028D00058500831801858501A60704700800040E6
:1028E000040500000122034B1A64A822D200985864
:1028F0007047C0460080004010B5FFF7F3FFFA2193
:10290000890005F007FC10BD00487047F8BD0000C5
:102910001D20704770B5054E0400335C0D008B42DE
:1029200002D003F09DFF355570BDC046BC050020A8
:1029300070B50024064D635D012B05D100212000F8
:1029400003F08EFF0023635501341D2CF2D170BDBE
:10295000BC05002070470D2070473B2070470000E9
:10296000F8B501240B6806000D00234204D10D20A8
:10297000FEF7ECFA2000F8BD5B102000052BFAD81A
:102980000E4A9B009C580E4F3B5D002B05D000214A
:10299000200003F065FF00233B55012E06DD6B6828
:1029A000042B03D10221200003F05AFF200003F082
:1029B00005FE012440002043DDE7C046E0BD0000E5
:1029C000BC050020F8B501260568354202D04468F0
:1029D000344203D10D20FEF7B9FAF8BD6D101C2D5D
:1029E000FBD80A4F7B5D012B04D03100280003F097
:1029F00037FF7E55064964108C4202DCE143C9175B
:102A00002140280003F060FEE7E7C046BC05002037
:102A1000FF03000070B501240D68254204D10D208C
:102A2000FEF794FA200070BD6D101C2D17D80024FD
:102A3000012804DD4C68043C63425C416400094E9B
:102A4000735DA34204D02100280003F009FF7455F0
:102A5000280003F039FF03000420012BE3D00020FD
:102A6000E1E7C046BC05002070B504000D001C283D
:102A70000ED8084E335C012B04D0012103F0F0FE88
:102A800001233355290020004D1EA94103F006FF04
:102A900070BDC046BC050020036810B5DA0703D43A
:102AA0000D20FEF753FA10BD4168581004394A4210
:102AB0005141FFF7D9FFF6E737B569460A00064BE3
:102AC00030CB30C203680220042B02D100F0F0FCAE
:102AD00037BD00F015FDFBE7B8BD000010B5084C90
:102AE0006379002B05D00021052003F0B9FE0023F7
:102AF0006371052003F0E8FE43425841800010BD99
:102B0000BC05002010B5084CE37A002B05D000214D
:102B10000B2003F0A5FE0023E3720B2003F0D4FE8C
:102B200043425841800010BDBC05002070477047EB
:102B300010B5034A0421034801F016FF10BDC0463A
:102B4000C0BD000098C40000E12170B549021448DE
:102B500003F02CFBFFF7B4FE0A2003F029FD00234D
:102B6000FF21104A995401331D2BFBD10122002073
:102B70000D4B01001A6004230C4A0D4D1468002C03
:102B8000FCD02C680002013B20431160002BF5D1E2
:102B90000122084B1A6003F0C5FC00F053FF70BD22
:102BA000801B0020BC05002000D0004000D1004068
:102BB00008D5004004D00040F8B50B4E07003000A7
:102BC0000D0003F03BFB0400A84200DD2C003D009B
:102BD000EB1B9C4205DD300003F03AFB2870013509
:102BE000F6E72000F8BDC046801B002010B50100AC
:102BF000014803F0E3FA10BD801B002010B5054C1E
:102C0000200003F0E9FAE1212000490203F0CEFAA6
:102C100010BDC046801B0020C3070CD4064B1B68A8
:102C2000834208D8054B1B68984204D8031F1B68D1
:102C3000002B00D018007047E4050020E0050020BC
:102C40000023012210B50A48990001334250642B39
:102C5000FAD1084C084B00211A602000074A07F0FF
:102C600027FC074B074A6360074B1A6010BDC0463C
:102C7000502D0020E805002008000020D4090000A5
:102C800030270000EC050020DC05002010B5044BC7
:102C9000044A1A60044B054A1A60FFF7D1FF10BDC1
:102CA000E4050020E8050020E0050020BC0F00201E
:102CB000044B1B68186800090238C343DB1718402F
:102CC0007047C046DC05002000B59BB002000549F6
:102CD00001A807F031FF01A802F064F802F0AEFA93
:102CE000FCE7C0465FBE00000A4BC20704D40428BC
:102CF00004D8094B00D0094B180070470F22036815
:102D00001A40031D042AF7D0054B092AF4D0054BBD
:102D1000F2E7C04645BE00001ABB000014BB00002D
:102D200058BE00004FBE00000020064A0649131F8F
:102D3000186013681B0902339B00D2188A42F6D32D
:102D40007047C046EC050020BC0F0020F7B50F24EB
:102D50000126304B304A1968304B314D18681368E2
:102D60001F002740072F25D813681B0902339B003B
:102D7000D218AA42F3D300242A4EA500AD19286820
:102D8000FFF74AFF01342860642CF6D1264C2068F6
:102D9000FFF742FF2060254C2068002802D0FFF793
:102DA0003BFF20600025224B1B680093009B9D4247
:102DB00013DBF7BD1B099B00D3189A42D4D01F68C0
:102DC000374208D1B94206D2B84204D3043F3F6823
:102DD000002F00D01F60043BEFE7F0236B43154A40
:102DE0009B181A78002A01D10135DFE71F693C23BF
:102DF00000266B43DB199B0001930136BB1BF3D408
:102E0000019BB4001C1B0B4B1C19A069FFF704FFAE
:102E1000A061F2E7E4050020EC050020E0050020B9
:102E2000BC0F0020502D002008000020BC0F002007
:102E3000B8050020F81B0020F7B50124204244D13A
:102E4000224B1B689C4698423FD3214B1B68019341
:102E500098423AD8031F1B68002B36D10200036842
:102E600000941B09002B0FD10099131F1960904289
:102E70002BD015682B1F1B68990069180C68013B43
:102E800014600A602A00EDE79D0055192968009C2E
:102E9000214218D18C4516D8019C8C4213D30E1FA9
:102EA0003468002C0FD10F680F343C40072C07D931
:102EB0002F60151F2B600B680A601B090A00D1E701
:102EC00000993160CEE7013BCCE7F7BDE405002077
:102ED000E00500200D49F0B50B000F260C4D1868D9
:102EE0001C1F276802090232002F0BD000208B42E2
:102EF00000D0080020609000091892009B18AB4297
:102F0000EDD3F0BDB0431860F7E7C046EC050020F4
:102F1000BC0F0020F8B5114C26000F2233681F09A2
:102F200013420DD07D1CAD00A64204D02A00310012
:102F3000200007F0AAFA00226319043564191A6008
:102F40000237BF00064BF6199E42E6D31B1B9B10AF
:102F5000013B1B012360034B1C60F8BDEC05002006
:102F6000BC0F0020DC050020F0B59BB0FFF7BAFCD9
:102F700000240700204AA300D0580134FFF75CFF6B
:102F8000642CF7D11D4B1868FFF756FF1C4B1868CF
:102F9000002801D0FFF750FF00261A4B1B689E4205
:102FA00016DBFFF797FFFFF7D1FEFFF7B3FFFFF741
:102FB00099FC154BC21B1B6814491B6801A81B090F
:102FC000023B07F0B9FD01A801F0ECFE1BB0F0BD1B
:102FD000F02575430E4BED182B78002B01D10136EF
:102FE000DBE72B695C1E002CF9DBA300EB1898696A
:102FF000FFF722FF013CF6E7502D002008000020DB
:10300000BC0F0020B8050020DC05002025BE000014
:10301000F81B0020F7B5164D4F1C2B6806001B68E7
:103020000C0001921B099F420ADBFFF79DFF2B68F2
:103030001B681B099F4203DB0A20FDF787FFFEBDCB
:103040002868A71CBA00DB1B81181B010B602960D4
:103050000021031F19600F231E4003002401264393
:1030600040C3083A9A189A42E9D9019902C3FAE78B
:10307000DC050020F7B503000122134004000D0019
:103080000193002B2AD1164B1B68834226D8154B7F
:103090001B68834222D90F23134F38600068184001
:1030A000FFF7B8FF019B3C68061E3B6016D0236803
:1030B00004301B099D4200DD1D00AA00211D251FB3
:1030C00007F0DAF9FFF730FE2E60FFF73FFE00232E
:1030D0002B6022680F339A43226034002000FEBD2B
:1030E000E4050020E0050020BC0F0020032304308D
:1030F00010B5C11719400918891000220420FFF7E4
:1031000089FF10BD70B5050008000C00FFF7EEFF49
:103110000023002804D170BDE95CC218117101338D
:10312000A342F9DBE343DB171C400023041923719E
:10313000F1E7000010B501240B681C4016D05C10AC
:10314000200005F005FB0B4905F0D0F907F0B6F8B3
:1031500003F0FEFC0022084B06F06AFA03F0A0FC24
:1031600007F03CF843000120184310BD0D20FDF787
:10317000EDFEE5E7D30237390000D040086870B5AE
:1031800001240500254006D1042804D90F23026834
:103190001340042B03D00E20FDF7D8FE70BDFFF7BF
:1031A000A3FD03782900233B5A4253411022C01843
:1031B00007F0B8FD80239B05C218044B9A4201D941
:1031C0001420E9E740002043E8E7C046FFFFFF3F47
:1031D00010B5034A0221034801F0C6FB10BDC046EA
:1031E00078BE000070BE00000020704710B51E20A1
:1031F000FDF7ACFE10BD10B51E20FDF7A7FE10BDFB
:1032000010B51E20FDF7A2FE10BD10B51E20FDF763
:103210009DFE10BD10B51E20FDF798FE10BD10B527
:103220001E20FDF793FE10BD10B51E20FDF78EFE8B
:1032300010BD10B51E20FDF789FE10BD70470000BF
:1032400010B5034A0921034801F08EFB10BDC046AA
:1032500098BE0000E0BE00000120034B1860034B45
:103260001B68834018437047E00F0020C00F002008
:10327000F0B5EFF310810123194083F31088134C4C
:10328000134AA4461268134E013A9340124F134A50
:10329000002B17D0146803420FD03D682C60C04645
:1032A000C046C046C046C046C046C046C0460C4C9C
:1032B0001568246825605B08EAE765462C60146899
:1032C0003460F8E781F31088F0BDC046080500506F
:1032D0000C0000200C050050CC0F0020D40F002063
:1032E000C80F002030B585B001AD0C22064928007A
:1032F00007F0C2F80024285D01210134FFF70AFB22
:103300000C2CF8D105B030BD6CBF0000F7B56A4693
:10331000394B01AD13801C239370384B2B800A234B
:10332000AB70FFF7DFFA364B364CC0182368984273
:1033300001D2002323602668002E3DD16B469F5D9D
:1033400001213800FFF7E6FA01360021380003F0CA
:10335000A5FA032EF2D10026AF5D01213800FFF758
:10336000D9FA01360121380003F098FA032EF3D17F
:10337000C8200138C046C046C046C046C046C04608
:10338000C046C046C046C046C046C046F1D1002136
:103390002878FFF7BFFA68780021FFF7BBFAA87812
:1033A0000021FFF7B7FAFFF79DFAFA2300251B016A
:1033B000C01820602800FEBDFFF794FA236800259E
:1033C0009842F7D3032003F0F9F80600042003F035
:1033D000F5F836180A2003F0F1F80B4B9B1B181A6E
:1033E0000A4BA84206DB18600023094A23601360D9
:1033F0000125DFE71D60F7E71A1B0000030400004A
:1034000010270000D80F0020E3030000C00F0020A9
:10341000E00F002010B50124044002D04410200029
:1034200010BD0D20FDF792FDF9E700000868F8B522
:10343000C3071AD5FFF7EEFF0300203B5E2B23D80E
:103440000520012258430023104E451DA84217D0E5
:1034500005211024375C3C4200D09B1801395200F2
:1034600064100029F7D10130F0E704280CD90F22AD
:1034700003681A40042A07D11B0905D00079DBE74D
:1034800001205B001843F8BD0120FCE778BF000075
:103490000022054B10B51A60044B1B68934201D003
:1034A00002F034FB002010BDDC0F0020A41A002025
:1034B00070B508680D00FFF7ADFF04006868FFF7FE
:1034C000A9FF621E0100042A14D8451E042D11D83C
:1034D00005236B439B18012215009D402B000648D5
:1034E00005682B430360054B1B68002B02D02000AE
:1034F00002F00DFB002070BDDC0F0020A41A00209C
:1035000070B508680D00FFF785FF04006868FFF7D5
:1035100081FF621E0100042A13D8451E042D10D815
:1035200005236B439B1801229A4007480368934385
:103530000360064B1B68002B03D00022200002F022
:10354000E6FA002070BDC046DC0F0020A41A00205F
:10355000F0B5050089B008680C00FFF75BFF069026
:10356000022D36DD6068FFF755FF0190A068FFF778
:1035700051FF04000127231D661E0793731C02934D
:10358000079B9E4235D0052373430593019B019D04
:1035900005330493049BAB421ED0042E16D86B1E39
:1035A000042B13D80122059B2349013B5B199A4048
:1035B0009446224A0B681068069A3A4003920DD04E
:1035C00062461A430A60012200280DD17F000135AE
:1035D000E0E701240194CDE7029ECFE762469343E2
:1035E0000B600028F2D0039A0299280002F08FFAAB
:1035F000ECE7019B1E1D042E1AD8012C18D10025C2
:1036000005273B0021006B439B1999400B000A4A98
:10361000013511689943094B11601B68002B05D0D7
:10362000019B0022581D290002F071FA052DE8D1F6
:10363000002009B0F0BDC046DC0F0020A41A002015
:1036400010B5041E10DA00240A4BA400E25801232E
:103650009340094A09491360094A1160094A0A4915
:1036600011600A4A136010BDFFF752F9A042EADD6B
:10367000EAE7C046ECCB0000D40F0020080500505C
:10368000CC0F0020C80F00200C050050180500507A
:103690002B4BF7B51B680C00002B03D101204042D7
:1036A000FFF7CEFF24680126250035401AD0FF22FF
:1036B0006310120260121040DAB21043FF221B02A4
:1036C0001204134018431F4B1B68202B06D1B44033
:1036D0001D4BA40EA400E35800021843FFF7C8FDD9
:1036E0000020FEBD042CFBD90F2322681340092BB8
:1036F000F6D1FF2763683F025B100193019B9D4257
:10370000EEDAAB00E3189B68334216D05A10581219
:10371000D1B238400843FF21120209040A40104385
:10372000084A1268202A06D15B009B0E06499B00BE
:10373000020258581043FFF79BFD0135DEE7C046F3
:10374000D40F00200C00002054C1000002000868C3
:1037500010B5C3070FD540101823012A03DD4A68AE
:10376000042A00D10833054A1360FFF7F3F8FFF786
:1037700067FF002010BD01204042EDE70C00002053
:10378000086810B5C30703D5FFF744FE054B186062
:10379000054B1B68002B03D0024B186802F0B8F9E8
:1037A000002010BDDC0F0020A41A00207FB5A04C23
:1037B0002368002B0AD19F4A1268002A06D19E4B2B
:1037C0001B68002B01D0FFF7A1FD7FBD9B4D2A6830
:1037D000002A26D1984A1268002A1BD0FFF796FDCE
:1037E0000028F2D0FFF77EFD924B24681A681C6017
:1037F000002A16D0002C14D101AD0C2290492800CB
:1038000006F03AFE285D00210134FFF783F80C2C06
:10381000F8D1DAE7874A1268002AE5D1002BE3D015
:10382000E0E700211A2003F039F800211B2003F003
:1038300035F800211C2003F031F82E68012E5CD0F1
:10384000022E00D1A2E0002E50D101363100794C79
:1038500003202368994303F021F8042021680140E4
:103860004B42594103F01AF8102123680A201940ED
:103870004B42594103F012F8802123680901194095
:103880004B425941062003F009F8802123680902C0
:1038900019404B425941072003F000F8802123686A
:1038A000490219404B425941092002F0F7FF80219B
:1038B0002368890219404B425941192002F0EEFF5A
:1038C00080212368C90219404B425941182002F057
:1038D000E5FF802321681B0319404B425941172003
:1038E00002F0DCFF31001A2002F0D8FF2B68032120
:1038F000581C04F07FFD296067E702214D4C17201A
:10390000236819404B42594102F0C8FF082123683F
:10391000182019404B42594102F0C0FF8021236812
:10392000C90019404B425941042002F0B7FF8021E1
:103930002368490119404B4259410A2002F0AEFF69
:1039400080212368C90119404B425941032002F0EC
:10395000A5FF80212368890319404B425941092062
:1039600002F09CFF802321681B0419404B425941FF
:10397000192002F093FF3100062002F08FFF310082
:10398000072002F08BFF31001B20ADE72021294CDE
:103990001720236819404B42594102F07FFF402114
:1039A0002368182019404B42594102F077FF8021CB
:1039B0002368192019404B42594102F06FFF8021C2
:1039C0002368490019404B425941092002F066FF23
:1039D00080212368890019404B425941072002F099
:1039E0005DFF80212368890119404B42594106201F
:1039F00002F054FF80212368490319404B4259418A
:103A00000A2002F04BFF80212368C90319404B4272
:103A10005941032002F042FF802321685B041940D2
:103A20004B425941042002F039FF01211C205BE781
:103A3000DC0F0020D00F0020E00F0020C40F00207A
:103A40006CBF0000012010B54042FFF7F9FD10BD2A
:103A500010B5034A0921034800F086FF10BDC04697
:103A600054C200009CC2000030B502248025094BDE
:103A7000094AED009C505C59002CFCD0A124E400C4
:103A8000884202D30021995030BD8025ED001851A5
:103A90004019F5E700E001400405000010B50028DA
:103AA00006D1C020B02140028902FFF7DDFF10BD22
:103AB000B02080218002C902F7E70000434258414C
:103AC000064B40421840B0239B02C01803680020F8
:103AD0001A0E532A01D11B02180A704700C0FEFFBC
:103AE00030B501248025054B054AED009C505C59FA
:103AF000002CFCD001600021995030BD00E0014055
:103B00000405000043425841074B40421840B0238F
:103B10009B02C018A62310B50902DB05090A194348
:103B2000FFF7DEFF10BDC04600C0FEFF70B50124E8
:103B300080250D4B0D4EED009C515C59002CFCD0A6
:103B4000002902DC00229A5170BD557814782D02AC
:103B500025439478013924042543D478043224067B
:103B60002C4310C0ECE7C04600E001400405000013
:103B700070B505004B680A009C1C2100A400FFF7EB
:103B8000D5FF281970BD0000134B1B68002B0CD00B
:103B90008022B023D2029B0200280BD11A1D5B6841
:103BA0001B0E522B00D110007047B022C02392028E
:103BB0005B02F1E782420DD903681B0E522B09D13B
:103BC000436802339B00C018824203D903681B0E6E
:103BD000522BE9D00020E7E7E410002070B5002068
:103BE000FFF7D2FFFF260500002801D1280070BD95
:103BF00003681C143440FFF7C7FFDA2CF4D105002A
:103C0000F2E700008022F0B55200A1B00021674821
:103C100006F04EFC802200215200654806F048FC68
:103C2000644BFF271B681A00049353425A4110004B
:103C30000592FFF733FF049C0020631E9C415E4BFE
:103C400064421C405D4BE418FFF7C8FF0600002EDD
:103C50002DD10498FFF732FF411C0598FFF752FF62
:103C6000059A574D534B2C601A60FEF7C7FF514B16
:103C700064201B68A0215A4253414F4A5B421340C3
:103C8000B0222C6892029B18E41A6043490204F0A7
:103C9000CBFAA0225202030000924A49220007A850
:103CA00006F04AFF07A801F07DF821B0F0BD3268A8
:103CB000131412123A403B4003921A000A3A092A9E
:103CC00049D83A4B039A995C002931D110223E48D9
:103CD00006F0EEFB35002B6803991A123A40914228
:103CE00009D11A143A400B2A27D0132A2DD00A2AB8
:103CF00001D1354B1D602800FFF746FF051EEAD1B4
:103D0000314B196800290FD02000FFF731FF040064
:103D10002D4B5B195968002903D02000FFF728FFBD
:103D2000040004350C2DF3D1204B0121039A995442
:103D30003000FFF729FF060089E73B40022BDADC61
:103D4000214A9B00D3185D60D5E7102200211E4850
:103D500006F0AEFBCFE71A00153A082AE8D8144A55
:103D60000399525C002AE3D13500152B00D01500D1
:103D7000300003681A143A40152A0FD01D2A00D1CA
:103D80000025FFF701FF0028F3D1002D04D020000B
:103D90002900FFF7EDFE0400054BC6E7039A1B124E
:103DA0003B409A42EDD10500EBE7C046E40F00200E
:103DB000EC100020E410002000C0FEFF04C0020050
:103DC000E810002035C30000E02E0020F0B50020F0
:103DD000B7B00024FFF7D8FE270005002600002D0D
:103DE0002ED1284D2868FFF769FE32003B00019074
:103DF0000094254904A806F09FFE04A800F0D2FF15
:103E0000224B64201C682B68A0215A425341204A4F
:103E10005B421340B02292029B18E41A60434902AD
:103E200004F002FAA0225202030000921949220073
:103E300004A806F081FE04A800F0B4FF37B0F0BD7E
:103E4000FF226B6829689C460233FF180B1201366B
:103E500013409C4200DA1C00FF200A140240039227
:103E60006246014001920091039A0B4904A806F0B2
:103E700063FE04A800F096FF2800FFF785FE05000A
:103E8000ADE7C046E4100020A6C30000E810002003
:103E900000C0FEFF50C3000092C3000070B50020B8
:103EA000FFF70CFE04000120FFF708FE844200DA51
:103EB00004000A4B1D686A42554128001D60FFF747
:103EC000EDFDA0226B4252021340054A28009B18C8
:103ED000044A611C1360FFF715FE70BDE41000205A
:103EE00004800100E8100020F8B50020FFF7E6FD8F
:103EF00007000120FFF7E2FD3E00204D0643204C65
:103F00000DD18021C020C9024002FFF7ADFD012183
:103F10003000FFF7F7FD1B4B2E6023601DE087424A
:103F200009DD0023B0212B60164B89022360236832
:103F30000020012517E0012380212B60124BC902CC
:103F40002360F4E7120E522A08D0002800D0236024
:103F50000E4800F027FFFFF7A1FFF8BD28005A68C0
:103F6000023292009B188B4205D21A68561CE9D186
:103F70000028F2D0D1E72160EFE7C046E41000202E
:103F8000E81000200480010004C002006BC30000A0
:103F9000F0B585B0039203220333DC17294D14409A
:103FA000E4182B68284F5A42534180225B42D202C8
:103FB000A4103B409B18A21C0291244E910000913A
:103FC0000190316800980A18934215D2FFF71AFE43
:103FD0002B685A42534180225B421F40D202BF18D5
:103FE0003368009A9B189F4206D2194800F0DAFE07
:103FF0000025280005B0F0BD029B356819066B4608
:104000001A7BA423DB051343FF222F00090C19435D
:10401000019B12041B04134019432800FFF760FDA5
:104020000837281D21003760FFF75AFD002C04D007
:104030000A9A21003800FFF779FD009B083BFF1822
:104040003760D6E7E410002000C0FEFFE810002033
:104050000FC3000010B5FFF7D5FD10BD70B59AB0C5
:10406000FFF742FFFF221E4CD2000021200006F085
:104070001FFAFF25FFF7B2FD0026002814D1020029
:10408000C300E3580130591E8B41D218FF28F7D1E5
:10409000144901A806F050FD01A800F083FE124863
:1040A00000F080FE1AB070BD03681A142A400A2A74
:1040B0000AD11A122A40FF2A03D0D200A1180B718C
:1040C000A050FFF761FDD8E7132AFAD11B122B404D
:1040D000FF2BF6D0DB00E2181671E650F1E7C04680
:1040E00058250020DBC30000EFC300000021094B6E
:1040F000094A59600131516059680029FCD00021FA
:104100001961012393600222044B8131FF315A501F
:104110001A607047FC1000400010004000E100E011
:104120000222064B0121DA670022054B5A61054A3B
:1041300011615A69002AFCD07047C04604E100E0D2
:10414000FC1000400010004010B5044C2378002BF8
:1041500001D0FFF7E5FF0020207010BDED11002019
:104160000120024B1B685B0018437047701200204F
:1041700003480368002B02D11422037102607047C8
:10418000082F00200120024B1B685B00184370477A
:104190001000002070B504000D001600FEF7ACFB07
:1041A0008023012200215B055B6E6270E270020ACF
:1041B000A271020CE2711A0A60716372000EA2729F
:1041C0001A0C1B0E26702571A1702072E2722373E7
:1041D00070BD0000124B10B51B68124C5A1C0FD05A
:1041E000114C002B0CD0114C012B09D0104C022B80
:1041F00006D00D4C042B03D00E4C052B00D10B4CDC
:1042000021000D4806F0D0FC200006F0D5FC03008C
:10421000042204339B0809481B011343036010BDAB
:104220001400002077C4000070C4000082C40000A5
:1042300087C400007CC40000F42E0020F02E002073
:1042400070B5214C2278002A3DD1204B01215A60C3
:104250008022D20511605A68002AFCD00022072073
:104260001B4B1C4901255A500439585008315A50EB
:1042700019481A4958501A491A485A501A495A5056
:10428000A622D2009D50082218495A500431585095
:1042900002201749585017491748585017480439F1
:1042A0005850182016495850C12189005A500539D4
:1042B000FF395858921802435A501249124A9950DD
:1042C000FFF714FF257070BDED110020FC000040C9
:1042D000001000400C050000746962751C050000A8
:1042E00024050000200004022C0500001405000035
:1042F000340500003C050000FFFF00002110010014
:1043000054050000EE1100200405000070B50E4BAE
:1043100006001B78002B01D1FFF792FF00200B4D08
:104320002C7884420ED00A4B202219780323091BD3
:104330001940084B4901C918300006F09DF80120CA
:10434000013C2C7070BDC046ED110020741200209D
:10435000EC110020EE110020002370B588B09842C7
:1043600027DD0D6801262C0034409C4221D123001A
:10437000042D1ED90F222B681A402300092A18D1B8
:104380006A681F2A15D96846FFF7C0FF2300002876
:104390000FD06B4619783300A14203DB6B461B5DDF
:1043A0005B003343A200AA1801349360202CF2D1A1
:1043B0000423180008B070BD70B5414B8AB01B785B
:1043C000002B01D1FFF73CFF02AD2800FFF79EFF55
:1043D000002802D100200AB070BD2B780B2BF9D930
:1043E0006B78012BF6D1EB78012BF3D10023354EFE
:1043F000354C336023712B79344A1360002B0ED176
:10440000152169444A780B7812021A438B781B04F1
:104410001A43CB781B0613433360002318E0012BAB
:1044200020D1152169444A780B7812021A438B78FF
:104430001B041A43CB781A211B06134333600E2347
:104440006A7C6944934200DD130000229A4232D113
:1044500004200021E21804339B101B010343117157
:104460002360B8E7022B03D16A7B10331621E8E7FB
:10447000042B0DD1152108226944684605F0FCFF84
:104480000098019902F07CFA05F0A8FE3060C4E7BC
:10449000052BC2D1152108226944684605F0ECFFBE
:1044A0000098019902F06CFA05F098FE30606A7D80
:1044B0000A231E21C5E78D5CA01805710132C5E7EE
:1044C000ED11002070120020082F002014000020A1
:1044D00010B5134B04001B78002B01D1FFF7B0FE81
:1044E000FFF71EFE00200F4A0F49104B5450586032
:1044F0000130106058680028FCD00020186101309D
:10450000906018690028FCD0094B0A481B785B01B1
:104510001B185350FFF704FEFFF7E8FD10BDC0461F
:10452000ED1100200010004004050000FC100040C8
:10453000EC110020EE11002010B588B000281DDD20
:104540000A68012113000B4018D1042A16D90F2044
:1045500014682040092811D150681F280ED99800EE
:10456000101880680024084201D04010C4B2684688
:10457000C4540133202BF2D1FFF7AAFF002008B06A
:1045800010BD000010B5002813DD0C68E30710D53E
:104590006410532C0DD8084B1B78002B01D1FFF76A
:1045A0004FFEFFF7BDFDA123044ADB00D450FFF707
:1045B0009DFD002010BDC046ED1100200010004000
:1045C00010B500280EDD0C68E3070BD56410FF2C36
:1045D00008D8054B1B78002B01D1FFF731FE034AA9
:1045E000034BD450002010BDED11002000100040FE
:1045F0002405000013B5002814DD0C68E30711D56D
:10460000094B64100093094B0193072C0AD8084BFF
:104610001B78002B01D1FFF713FE6B46054A195793
:10462000054BD150002016BDE2ECF0F4F8FC00047C
:10463000ED110020001000400C05000070B588B09E
:10464000002820DD0124086804401CD104281AD960
:104650000F2302681340042B15D1FEF745FB06001B
:1046600006F0AAFA0500122800D912252A00022114
:104670000D326846FFF78EFD6B465D73A54205DC83
:104680006846FFF725FF002008B070BD2300325DAB
:104690006B449A730134F1E7F0B50D008BB001283B
:1046A00032DD08680122040014402DD104282BD9E2
:1046B0000F2301680B40042B26D16B68134223D0D3
:1046C000FEF712FB6E6807007310019306F074FA90
:1046D00005000E2800D90E252A000121113202A85A
:1046E000FFF758FD6A46127902AB5A7302AA731299
:1046F0009373019B76141B0ED67313745574A542E5
:1047000005DC02A8FFF7E4FE00200BB0F0BD3A5D27
:1047100002A963189A740134F1E730B589B0002812
:1047200014DD0C68E30711D5102268460021FFF75D
:1047300031FD6B466A4665105D73684663122D0E47
:1047400064149373D4731574FFF7C2FE002009B08C
:1047500030BD0000174B184A5968002903D00021CA
:10476000596001319160196900291FD0002018613A
:104770008023DB00D3581149012B18D1A923DB007A
:10478000D3585B420B600E490B78032B01D80133E1
:104790000B7003200B490B78013303400B700A495F
:1047A0005B015B180949535001239360704708600F
:1047B000FAE7C046FC100040001000401000002046
:1047C00074120020EC110020EE11002004050000FE
:1047D00010B5034A0E21034800F0C6F810BDC046CC
:1047E00000C40000F7C30000044A05491368C85418
:1047F00001339B059B0D13607047C0469016002047
:104800009012002070B5114C114A2368834202DCDB
:104810000023236016E0155C411C2E00FA3E012E99
:1048200005D899420FDA555C013D1F2D01D90800CA
:10483000ECE70100151A565C6E5401318B42FADC2C
:10484000181A206070BD1570FAE7C0469C1A002047
:104850009C16002010B5FEF745F8064B1A688242F8
:1048600001D900221A601B68C31A0348984280418C
:10487000404210BD8C120020204E000010B5094CA3
:10488000094A23681268934200D110BD074AD05CE0
:10489000FEF7ACF90028F8D0236801339B059B0D87
:1048A0002360ECE794160020901600209012002060
:1048B00010B50400064B074A1B6812689B1ADB43BD
:1048C0009B059B0DA34200DB10BDFFF7D7FFF1E76F
:1048D000901600209416002070B50020FFF754F9C0
:1048E000FF260500002801D1280070BD03681C14B4
:1048F0003440FFF749F9DA2CF4D10500F2E7F7B5B7
:10490000050056680191B000441C06301700FFF7FF
:10491000CFFFFB20FFF768FF1C20FFF765FFE8B221
:10492000FFF762FFE0B22412FFF75EFFE0B2FFF78D
:104930005BFF6B461879FFF757FF0025AE4200DC9E
:10494000F7BDAB00FB189C680135E0B2FFF74CFFE8
:104950002012C0B2FFF748FF2014C0B2FFF744FF97
:10496000200EFFF741FFE9E770B5074E3368092BCA
:1049700008DC0C255D43054C013328516419616046
:10498000A260336070BDC046981600202C2F002016
:10499000F0B587B002900C00012803DC1B20FCF767
:1049A000D5FA45E0244B08680093C30709D40428CE
:1049B00007D90F2302681340042B02D1FEF794F9A4
:1049C00000901D4B60680193C30709D4042807D9E0
:1049D0000F2302681340042B02D1FEF785F90190E2
:1049E0000027164B1B680493049BBB42D6DD0C26A4
:1049F0007E43134B0099F618306806F0CBF8051E7D
:104A000005D17368B6680593059B9D4201DB0137AC
:104A1000EAE730680199039606F0BCF808360028EA
:104A200008D121000298039B083102385B6898473F
:104A300007B0F0BD0135E7E76FBE00009816002013
:104A40002C2F002010B5FCF7CDF9FFF701F8FEF789
:104A50006FF8FEF7BDFBFEF7F3FBFFF7B9FE00F0C2
:104A60007DFE01F057F810BD962210B5120100210D
:104A7000034805F01DFD0022024B1A6010BDC04620
:104A8000F81B0020B8050020064B074A1B68126877
:104A90009B1ADB439B059B0D0122834200DC002215
:104AA000100070479016002094160020F8B50500FD
:104AB0000C0016001F1E0ED10320FFF7E5FF002893
:104AC00008D0FA20FFF790FEE8B2FFF78DFEE0B2C3
:104AD000FFF78AFEF8BD501DFFF7D6FF0028F9D07A
:104AE000FB20FFF781FEE8B2FFF77EFEE0B2FFF7A2
:104AF0007BFEF0B2FFF778FE3012C0B2FFF774FE13
:104B00003C00E31B9E42E5DD2078FFF76DFE01349B
:104B1000F7E7000070B50024F0250B4B1B68A3429B
:104B200002DCFFF7A1FF70BD2B006343074A9B180F
:104B30001A78002A05D05978002311201A00FFF7AF
:104B4000B5FF0134E9E7C046B8050020F81B002096
:104B5000F8B507000024F0252B0063430C4A01340C
:104B60009E18B74211D0317800290BD00133D15CA7
:104B7000002311201A00FFF799FF2A0000213000BE
:104B800005F096FC0A2CE7D1F8BD024B1C60F9E752
:104B9000F81B0020B8050020F0B5150001222F00F9
:104BA0005E4C1740A54401900291002F11D005AB37
:104BB0001A706A105A70120E1A71052269129970D1
:104BC0006D140299DD70FFF771FFCF239B009D44A8
:104BD000F0BD042D1ED90F232A681340042B25D1C4
:104BE000023B04AA28001371FEF77EF8040005F0CA
:104BF000E3FF4B4B984200D91800B84204DC421C3A
:104C000005AB02990198DEE701377B1EE35C05AA3C
:104C1000D355F2E7042D7CD1032304AA043D13717C
:104C20006B425D4105AB55710222EAE7092BCCD1FD
:104C3000042205AB1A706A6851100091694652123D
:104C400009789A70009A59701F2A01DD202200927B
:104C50006A46127806ACDA70009BBB4202DC05ABF8
:104C6000E21ACEE70126BB00EB189868064006D191
:104C7000042837D90F2302681340022B0CD10123DB
:104C800023704310637042121B0E4014A270E07038
:104C9000237105340137DFE7042B21D1023B237058
:104CA000FEF722F8039005F087FFA31C0C2809D813
:104CB0006070864201D19C19ECE7039A925D9A5587
:104CC0000136F6E70C226270039A925D9A5501361E
:104CD000092EF9D12E23E372237363730E34D9E7BF
:104CE000012B07D1032304382370434258416070DD
:104CF0000234CFE7092B09D1053B23704368E670E6
:104D00005A105B126270A3700434C3E7267001343A
:104D1000C0E7002D00D058E77EE7C046C4FCFFFF87
:104D20002303000070B502000024F0210D4E08009E
:104D3000604380194578954203D001340A2CF6D19E
:104D400070BDF022002105F0B3FB074A1368013B58
:104D5000A34200D11460002329001A001120FFF79C
:104D6000A5FEEDE7F81B0020B805002010B5B2B095
:104D700002236A460400137005F01EFFC72800D9FD
:104D8000C7200023984207DC421C6B46FE211420FA
:104D9000FFF78CFE32B010BD694601335A1EA25C8B
:104DA000CA54EFE730B5B3B002236A46050013706A
:104DB00005F002FF0400C72800D9C72400239C4245
:104DC0000BDC20003230FFF773FD621C6B46FF21C5
:104DD0001420FFF76BFE33B030BD694601335A1E15
:104DE000AA5CCA54EBE70000F7B5234B06001B682A
:104DF000F02100930023009A9A4211DC0024F02352
:104E00001A006243019201991C4A55182F78002F0D
:104E100012D001340A2CF3D11948FFF7C3FF29E05F
:104E20000A005A43154882185078B04202D11278CD
:104E3000002A1FD10133DEE7F0223900280005F0F7
:104E400037FB02230D4A0199EB6053540D4AF100E0
:104E50008A58009B6E70AE70AA602F616F61A3428A
:104E600002DC054B01341C60002331001A001020C5
:104E7000FFF71CFEF7BDC046B8050020F81B002058
:104E800071C900005825002010B5FFF743FEFF242C
:104E9000084AE3005B429B18074AD35C043B012BA2
:104EA00003D8E043C0B2FFF79FFF013C002CEFD1D5
:104EB00010BDC046FC07000058250020F7B50F00C4
:104EC000FF247F2501901E4AE300D31A1D4A9A1839
:104ED0001278062A01D0032A20D1FF22D2009B1883
:104EE000186883682B401C2B18D1C3681A002A400D
:104EF000042A13D102692A40192A0FD11B0A01334F
:104F00009B000C30C018FDF7EFFE03780600002B65
:104F100010D005F051FE0023B84209D0013C002C0E
:104F2000D1D1F7BD019AF15CD25C9142F6D1013347
:104F30009F42F7DCE043C0B2FFF756FFEEE7C04602
:104F400058250020FC07000070B50500FF24084A22
:104F5000E3005B429B18074AD35CAB4203D1E043BA
:104F6000C0B2FFF741FF013C002CF0D170BDC0463C
:104F7000FC07000058250020F7B5FDF7B3FC514BA6
:104F80001A68824201D900221A601A684E49821AB0
:104F90008A4200D883E01860FDF7AEFC071E00D1FE
:104FA00001370020FDF79AFD01900020FDF7AAFDD2
:104FB000019B0090454C464D002B14D02368002BDC
:104FC00000D07AE02B682760002B00D171E0414BC4
:104FD00001261B78002B63D10920FFF7B5FF3E4B5C
:104FE0001E703C4B1E70009B002B12D02B68002BB8
:104FF0000FD123682F60002B1ED0374B01261B7862
:10500000002B52D10920FFF79FFF334B1E70314B0D
:105010001E702368002B0FD02F4E3278002A0BD140
:105020009F4200D227602368FB1A312B04D9072046
:10503000FFF78AFF012333702B68002B0FD0254E1A
:105040003278002A0BD1BB4200D92F602B68FF1A9F
:10505000312F04D90820FFF777FF0123337023682D
:10506000002B0CD0019B002B09D11B4E3378002B59
:1050700002D10720FFF768FF0023236033702B68FD
:10508000002B0CD0009B002B09D1124C2378002B55
:1050900002D10820FFF758FF00232B602370F7BDD3
:1050A0000720FFF751FF0C4B9CE70820FFF74CFF50
:1050B000ADE7009B002B9CD1ABE7009A002A95D16D
:1050C000AAE7C046881200200F27000078120020AF
:1050D00080120020841200207C12002037B50024AA
:1050E0000500FFF717FD01A80194FDF7E5FC21007D
:1050F0002000FEF7CDF9FEF759FBFDF717FDFDF790
:1051000016FDFEF79FFCFDF713FCA54204D0FDF74A
:1051100097FD0248FFF746FE37BDC04662C9000052
:10512000002310B501001A001120FFF7BFFC10BDCD
:1051300007B56B46197069465A7013128B701314B9
:10514000120ECB700A716B46010005221320FFF787
:10515000ADFC07BD10B50A0001001220FFF71CFDD1
:1051600010BD70B5050008000C003230FFF7A0FB41
:105170002B00220000211B20FFF798FC70BD10B50A
:105180000C000300110014202200FFF78FFC10BD5B
:10519000012370B5FF24084A41185B42884201D3BD
:1051A000D84370BD06781D0A234073409B009B586E
:1051B00001306B40F2E7C04644C50000002313B540
:1051C00001930B4BC2000400D058002805D043685F
:1051D00008309900FFF7DCFF01900920FFF768FB1A
:1051E00001AB042221001720FFF760FC13BDC0466D
:1051F00058250020F7B50190FFF76EFB012504004C
:10520000FF276D42002C01D12800FEBD2668331413
:105210003B40152B0DD121000198083105F0BAFC57
:10522000002801D135123D402000FEF7ADFC0400FE
:10523000E8E71D2BF8D101256D42F5E7F0B5802791
:105240009DB0FFF71BFBA54CA54D2068FF00391A48
:105250004019FDF7B1FC23680600C3182360002B3A
:105260000ED11DB0F0BD2068391A2818FDF7A4FC36
:10527000236806001B182360FDF734FB994B186068
:10528000002EF0DC2B78FA2B00D037E12368022BBC
:1052900007DCFFF7DFFA0028E3D00120FFF7B2FABE
:1052A000DFE76878AC78023818282BD802F028FF9E
:1052B00019002C0030003400370040002A004A005A
:1052C0007C0086008A00A000F10002012A002A006A
:1052D0002A002A002A002A002A002A002A002A007E
:1052E0001001FF2C0ED02000FFF71CFD00227E4B8A
:1052F000E100CA505B181A712100009213001320BC
:10530000FEF746FE0320C9E72000FFF76DFDF9E731
:105310002000FFF707FDF5E7FFF7B6FDF2E7FFF71F
:10532000F9FB0020FFF7DAFE7048FFF73BFDE9E7E5
:10533000632CE7D86E4BA200D25821001520FFF74E
:105340002BFCDFE7FFF7C8FAFF270400002CD9D0B9
:1053500025682B143B40152B04D02000FEF714FCCD
:105360000400F3E72000083005F026FC06000530B5
:10537000FFF79EFAFB20FFF737FA2D121D20FFF7EB
:1053800033FAE8B2FFF730FAF0B2FFF72DFA301235
:10539000C0B2FFF729FA25002B1B9E42DDDD287ADB
:1053A000FFF722FA0135F7E700211D2000910B00DD
:1053B0000A00FEF7EDFDFDF743FCA3E72000FFF731
:1053C000FDFE9FE7FDF7A0FA03AC4A4A6421009076
:1053D000494B200005F07EFB02232000237005F0DE
:1053E000EBFB2300020000211620FFF75FFB89E79B
:1053F00000243D4AE300D558002D27D06B689E005D
:10540000701DFFF755FA2B000025320008332100EC
:105410000120FFF74BFB2F00FFF75EFA2E0000285C
:1054200018D1002F04D03A0001212000FFF767FABD
:10543000002D04D02A0002212000FFF760FA002E80
:1054400004D0320000212000FFF759FA0134FF2C6C
:10545000CFD157E7FF2103681A120A40A24209D1AF
:105460001A140A400B2A08D10B400CD0012B0CD087
:10547000022B0CD0FEF788FBD1E7132AFAD10025C6
:105480002F002E00F6E70600F4E70700F2E705001C
:10549000F0E70024FFF73EFB2200210000942300E8
:1054A000DA20FEF775FDFF222100D2000E4804F03D
:1054B000FFFF80E7012C02D1FEF788FC22E7022CD7
:1054C00002D1FEF7C7FD1DE70120FFF707FE19E730
:1054D000002321001A001A2087E7C0469C1A0020EA
:1054E0009C1600208C1200205825002044C9000082
:1054F000502D00205BC9000056C90000FB2B00D0D6
:10550000CBE62268042A00DCC3E62E79E878574B04
:10551000360206439E4200DDBFE6331D9A4200DCA0
:10552000B7E6EB5CFE2B00D0B7E66B78AC78771E65
:105530001B2B61D019D8072B47D0082B1CD0012B6F
:1055400018D1FF2C16D02000FFF7ECFB6D79484AEC
:10555000B31E009221002A000A20FEF719FD454BD8
:10556000E400E0501B191D7104E01D2B56D048D3F8
:105570001E2B6AD0701D91E6632CFBD86A79022A33
:1055800013D0032A1BD0012AF4D1E979AB7909029F
:1055900019432B7AA4001B0419436B7A1B060B4397
:1055A0005B001343344AA350E4E7002FE2DDB11E51
:1055B0002F48FDF7A7FD304BA400E050DAE7AB79A8
:1055C000A4005A1E93419B00ECE7632FD2DC03AD8D
:1055D0003A002A49280004F04FFF00232800EB5529
:1055E000FFF708FE0028C5DB234B8000C2582100CE
:1055F0001520FFF7D1FABDE739002048FFF75EFC20
:10560000B8E7FF2CB6D06A79022AB3D818490B2024
:1056100000912100B31EFEF7BBFCABE7632F00DD5A
:105620006327002303A99F420ADCFB430022DB1708
:105630003B40CB181A70152000917B1C2100EAE733
:10564000EA185279CA540133EDE7012C92D1002FA8
:1056500090DD6B79002B03D01C00322B00DD32244F
:1056600064235C43064B1C6084E7C046F6030000DD
:10567000A216002058250020502D0020A116002041
:10568000040000200122094B1A60094A1368002B0C
:10569000FCD00322074B1B68D8171040C018012309
:1056A00080100638400018437047C04600C00040D4
:1056B00000C1004008C500400120704710B5064CED
:1056C000200000F05DFB0549200000F081FB012275
:1056D000034B1A6010BDC046C81A0020801A06008D
:1056E000A01A002010B501210D20FDF713F90121AA
:1056F0000E20FDF70FF900210F20FDF70BF9044CE8
:10570000200000F079FA1021200000F091FA10BD7D
:10571000A81A002010B504680D20E30703D5641013
:10572000FF2C03D91720FBF711FC10BDFFF7DAFFA0
:10573000E1B2024800F09EFA0020F6E7A81A002025
:1057400010B5FFF7CFFF0021034800F093FA4300A4
:105750000120184310BDC046A81A002010B5034A06
:1057600008210348FFF700F910BDC04688C90000B2
:10577000C8C900000D4B70B51B6804000E00150071
:10578000002B01D1FFF79AFFE1B2094C200000F095
:10579000B6FBF1B2200000F0B9FAE9B2200000F047
:1057A000B5FA200000F016FC70BDC046A01A00201B
:1057B000C81A002010B501240368234205D04168AF
:1057C000214202D08268224203D10D20FBF7BEFBAA
:1057D00010BD5810802801D91520F7E74910FF297E
:1057E00001D91620F2E75210FF2A01D91720EDE760
:1057F000FFF7C0FF0020EBE7F7B501242300A0422C
:105800001DDD0D682C421AD01A4B25411B684C68CF
:10581000002B01D1FFF752FFE9B201272500164EF8
:105820003D40300000F06BFB002D0AD03C413000C1
:10583000E1B200F06BFA300000F0CCFB002318005E
:10584000FEBD042CF7D90F2322681340092BF2D197
:1058500063685B100193019BAB42ECDDAB00E31886
:105860009968394204D04910C9B2300000F04EFAAC
:105870000135F0E7A01A0020C81A0020144B70B5BB
:105880001B6805000E00002B01D1FFF717FF114C1C
:10589000EDB22900200000F032FBF1B2200000F050
:1058A00035FA0021200000F035FB002801D04042ED
:1058B00070BD01222900200000F01CFB200000F038
:1058C00016FA0028FAD0200000F016FAF0E7C046D9
:1058D000A01A0020C81A002010B501240368234232
:1058E00002D04168214203D10D20FBF72FFB10BDF0
:1058F0005810802801D91520F7E74910FF2901D950
:105900001620F2E7FFF7BAFF40002043EFE7000060
:10591000002370B5344D0400EB5601330BD10D213B
:105920001D20FFF7ABFF5A2814D101222A212A702B
:105930003D38FFF71FFF0023EB56022B2AD0032B25
:1059400049D0012B4CD121001D200124FFF796FFE7
:10595000644225E00F211920FFF790FF332805D17D
:1059600002235F222B7020211A38E2E70D211E202E
:10597000FFF784FFC7280AD1032300222A21A93870
:105980002B70FFF7F7FE1B222A211E20D1E70023F0
:105990002B70D0E7012C13D129211920FFF76EFFBE
:1059A0007F2801DD0138FF3803007F3301DA7F20D3
:1059B000404264237F21584302F036FC604370BDAF
:1059C000032C0BD12B211920FFF758FF043CE7E7EC
:1059D0002D211920B9E721001E20B6E7052CF7D0AC
:1059E000012400206442E4E71800002070B5012083
:1059F000FFF78EFF04000320FFF78AFF0500052054
:105A0000FFF786FF6D43644340436419201804F098
:105A10001BFC01F0E5F804F0E1FB43000120184312
:105A200070BD10B50120FFF773FF4300012018433C
:105A300010BD10B50320FFF76BFF43000120184392
:105A400010BD10B50520FFF763FF43000120184388
:105A500010BD0000F8B501231C00984234DD0F682A
:105A60003B4231D04E6835001D402DD1042E2BD93C
:105A70000F2231680A40092A26D173685C10202C55
:105A800000DD2024114B1B68002B01D1FFF716FE0F
:105A90007F10F9B20E4F2200380000F02BFAA54219
:105AA0000FDA380000F023F90028FAD0380000F0AF
:105AB00023F90122AB004000F31810439860AD18A1
:105AC000EDE70120640004432000F8BDA01A002087
:105AD000C81A00200020704701207047002070473E
:105AE0000020704701207047002070470020704759
:105AF000002070470020704700207047002070474A
:105B000000207047002070470020704770477047A2
:105B10007047000010B5034A0E210348FEF724FF2A
:105B200010BDC04618CA000088CA000010B5FDF7B5
:105B30000BF8FDF7ABF8FEF785FF0448FFF732F9E5
:105B4000FEF78CFAFFF7A0F910BDC04611CB00009C
:105B500010B5FCF761FE10BD70B5002504AC2478CB
:105B60000573A94205D10A4B0A4A23210A4804F0C9
:105B700015FC01600949920052589B0002715B5864
:105B8000A40083716358856043710223C37170BDA3
:105B900029CB00008ECB000037CB0000ECCB0000FF
:105BA000037B002B04D143738373036101330373BD
:105BB000704700001FB50191A02100240068C900B2
:105BC000D2B24450012A10D0A24209D0032A0AD0EE
:105BD000074A8350074B019AC250012343501FBD0F
:105BE00002221343F4E70422FBE70622F9E7C0464A
:105BF000540500002405000010B50400FFF7D0FF95
:105C0000A1222368A179D20099506179064A200027
:105C10009950217904329950044B19685A689B684D
:105C2000FFF7C8FF10BDC0460C050000BC1A0020DD
:105C30004BB2002B0FDB80233F290FD81F290FD831
:105C40000F290FD807290FD803290FD81B06016881
:105C5000074A8B50704780239B04F8E7DB04F6E784
:105C60001B05F4E75B05F2E79B05F0E7DB05EEE7D4
:105C7000240500000368074A99501A00FC32D168D5
:105C80000029FCD0A321C90058580023C0B2D3601A
:105C90007047C0461C05000007B58022074BD2059F
:105CA0001A6000229A6002321A710F230C3200939C
:105CB0000349023B0348FFF74FFF07BDBC1A002012
:105CC00000300040A81A0020F8B505000E001700AB
:105CD0000024BC4208D02B68315D1B68280098471F
:105CE000002801D00134F4E72000F8BD704710B55A
:105CF0001C3000F0A9F910BD10B51C3000F096F969
:105D000010BD10B51C3000F0A5F910BD70B5437E74
:105D10000D00002B01D1002070BD6430040000F0A4
:105D2000A2F90028F7D12000290000F070F9012025
:105D3000F2E70000F7B50193FA23002504009B0069
:105D400083600D4B4560083303601C300F00160064
:105D500000F052F92000643000F04EF9074A276144
:105D6000B600B35820006375019B9B009B58657675
:105D7000A576A375FEBDC046CCCB0000ECCB0000E1
:105D80000123A022C375837D0E49C133FF33D205A1
:105D90009B009950437DC133FF339B009950CC2227
:105DA0000169094B5204CA5005220169243BCA50BB
:105DB000827D01690833CA500269417D034BD1508D
:105DC0007047C0460C060000240500000C050000CA
:105DD000A022002310B50469D200A3500A4CA142AE
:105DE0000FD90A4C8C425B4109495B420B40CD21E3
:105DF000C9045B1804690749635005210369995078
:105E000010BDCC235B04F5E7A086010090D0030011
:105E1000000098FD24050000F7B5040000200D00E7
:105E20000193824265D01600402A00D940262700FF
:105E30001C37380000F0F6F8B1232269DB00D5509A
:105E400080220123216992008B50A27E002A03D177
:105E500022691362226913600025731EAB4207D1C9
:105E6000019B002B04D080220221236992009950CB
:105E7000012223691A622369FC33DA68002A02D1FD
:105E80009A6A002AF9D09A6A002A0BD1DA60A32311
:105E90002269DB00D1583800C9B2013500F0B7F8EB
:105EA000B542DAD3019B2269002B0FD11300FC33DA
:105EB0009B6A002B0AD10133A376D3612369FC339B
:105EC000DA6C002AFCD00022DA640AE00023012107
:105ED000A37651611A002369FC3399680029FCD02C
:105EE0009A602369FC339A6A002A01D000229A62E0
:105EF000E8B2FEBD10B50123FFF78EFF10BD030011
:105F0000AC3310B504001970643000F08BF8012335
:105F1000637610BD0023020070B5AC3243760D00ED
:105F20001178B12204000069D200815080222169D9
:105F300092008B502269013313622269936026001C
:105F40006436300000F080F8002812D0300000F0F5
:105F50006DF81E4B2269D0502369FC331A6A002A5F
:105F600002D19A6A002AF9D09A6A002A01D11A62EB
:105F7000E5E723690122002D0DD11900FC31896A62
:105F8000002908D1DA612369FC33DA6C002AFCD0DD
:105F90000022DA6407E05A612369FC339A68002A18
:105FA000FCD000229A6000202369FC339A6A824266
:105FB0000BD098622169064A8B588B501800022B2F
:105FC00003D0181F431E9841033070BD1C0500000C
:105FD000C404000010B50121FFF79CFF10BD0000B4
:105FE00010B51323142202490248FFF7A3FE10BD87
:105FF00000400040C81A002010B5402200210400D3
:1060000004F056FA002320002364636410BD10B529
:106010003F24026C531C2340446C9C4201D08154A9
:10602000036410BD0023036443647047436C026C37
:10603000934206D03F21C25C01330B404364100001
:10604000704701204042FBE7036C406C181A00D5F2
:1060500040307047436C026C934201D0C05C704783
:1060600001204042FBE73F22036C406C01331340A8
:10607000181A43425841C0B27047000003210A4831
:1060800002680A430260094802680A43026008493C
:10609000084A094B9B1A03DD043BC858D050FBDC6F
:1060A00000F012F8FAF730F82405004054050040DB
:1060B0003CD100000000002050020020FEE7FEE777
:1060C000FEE7FEE7FEE7FEE72D4B10B51A68D2B2F9
:1060D000012A0FD12B4A126812070BD12A4AE02459
:1060E0001168F0220800104021422DD1274909688B
:1060F00011422CD01A68D2B2012A12D12149096862
:1061000009070ED1F020204909680140402908D133
:106110001E490968014204D18020C121C005C9007F
:1061200042501B68DBB2012B0DD1164B1B681B07BD
:1061300009D1154B1A68F0231A40A02A0FD1134A2F
:1061400012681A420ED010BD3028CFD0D2E7104AC4
:10615000104911608021104A09021160CAE7D02A53
:10616000F1D1ECE70D4B1A68012A04D00C4A1A60F1
:106170001A68012AFCD1C0220A4B1A60E3E7C04624
:10618000E00F00F0E40F00F0E80F00F0EC0F00F07B
:1061900004050040DFFF07C0186C004000EC06401B
:1061A0007593000014EC06400120704710B5036899
:1061B0001322DB69984710BD70470000054B026948
:1061C000D1500369FC331A6A002AFCD00022012056
:1061D0001A6270471C050000030010B55C331A7882
:1061E0001F231A401E3B19009140114AD167C22259
:1061F000042104699200A150026953600269D360CE
:10620000A02300220169DB00CA5001230169094A69
:106210005B428B500169084A8B5001690C3A8B50E4
:10622000016908328B501430FFF7FCFE10BDC046E8
:1062300004E100E00C0500001405000010B5143066
:10624000FFF702FF10BD10B51430FFF703FF10BDBC
:1062500010B51430FFF7EAFE10BD0000030070B562
:106260005E331A780469724BE25003005D331A788A
:106270000469704BE250030061331C7802696E4B75
:10628000012C00D09EE005005F352E78A225ED00A0
:106290005651020060321578A1220669D200B5502D
:1062A0000269D4509623DB00994200D88CE09623F3
:1062B0001B01994200D88AE096235B01994200D8DD
:1062C00088E096239B01994200D885E0E1239B0159
:1062D000994200D882E09623DB01994200D880E001
:1062E000E123DB01994200D87DE096231B0299420D
:1062F00000D87AE0E1231B02994200D877E0962388
:106300005B02994200D874E0E1235B02994200D815
:1063100071E0E1239B02994200D86EE0474B99421D
:1063200000D86CE0E123DB02994200D86AE0E12268
:10633000002312038A425B41414A5B4213408022A0
:1063400052059B1801693F4A8B50A0230422016922
:10635000DB00CA5000210369FC33D9600369FC33B8
:106360001962012301690B6001698B60C121046915
:10637000890062501F215C3002780A4093406231EC
:10638000314AFF3153500021415600293CDA0F2396
:106390000B40083B2D4C9B089B001B1903242140FC
:1063A000A140FC348C40DD69A5432C00C0258D4004
:1063B00029002143D9611F23017819401E3B8B40DE
:1063C000136070BD00246CE79E23DB02BAE79D23B7
:1063D0001B03B7E71E4BB5E71E4BB3E7EC239B034C
:1063E000B0E71D4BAEE71D4BACE71D4BAAE71D4BBD
:1063F000A8E71D4BA6E71D4BA4E71D4BA2E7802392
:10640000DB049FE71B4B9DE78C080F4BA400E418AF
:1064100003230B40FF21C025DB009940AD006659E6
:106420008E433100C0269E4033000B436351C2E7C8
:106430000C050000140500006C05000090D003005E
:1064400000D0BEFE2405000000E100E000ED00E009
:1064500000B013000050270000A04E0000F07500AF
:1064600000509D0000F0EB0000903A0100E0D701E1
:1064700000B0AF0300705F07F7B5009308AB1B785F
:1064800000250193FA2304009B0083600E4B4560B6
:106490000833036014300F001600FFF7ADFD230032
:1064A0005C3327611E70009B084A9B0099582300AB
:1064B0005D331970019B20009B009A5823005E33C6
:1064C000DD701A70FEBDC04670CC0000ECCB000041
:1064D000036910B51A00FC32D2680400002A0AD001
:1064E000A322D20099581430C9B2FFF790FD0022C0
:1064F0002369FC33DA6010BD10B50248FFF7E8FFEE
:1065000010BDC046801B0020162307B50222009351
:106510000249013B0248FFF7AFFF07BD00200040E2
:10652000801B002010B5002801D004F07DFA10BDBA
:106530007047000010B500F011F8FFF7F9FF0120D7
:1065400000F000FAFFF7F2FAFFF702FB024B002B14
:10655000FAD000E000BFF7E700000000C420114BB4
:1065600080001A5810491140C02212020A431A50E2
:10657000C0218022490092025A501A608023A3222F
:106580000021DB05D20099500122F9309A60074BB7
:10659000FF301950C120023180001950403019508D
:1065A0001A60704700E100E0FF00FFFF00100140AB
:1065B000014B18607047C04664000020F7B5002307
:1065C00020285AD8384B8000C258042A5BD007D8FC
:1065D000022A54D055D80423012A09D000234CE0C4
:1065E000062A54D051D31A2A53D002231B2AF5D19C
:1065F0002E4A116808294ED909294FD00A240226AB
:10660000A02001252A4AC00015502A482A4D0768B3
:106610001C20BF0007402948019700685759009087
:1066200027481B0207401F43C02300989B020340DA
:10663000FF2057515759000207401F43019B1F433A
:10664000009B58016023184007433E4356510125E3
:106650001C4B156058680028FCD000205860A1230E
:106660000125DB00D3585560A025ED0050511BB229
:10667000A14202D015D2611ACB401800FEBD0823FA
:10668000B6E71023B4E72023B2E74023B0E7802326
:10669000AEE70123ACE708240026B1E70C00012691
:1066A000AEE7091B8B40E8E7ECCB00006000002060
:1066B000007000401C0000200405000020000020A5
:1066C000FF00FFFFFC700040F0B520285BD8364B80
:1066D0008000C258354B1E68002E30D1C227344B83
:1066E000BF00D859334C03250440C020000220438A
:1066F000D851C02480206400800018512E4F1860AB
:106700002E4B803CD859FF3CA043D8510437D85970
:10671000A8432043D8510837D8590C35A84384469C
:10672000072065462843D851A820C0001E50C1202C
:106730008026800076021E501C601C4B1C601425B5
:1067400000202B001E4C2E0046433659771C1BD1CF
:106750004343E250A0230325C132FF329200DB0500
:10676000D550184B1A68082A14D114234343E31850
:106770009A6812485132FF32920059601150DA681B
:10678000C1239B00C250F0BD9642E1D001300328E6
:10679000D9D1F8E7082A02D9083AD140E5E7082319
:1067A0009A1A9140E1E7C046ECCB0000E41B0020C0
:1067B00000E100E0FF00FFFF040500000090004042
:1067C00024000020640000202149F0B54A6C2148D3
:1067D000002A14D0A025A12600230124ED05F600EF
:1067E000C258571C06D0C7187F68002F02D0270058
:1067F0009740AF5114333C2BF2D100234B64A023BC
:106800000121DB0500260F009C4614234B43C318CF
:106810001A1F1268104C0E4D920014195219526C26
:10682000002A10D01A00143A1268551C09D0103BE7
:106830001B68FF2B05D03B00934065461A00074BB1
:10684000EA50FC34666401310429DED1F0BDC04653
:10685000FC90004024000020009000400C05000047
:1068600000B5202810D80C4A8000835803290BD883
:10687000A0220800C133FF33D2059B0001F036FC93
:10688000020905070021D15000BD0C21FBE70421BE
:10689000F9E70321F7E7C046ECCB000020280AD82F
:1068A000074B8000C25801239340A022D205002943
:1068B00002D1044953507047A121C900FAE7C046EC
:1068C000ECCB00000C05000003000020202B0AD8B0
:1068D000A021A222C905D2008858034A9B009B58D8
:1068E000D840012318407047ECCB0000F7B50600F4
:1068F0000D000C008B180193019B671B9C4207D075
:10690000336821781B683000984701340028F3D1A0
:106910003800FEBD0849094A094B10B51B68885864
:10692000FA22190A1B0618439200002301F0B4FD55
:106930004904C00B084310BD0010014004050000CD
:10694000E81B002070B5041E09D0FFF7E3FF050027
:1069500000F014F8FFF7DEFF401BA042F8D370BD33
:106960000022044B9A60044A13680133DBB21360BF
:106970007047C046FC100140E81B00207047000033
:10698000F0B5C64600B5CB0F9846404A4B005B0DAC
:106990009A1882B00D000400132A2FDC002A49DB6C
:1069A0003B4F17413E000E40064323D07F0839007D
:1069B00029400C430AD03749BD438C4663445C42AE
:1069C0005C418023DB021341E4071D434146CE00B6
:1069D00031492B008E192200346875682000290087
:1069E00001F000FF009001910098019922002B0016
:1069F00003F090F802B004BC9046F0BD332A08DDE5
:106A00008023DB009A42F5D102000B0001F0EAFE80
:106A1000F0E7224A9446012263445242DA4002429D
:106A2000E8D052080242D1D094438022D2051A41C4
:106A30001443CBE74B005B080343DBD00B031B0B7A
:106A40001C436342234380244D0C24031B0B23402F
:106A50006D042B4319004346DA000F4B9B181C684A
:106A60005D6802000B002000290001F0BBFE0090D1
:106A700001910098019922002B0003F04BF8424647
:106A80004B005B08D60733431900B3E701FCFFFF57
:106A9000FFFF0F00EEFBFFFFA0CC0000EDFBFFFFB0
:106AA000F8B5274A4B005B0D9A180C000700132A13
:106AB00010DC002A36DB234B13410B423AD08024F2
:106AC00024031441002064189C4306002500300074
:106AD0002900F8BD332A0EDD80230600DB000D00FF
:106AE0009A42F4D102000B003800210001F07AFE36
:106AF00006000D00EBE7144D0600AC46012563448B
:106B00006D42DD40AC4663460D000342DFD03323C7
:106B10009A1A323B93401818874200D94C1C63469E
:106B20009843D2E7C90FCC070020531CCDD1074BA7
:106B30001C43CAE706000D000028C0D1C7E7C046C5
:106B400001FCFFFFFFFF0F00EDFBFFFF0000F03F28
:106B500030B5214A4B0087B05B0893421EDD1F4AC7
:106B6000934205DD02000B0002F0D4FF07B030BDF8
:106B700002AA00F095F803231840049A059B012807
:106B800013D002281DD0002814D00298039900F0D9
:106B90006FFB80231B069C466144E7E7002300222D
:106BA0000093002301F0DEF8E0E70298039900F07B
:106BB0005FFBDBE7012402980399009401F0D2F80F
:106BC000D4E7012402980399009401F0CBF88023C4
:106BD0001B069C466144C9E7FB21E93FFFFFEF7FAD
:106BE000F0B54746CE4680B58DB004000D0000F0EC
:106BF00067FA294B06001B780F005BB298460133F9
:106C000010D022002B002000290003F0CBFA81468F
:106C1000002807D1002200232000290001F014FCE5
:106C2000002806D1300039000DB00CBC90469946C2
:106C3000F0BD01230293194B0694079503934B462D
:106C40000A93434604940595002B15D00023002297
:106C50001900100002F0E2F8434608900991022B57
:106C60000ED103F0B9FB212303600A9B0193002B93
:106C70000CD1089E099FD5E70023002408930994AE
:106C800002A801F0C1F90028EFD1EAE703F0A4FB64
:106C90000A9B01930360ECE768000020B0CC000081
:106CA000F0B54E464546DE465746E0B5E14B4C0052
:106CB0008FB09046894664089C4200DC87E0DE4B3A
:106CC0009C4222DCDD4A002900DC92E0DC4B02F031
:106CD00021FFDB4B06000F009C4200D17EE1D94A28
:106CE000D94B02F017FF02000B00414630000A604A
:106CF0004B60390002F00EFFD34BD24A02F00AFF7C
:106D0000434601259860D9606BE0D04B9C4200DC83
:106D10008FE0CF4B9C4200DD55E1CE4A23159246D1
:106D20009A4451460905631A19001D00040003F036
:106D300055FA03F089FA02000B002000290008929E
:106D4000099302F0E7FE0022C34B02F071FC0F0032
:106D5000060003F043FA03F077FA04000D00020086
:106D60000B00300039000A940B9502F0D3FE00228C
:106D7000B94B02F05DFC002200230C900D9101F054
:106D80005DFB002800D192E10023002220002900B1
:106D900001F054FB434243410133B04A4146019262
:106DA000022208A80092524600F07CFB4B460500E8
:106DB000002B16DA802243461206944642465B6850
:106DC000454263445360D3686344D36009E00B00D9
:106DD000020041460A604B600022002300258A60C1
:106DE000CB6028000FB03CBC90469946A246AB460B
:106DF000F0BD934B01F0F6FC914B06000F009C4256
:106E000000D13DE18F4A904B01F0ECFC02000B00F9
:106E1000414630000A604B60390002F07BFE894A2F
:106E2000894B01F0DFFC012543466D429860D96033
:106E3000D7E701F049F88A4A8A4B06000F0002F0B2
:106E4000F7FB0022884B01F0CDFC03F0C7F90500E9
:106E500003F0FAF9794A7A4B0490059102F0E8FBC5
:106E600002000B003000390002F054FE754A0600A3
:106E70000F0004980599744B02F0DAFB029003911D
:106E80001F2D00DCC7E0029A039B3000390002F09E
:106E900041FE83468A4653465B0024155B0DE31A88
:106EA000102B6CDD04980599D322674B520502F034
:106EB000BFFB02000B00300039000292039302F086
:106EC00029FE0A0001001300069107920200390012
:106ED000300002F01FFE029A039B02F01BFE060028
:106EE0000F0004980599614A614B02F0A1FB320042
:106EF0003B0002F00FFE069E079F0B0002003900C8
:106F000030000292039302F005FE4B005B0D8346B6
:106F10008A46E41A312C32DD04980599B822544B84
:106F2000920502F085FB03000C000200029303941B
:106F30000B000698079902F0EDFD02000B00060019
:106F40000F000698079902F0E5FD029A039B02F0F4
:106F5000E1FD484A0290039104980599464B02F0DE
:106F600067FB029A039B02F0D5FD02000B00300084
:106F700039000292039302F0CDFD83468A465A46B9
:106F80005346414630000A604B60390002F0C2FDB2
:106F9000029A039B02F0BEFD44460B000200A26071
:106FA000E3604B46002B00DB1BE75B46236080233E
:106FB0001B065344636080231B069C466144A0600B
:106FC000E1606D420DE70B00020002F0A3FD4346B5
:106FD00000259860D9601860596002E7D3221A4BE7
:106FE000520502F097FD214A214B0D00040002F0EA
:106FF00091FD02000B00414620000A604B60290011
:1070000002F088FD1A4B194A02F084FD434601251F
:107010009860D960E5E602000B003000390002F00C
:1070200079FD6B1E154A9B009B5883468A46A342F6
:10703000A5D130E7FB21E93F7BD902400000405455
:10704000FB21F93F3163621A61B4D03DFB21394124
:10705000FFFFEF7FEAFBFFFF0000704138CD00002B
:1070600083C8C96D305FE43F0000E03F7370032EBA
:107070008A19A33BC14920259A837B39B8CC0000EB
:10708000D3220C4B520501F0ADFB0B4A0B4B040015
:107090000D0001F0A7FB02000B00414620000A6032
:1070A0004B60290002F036FD034A044BB9E6032386
:1070B00073E6C04661B4D03D7370032E8A19A33BBA
:1070C000F8B54746CE46674B80B50A000F00190059
:1070D00005003940994200D19BE004000100002FD7
:1070E00069DD3F1500D1B4E05F4B12039C4680235D
:1070F000120B5B0313435B00CA0F67449B184A00E3
:10710000F80703D5D20F5B009B188A0079108C46D4
:10711000002180201624894680030D189D4202DC40
:1071200029185B1B8144D50F5B00013C5B195200A1
:107130004008002CF1D10020804680202025002727
:10714000000609E08B425CD0D40F5B00013DE318E0
:1071500052004008002D16D0C4198B42F2DD2718CA
:107160000E00002C49DB5B1AA242894149425B1A9E
:10717000121BD40F5B00013D80443100E318520024
:107180004008002DE8D113434ED143465B083749F0
:107190004A468846494652104244C90702D58021D2
:1071A00009060B4361460F05BD18180029000CBCE9
:1071B00090469946F8BD7B005B0803433900002BDD
:1071C000F5D0002F3CD1E30A153A6405002BFAD024
:1071D0008020400303423FD1002700E00F005B0006
:1071E000791C0342FAD0250020208D40401A290046
:1071F000D71B2200C2401A4376E7FE43F60F8E19D2
:10720000B1E79442A0D82718002CF6DB1E0000231B
:10721000AEE702003B002800390002F009FA2A001C
:107220003B0001F0DFFAC2E74346013303D0434697
:1072300001335B08ABE7012398460023C144A6E76E
:107240003B00020002F066FC02000B0001F0E6FDCC
:10725000ADE713000022BBE70127210020207F4279
:10726000C6E7C0460000F07F01FCFFFF0000E03FE2
:10727000F0B54746CE4680B587B000920193754B76
:107280004F00814688467F089F4263DC02F0A6FFDC
:10729000002800D1D4E04A4643464846414602F021
:1072A000C7F904000D006C4A6C4B02F0C1F96C4A3E
:1072B0006C4B01F097FA22002B0002F0B9F96A4AF0
:1072C0006A4B02F027FC22002B0002F0B1F9684A59
:1072D000684B01F087FA22002B0002F0A9F9664AF8
:1072E000664B02F017FC22002B0002F0A1F9644A61
:1072F000644B01F077FA22002B0002F099F902901A
:1073000003910022604B2000290002F091F9029ABB
:10731000039B06000F002000290002F089F9009A63
:10732000019B04000D004846414602F081F902002D
:107330000B002000290002F0EDFB02000B003000E2
:10734000390002F0E7FB02000B0000204F4902F079
:10735000E1FB70E002000B0002F06AF904000D008E
:107360003D4A3E4B02F064F93D4A3E4B01F03AFA89
:1073700022002B0002F05CF93B4A3C4B02F0CAFBB6
:1073800022002B0002F054F9394A3A4B01F02AFA54
:1073900022002B0002F04CF9374A384B02F0BAFBBE
:1073A00022002B0002F044F9354A364B01F01AFA5C
:1073B0002B00220002F03CF9354B029003919F42D2
:1073C0009FDD344B00229F423DDC334900207B1877
:1073D0002E4916001F0002F09DFB0490059100222B
:1073E000294B2000290002F023F932003B0002F073
:1073F00091FB029A039B06000F002000290002F077
:1074000017F9009A019B04000D004846414602F01E
:107410000FF902000B002000290002F07BFB0200A4
:107420000B003000390002F075FB02000B000498DD
:10743000059902F06FFB07B00CBC90469946F0BD71
:1074400000201249F7E7154B002604920593144FCC
:10745000C5E7C046FFFF3F3ED43888BEE9FAA8BD65
:10746000C4B1B4BD9EEE213EAD529C804F7E923E93
:107470009015CB19A001FA3E7751C1166CC1563F49
:107480004C5555555555A53F0000E03F0000F03FD5
:107490003233D33F0000E93F0000E0FF0000E73F48
:1074A0000000D23FF0B5DE464E4645465746E0B5B1
:1074B000DC4CA5440D9114001900A49A0993DA4BF1
:1074C0009200D6584D1E03901821E01E0696029594
:1074D00000F0AAFEC3430100DB1719404B1C9A00C1
:1074E0009B1ADB001B190B9105934C1B771918D4C1
:1074F000A59BA5009C463F1922AE6544013707E0D5
:10750000286802F0A1FE013403C60435BC4208D04D
:10751000002CF5DA00200021013403C60435BC42FA
:10752000F6D1069B002B01DA00F0FDFB069B0399C8
:107530000133DB009A46099BDA0094460092002250
:10754000914672AA0492B94A6144934688469AAB1E
:1075500063449B44029B002B00DABCE15D4600269D
:107560000027039C4D442A686B6803CC02F060F846
:1075700002000B003000390001F034F9083D06002C
:107580000F004445EFD1049B4B441E605F6008230D
:107590009C46E144D145DDD10EA8042184464942F0
:1075A00061448C46069A93009C44614684460A9145
:1075B0000399083B63448C460C93009B0092634400
:1075C0009B46009A0498D10003008C4663440891BE
:1075D0001E685F68002A33DD954980468C46624408
:1075E000D300984470AB9A460EAB99460022914B5B
:1075F0003000390002F01CF802F0F0FD02F024FE29
:1076000000228D4B04000D0002F012F802000B0066
:107610003000390002F07EFA02F0E0FD4B4601C373
:107620009946434620001A685B68290001F0DAF8A1
:1076300008235B429C46E04406000F00D045D5D1AC
:10764000059B30001A003900984600F0DFFCFF234C
:1076500000229B0504000D0001F0EAFF00F038FC59
:107660000022764B01F0E4FF02000B00200029000D
:1076700002F050FA0D00040002F0B0FD814602F065
:10768000E3FD02000B002000290002F043FA06008F
:1076900040460F00002800DCEEE0009B18215A1E37
:1076A00092000EAB9B58091A1D000D41A9448D4054
:1076B0005D1B0EAB9D5017231B1A1D41002D2DDDA8
:1076C00001239C46009BE144002B00DC1CE20E9C45
:1076D0000123002C00D0B5E0009A012A09D09900BE
:1076E0000EAA54580133002C00D0ACE0009A9A4204
:1076F000F5D1059B002B0EDD012B00D1A8E1022B5B
:1077000009D1009B0EA95A1E92000EAB9B580793FD
:107710009B029B0A8B50022D00D1C1E00023002266
:107720003000390000F08AFE009B002800D194E26E
:10773000069A591E8A4210DC414A0A9894460EAABB
:107740006344944600229B0063441C68043B22432C
:107750008342FAD1002A00D0C0E0069B0EAA013B6A
:107760009B00D358002B00D0B3E001220C9B043BBC
:10777000596801320029FAD0009B9C4662441100EE
:1077800007921A0001338B4246DC0B986346804611
:10779000A59C4344A046099C9B00A1464A449844AA
:1077A000D30022AA9146049A99449446089BA59A2C
:1077B00063448446614494469A468B006344009334
:1077C0004346586802F040FD4B4618605960029BE2
:1077D000002B24DB4D46039C0026002701E028688F
:1077E00069680CCC01F024FF02000B003000390066
:1077F00000F0F8FF083D06000F005C45EFD153464E
:107800009E60DF6004239C460433E0449C46009B5A
:10781000E144E2449845D3D1079B0093D1E600268A
:107820000027ECE794FDFFFF80CE000018FEFFFF6D
:10783000FFFFFF1F0000703E00007041000020406D
:10784000FFFFFF3F002180225204141B0EAA545058
:10785000009999420EDD0EA884469B000EAA89006D
:10786000D25861446344CF4800E01A68821A04C3C6
:107870008B42FAD101243CE7059B002B06D1009BEB
:107880000EAA013B9B00D558ED1517E70022C64B09
:10789000300000F0F7FD002800D024E100253DE78E
:1078A00032003B000020C14902F034F906000F000D
:1078B000002C00D132E7059A0020BC4900F0A6FB5D
:1078C00002000B003000390002F024F906000F001E
:1078D00024E7012250E70026002754E64B46059A8C
:1078E000079388468B000EA9CB58183A0895059245
:1078F000002B0DD18C464146AD4B43449B00634465
:10790000043B58680139183A0028F9D08846059296
:10791000059A0020A54900F079FB434604000D00BC
:10792000002B00DA05E29E000EAB9C464346DB00CE
:1079300066449C46059370AB9946049F6744009744
:10794000306802F081FC22002B0001F071FE002261
:1079500038607960974B2000290001F069FE083FEC
:1079600004000D00043EB945EAD14AAB03939B469F
:1079700000239A46069B42469946434601320292AC
:1079800004934B46002B00DAAAE080208A4B009D2E
:107990009846C005894900260027002408E00823EE
:1079A0009C460835E044544511DC43461868596844
:1079B0002A686B6801F03CFE02000B0030003900C1
:1079C00000F010FF013406000F00A145E7DA5B4626
:1079D000C0C39B4601239C46009BE244083B0093A6
:1079E000029B9A45CDD1049B9846A49B022B00DDB7
:1079F0008EE0002B37DC1FD1059B00271D00039B69
:107A000000249C461E006544083E2A686B683800C6
:107A1000210000F0E7FE083D07000C00AE42F4D163
:107A2000089B002B03D080231B069C4664443A002D
:107A300023000D990A604B600720079B18409B2389
:107A40009B009D443CBC90469946A246AB46F0BD87
:107A5000009B0EA95A1E92000EAB9B5807935B0227
:107A60005B0A8B5057E64346002B00DA70E100209A
:107A70000021DB004AAAD61848AF32687368083E76
:107A800000F0B0FEB742F8D1089B002B00D025E1F2
:107A90000B0002004A984B990D9C2260636002F033
:107AA00039F8434607000C00002B13DD01254CAECE
:107AB000B14638002E0021004C4601360CCC00F0B7
:107AC00091FEA146B045F7DA089B07000C00002B99
:107AD00000D015E13A0023000D998A60CB60ABE736
:107AE0000026002773E701239C46009BE144022502
:107AF000002B00DDEBE532003B0000202B4902F0BB
:107B000009F806000F0009E60024F2E54AAB0393EA
:107B1000A49B032B00D08FE74346002B00DC14E12D
:107B2000039ADB009B46130091465B441E685F6826
:107B3000234B43440293DB00994448AB9A464B469F
:107B40005C681B681800210032003B000090019126
:107B500000F048FE04000D0002000B00009801999F
:107B600001F0D8FF3B00320000F03CFE4B4698602D
:107B7000D9601C605D6008235B429C46E14426009E
:107B80002F00CA45DBD14346012B00DCE3E0039A1A
:107B900013005B441E685F68029BDB0099464A4401
:107BA000904610E0FFFFFF000000E03F0000F03FC4
:107BB000FFFFFF3F0000703E40CE0000FB21F93F79
:107BC000FFFFFF1F984643465C681B6818002100B2
:107BD00032003B000090019100F004FE04000D0013
:107BE00002000B000098019901F094FF32003B0065
:107BF00000F0F8FD4346039A9860D9601C605D6010
:107C0000083B26002F009A42DCD14D4694460026C0
:107C100000244746083565442A686B683000210017
:107C200000F0E0FD083D06000C00AF42F4D1039BDC
:107C30004A9F5D689968D868089B002B65D08022B0
:107C4000120694460D9B6544604464441F605D6069
:107C50009960D8601E615C61EEE69A464B460793D8
:107C6000059B30005A423900089500F0CFF90022F8
:107C70003A4B06000F0000F005FC002824D0384BDA
:107C800000223000390001F0D3FC02F0A7FA52467E
:107C90000400950002F0D8FA0022304B01F0C8FC35
:107CA00002000B003000390001F034FF02F096FAB8
:107CB0000EAA50510122059B524418339046059359
:107CC00093000EAAD45023E65346300039009C009E
:107CD00002F084FA0EAB1851D04619E680230D9AB3
:107CE0001B06CB18106053600B0002004A984B999A
:107CF00001F010FF434607000C00002B00DDD5E625
:107D000080231B069C466444E4E62B003A000D9D4C
:107D10002A606B600A000300AA60EB603200230057
:107D20002A616B6188E6099BDB00009372AB0493C8
:107D300032E4A49B022B00DDE8E6002B00DD92E696
:107D400000D079E6002700246AE6002600246EE7CA
:107D50000020002198E60026340068E7000070410A
:107D60000000703EF0B5CE46474680B587B0009221
:107D70000193474A4B00814688465B08934207DCE3
:107D80004146484602F02AFA4146031E484666D05C
:107D90004A4643464846414601F04AFC04000D006D
:107DA00002000B004846414601F042FC394A3A4B7A
:107DB00006000F002000290001F03AFC374A384B3A
:107DC00001F0A8FE22002B0001F032FC354A364BB0
:107DD00000F008FD22002B0001F02AFC334A344B4E
:107DE00001F098FE22002B0001F022FC314B324AB8
:107DF00000F0F8FC0E9B02900391002B34D0009809
:107E0000019900222D4B01F013FC029A039B049070
:107E100005913000390001F00BFC02000B000498C2
:107E2000059901F077FE22002B0001F001FC009A79
:107E3000019B01F06FFE224A04000D00214B30002F
:107E4000390001F0F5FB02000B002000290000F0D2
:107E5000C9FC02000B004846414601F05BFE07B03A
:107E60000CBC90469946F0BD02000B002000290092
:107E700001F0DEFB124A134B01F04CFE32003B00D6
:107E800001F0D6FB4A46434600F0ACFCE7E7C046AB
:107E9000FFFF3F3E7CD5CF5A3AD9E53DEB9C2B8A7C
:107EA000E6E55A3E7DFEB157E31DC73ED561C119D7
:107EB000A0012A3F1111813FA6F810110000E03FF8
:107EC000495555555555C53F49004B081900704750
:107ED000474AF0B54F4691464B005B0D99444646E4
:107EE000D6464A46C0B505000C000E00884607007D
:107EF000132A27DC002A4BDB3E4B13419A460B002A
:107F000052461340034318D03B4A3C4B2800210003
:107F100000F068FC0022002300F0AAFA002847D0F5
:107F2000002C04DA80234A465B03134198444646FA
:107F3000534600279E43380031001CBC90469946AA
:107F4000A246F0BD332A08DD8023DB009945F4D139
:107F500002000B0000F046FCEFE7294A944601229C
:107F600063445242DA4092460242E6D0224A234B10
:107F70002800210000F036FC0022002300F078FAEF
:107F8000002815D0002C1EDB534646469F430FE0C9
:107F9000194A1A4B2800210000F024FC002200237B
:107FA00000F066FA002803D0002C04DB002700262E
:107FB00038003100C1E76400640825430027002D24
:107FC000F6D0104EF4E74B46142B0BD03422D21AC5
:107FD000012393405D19BD4208D201239C462F0026
:107FE000E044D1E7133B9C46E044CDE72F00CBE7CC
:107FF00001FCFFFFFFFF0F009C7500883CE4377E0B
:10800000EDFBFFFF0000F0BF002070474B0070B594
:108010005B0D14000A00002B1AD14B005B080343D0
:1080200015D0234B002201F003FB224B9C422DDB99
:108030000A004B005B0D363B1F4DE318AB422ADCB8
:10804000002B0DDD1D4C1B0522401A43110070BD95
:108050001B4DAB42F0D102000B0000F0C3FBF6E772
:108060001D00353519DA174B02009C4209DD0B0063
:108070001548164900F032F8134A144B01F0D8FAAB
:10808000E5E70B001248134900F028F8104A114B9D
:1080900001F0CEFADBE70200E9E7084C3633224074
:1080A0001B051343190000220B4B01F0C1FACEE768
:1080B00000005043B03CFFFFFE070000FFFF0F80B1
:1080C000FF07000050C300009C7500883CE4377E29
:1080D00059F3F8C21F6EA5010000903C30B54A006C
:1080E000DB0FDB0752081A43110030BD02B47146A2
:1080F00049084900095C49008E4402BC7047C046EB
:1081000003B47146490840004900095A49008E44A9
:1081100003BC7047002243088B4274D303098B428F
:108120005FD3030A8B4244D3030B8B4228D3030C47
:108130008B420DD3FF22090212BA030C8B4202D3E9
:108140001212090265D0030B8B4219D300E0090A11
:10815000C30B8B4201D3CB03C01A5241830B8B421A
:1081600001D38B03C01A5241430B8B4201D34B0303
:10817000C01A5241030B8B4201D30B03C01A524168
:10818000C30A8B4201D3CB02C01A5241830A8B42ED
:1081900001D38B02C01A5241430A8B4201D34B02D6
:1081A000C01A5241030A8B4201D30B02C01A52413A
:1081B000CDD2C3098B4201D3CB01C01A52418309EE
:1081C0008B4201D38B01C01A524143098B4201D328
:1081D0004B01C01A524103098B4201D30B01C01A53
:1081E0005241C3088B4201D3CB00C01A52418308CD
:1081F0008B4201D38B00C01A524143088B4201D3FA
:108200004B00C01A5241411A00D201465241104659
:108210007047FFE701B5002000F0F0F802BDC0464E
:108220000029F7D076E7704703460B437FD400223E
:1082300043088B4274D303098B425FD3030A8B42FA
:1082400044D3030B8B4228D3030C8B420DD3FF2264
:10825000090212BA030C8B4202D31212090265D032
:10826000030B8B4219D300E0090AC30B8B4201D3E5
:10827000CB03C01A5241830B8B4201D38B03C01A2C
:108280005241430B8B4201D34B03C01A5241030BA3
:108290008B4201D30B03C01A5241C30A8B4201D354
:1082A000CB02C01A5241830A8B4201D38B02C01AFF
:1082B0005241430A8B4201D34B02C01A5241030A76
:1082C0008B4201D30B02C01A5241CDD2C3098B425B
:1082D00001D3CB01C01A524183098B4201D38B01D8
:1082E000C01A524143098B4201D34B01C01A52417B
:1082F00003098B4201D30B01C01A5241C3088B42C0
:1083000001D3CB00C01A524183088B4201D38B00AA
:10831000C01A524143088B4201D34B00C01A52414C
:10832000411A00D201465241104670475DE0CA0F23
:1083300000D04942031000D34042534000229C46E3
:1083400003098B422DD3030A8B4212D3FC228901ED
:1083500012BA030A8B420CD3890192118B4208D3C3
:10836000890192118B4204D389013AD0921100E025
:108370008909C3098B4201D3CB01C01A5241830939
:108380008B4201D38B01C01A524143098B4201D366
:108390004B01C01A524103098B4201D30B01C01A91
:1083A0005241C3088B4201D3CB00C01A524183080B
:1083B0008B4201D38B00C01A5241D9D243088B4261
:1083C00001D34B00C01A5241411A00D20146634604
:1083D00052415B10104601D34042002B00D5494268
:1083E000704763465B1000D3404201B5002000F0A7
:1083F00005F802BD0029F8D016E770477047C0465F
:10840000D0400B1C1141203A03D49C461341184321
:1084100063465242934018437047C0468446101C3E
:1084200062468C46191C634600E0C0461FB501F049
:1084300097F8002801D40021C8421FBD10B500F0F4
:10844000EFFF4042013010BD10B501F089F800285F
:1084500001DB002010BD012010BDC04610B501F0A9
:108460007FF8002801DD002010BD012010BDC046AE
:1084700010B501F011F8002801DC002010BD01202A
:1084800010BDC04610B501F007F8002801DA002041
:1084900010BD012010BDC046F0B5CE4647461504BC
:1084A0002D0C2E0080B50704140C3F0C9946030CCC
:1084B0007E435D43674363437F19340CE4199C4654
:1084C000A54203D980235B029846C4444B464343EC
:1084D0005143250C36046544360C2404A4195B1959
:1084E000591820000CBC90469946F0BDF0B54E4698
:1084F00057464546DE46E0B543025B0A450083B079
:108500000F1C99462D0EC60F002D57D0FF2D24D0DD
:108510008020DB00C0041843002381469A469B4616
:108520007F3D7C027A00FB0F640A120E984623D02E
:10853000FF2A4BD0E30080240020E4047F3A1C4350
:10854000AD186B1C47460193534677403A000F2BFA
:1085500048D87D499B00CB589F46002B00D085E032
:1085600008339A46063B9B467C027A00FB0FFF25A8
:10857000640A120E9846DBD1002C00D090E05246DF
:1085800001231A4392460120DBE74C465846170068
:10859000022824D0032800D1CFE0002200230128A4
:1085A0004DD15802D205400AFF071043384303B0AB
:1085B0003CBC90469946A246AB46F0BD002B5BD131
:1085C00004239A46033B00259B46AAE7FF35002C6F
:1085D00060D1524602231A4392460220B1E7FF229D
:1085E0000023DEE74B461B0C9C464B462604360C0C
:1085F000180461463300220C6446000C43434E438A
:108600005043544380191A0C1218964203D9802102
:1086100049028C4664441B041B0C1004C0188301DF
:108620005E1EB341800E1843130C1B199B010343BC
:108630001C00230179D5012362081C401443019AD0
:108640007F32002A4DDD630704D00F232340042B23
:1086500000D00434230103D53C4B019A1C408032E6
:10866000FE2ABCDCA3015B0AD2B29AE70C239A462D
:10867000093BFF259B4654E7180001F071FE4A466E
:10868000431F76259A4000236D4291462D1A9A4643
:108690009B4646E7524603231A439246032050E77F
:1086A000200001F05DFE431F2D1A9C40763D002006
:1086B00047E780230027DB03FF2272E7424666E795
:1086C0004C463200584662E780234A46DB031A4292
:1086D00022D01C4220D123435B025B0A4746FF2283
:1086E0005FE701239A1A1B2A21DC23000199D3405A
:1086F0009E318C401A0023005C1EA34113435A078D
:1087000004D00F221A40042A00D004335A0111D495
:108710009B015B0A002244E780234A46DB031343A4
:108720005B025B0A3700FF223BE7019587E70022E7
:10873000002336E70122002333E78023DB032343B2
:108740005B025B0AFF222CE790CE0000FFFFFFF7E1
:1087500070B500283DD0C317C5185D40C40F280070
:1087600001F0FEFD9E22121A962A07DCD2B20828DA
:1087700033DD083885406802400A23E0992A0BDD82
:10878000052329001B1AD94003001B339D402B00F1
:108790005D1EAB4119430D00052801DD431F9D40BF
:1087A0002B000F490B406E0709D00F263540042DD2
:1087B00005D004335D0102D59F220B40121A9B01A4
:1087C000580AD2B24002D205400AE40710432043BF
:1087D00070BD002400220020F4E76802400AF1E79F
:1087E000FFFFFFFBF0B54F464646D6460C00090397
:1087F000C0B5490A470F5E0039431F03DB0F9C4693
:1088000065007B0A570F1F436D0DE40F760DA146DF
:10881000C000B846D200AB1B64457BD0002B5FDDA7
:10882000002E00D0A4E03E00164300D112E15E1EEF
:10883000002E00D09EE1871A4346B84280410125B0
:10884000C91A4042091A0B0200D431E149024E0A0A
:10885000002E00D16EE1300001F082FD0300083BE4
:108860001F2B00DD61E120223900D21A9E40D14049
:108870009F400E439D4200DD51E15D1B6B1C1F2B91
:1088800000DD7CE12021C91A3D0030008F40884086
:10889000DD40791E8F41310007222843D940002551
:1088A00007433A40002A09D00F233B40042B05D050
:1088B0003B1DBB42BF417F42C9191F000B0200D4C0
:1088C00026E26A1CC64B55056D0D9A4200D106E1A1
:1088D000C44AFF080A40530752023B43120B8EE082
:1088E000002B00D0B8E06B1C5B055B0D012B00DC9E
:1088F00030E1871A4346B842B641CB1A76429E1BF6
:10890000330200D54CE13B003343A1D100220024C7
:10891000002570E0002B00DCE5E0002E00D183E0B4
:10892000AF4EB54260D0802636043743B846382B68
:1089300000DC3EE1434613431F007A1E97413F1877
:1089400087428041404209180B0200D4B0E0A44B9A
:1089500001359D4200D1C3E0A24A7B080A400121B3
:108960000F401F435108D30707221F433A4099E79E
:108970009B4EB54238D0802636043743B846382B54
:1089800000DDDCE01F2B00DC30E11E004746203E0E
:10899000F740BC46202B04D04026F31A46469E40A2
:1089A0003243170063467A1E97411F43CCE0002BE9
:1089B00000D104E24346134300D159E14B07C008FC
:1089C00018438023C9081B03194208D04546ED0807
:1089D0001D4204D14346D008590708432900420FDD
:1089E000C9007F4D1143C0004B07CA087C49C0082D
:1089F00003438D4268D012036D05120B6D0D0021EB
:108A000012031800130B0A0D12051A43764B2D059D
:108A100013402B435B00E4075B08234319001CBC95
:108A200090469946A246F0BD3E00164312D05E1E07
:108A3000002E00D000E18718874280414144404227
:108A4000091801250B0233D5022585E7644633005A
:108A5000414610001D00C7E7002D00D0DAE00C00F1
:108A60000443F3D05C1C00D19FE15D4CA64200D1D1
:108A70002FE1DB43382B00DD66E11F2B00DD83E1B6
:108A800020240500E41A0F00DD40D940A0404346F1
:108A9000A7405B1A441EA04198462F433843171A3B
:108AA000BA42924143465242991A64463500CAE698
:108AB00007223A40002A00D0F6E64B07CA08484988
:108AC000FF083B438D4296D11900114300D19EE12E
:108AD000802109030A431203120B414D8FE7150051
:108AE000002200238BE7002B00D0C7E06B1C5F0542
:108AF0007F0D012F00DCF1E0394DAB4200D1B9E030
:108B000085180A008542894142444942511807228A
:108B1000CF076D082F4349083A401D00C2E60722DF
:108B20003049ED1A31403A40BCE63E0028388640D4
:108B300000279FE6380001F013FC20308EE6434604
:108B400013431F007A1E9741C71BB8428041404221
:108B5000091A78E60E003B0006431343002D61D14D
:108B6000002E00D0F4E0002B00D11BE16446390058
:108B7000100039E71A4FBB427AD03300FFE63000CD
:108B80001F3DE840202B03D04021CB1A9E403743A5
:108B90007B1E9F41072207433A400021002589E7B9
:108BA000171A4346BA42B641591A76428E1B64469A
:108BB0004EE61F2B00DDADE020264746F61AB740F3
:108BC000B9461700B246DF404E463E433700564690
:108BD000B240561EB24117434246DA408918AEE60B
:108BE000FF070000FFFF7FFFFFFF0F8020264746A3
:108BF000F61AB740B9461700B246DF404E463E432C
:108C000037005646B240561EB24117434246DA403C
:108C1000891A99E77F4CA6425BD0802424045B42EA
:108C2000214327E7002E0CD1002B00D1CBE0644676
:108C300039001000774DD7E6764FBB4218D033008D
:108C400075E6002B14D04B07C00818438023C908D1
:108C50001B03194207D0FC081C4204D17907D00835
:108C60000843E14621004C46420FC9001143C000B1
:108C7000684DB9E61D0000220023C0E6002D5BD13F
:108C80000D00054300D1E2E65D1C00D1B0E0614D6E
:108C9000AE421FD0DB43382B71DC1F2B00DD96E08A
:108CA00020250F00ED1AAF40B9460700AA46DF4065
:108CB0004D463D432F005546A840D940451EA8418A
:108CC00088440743BF1897429241514241443500BE
:108CD0003AE6644635004146100085E60B00034342
:108CE000002D00D063E6002BF5D04346134300D19E
:108CF0007AE687188742804107224144404209189A
:108D00003A400B0200D4D5E6434B01351940C9E582
:108D1000380069E61E004746203EF740BC46202B3F
:108D200004D04026F31A46469E403243170063465D
:108D30007A1E97411F4302E6364DAE42CAD08025C7
:108D40002D045B422943A6E70843411E8841A6E65D
:108D5000002B00D148E6871A4346B842B641CB1AE9
:108D600076429E1B33024BD5171A4346BA429241B4
:108D7000591A5242891A072264463A4092E5014341
:108D80000F00791E8F419DE71C000F00203CE7403B
:108D9000202B03D04024E31A99400843411E884108
:108DA00038437CE60022002425E6171A4346BA42DF
:108DB0009241591A5242891A6446350043E54146A8
:108DC0001000144D10E680220024120380E61D00DE
:108DD0000F00203DEF40BC46202B03D04025EB1A6E
:108DE0009940084307006346781E87411F4369E79F
:108DF000871897429B4141445B42C9183500A3E55F
:108E00003B003343CED0072231003A4052E60023E4
:108E10001A00F4E5FF070000FFFF7FFFF0B557469B
:108E2000DE464E464546E0B5834607000E03480041
:108E300085B092461C00360B400DCD0F002800D1A6
:108E40009DE0954B984239D08023F6001B041E43C9
:108E5000924A7B0F33439946944603006344009340
:108E600000230026FF00029323031B0B9846630098
:108E7000E40F52465B0D019400D1B3E086498B426A
:108E800000D19EE04246D100802212040A4351469E
:108E9000490F11438B46814952468C4600996344E1
:108EA000CB1A0021D20000932B0063409A460F2E6C
:108EB00000D905E17A4BB6009B599F465B46334388
:108EC000994600D0B8E002230826002700900293BC
:108ED000CAE7CB463A0002990195019B9A460229BE
:108EE00027D0032900D180E2012944D06D49009B9D
:108EF0008C4663441C00002C38DD530700D013E27D
:108F0000D2085B46DB0109D55946674B19408B46B1
:108F10008021C9008C46009B63441C00634B9C422B
:108F200007DC5B4664055F075B0217431B0B620DA2
:108F300002E000230027584A00211B031C0B0B0DE5
:108F40001B05234314055A4A380013401C4353465B
:108F50006400DB0764081C43210005B03CBC90465C
:108F60009946A246AB46F0BD0122524201231B1B8B
:108F7000382B00DCADE1002200230027DCE75B4654
:108F8000334399465ED0002E00D18AE1300001F0D3
:108F9000E7F903000B3B1C2B00DD7BE11D22D31AFC
:108FA0005A460100DA4008398E4013005F463343C9
:108FB00099468F403F4B00261B1A009300230293D3
:108FC00052E7414653460B433B499B468C46009B28
:108FD000634400935B46002B3BD1022300221E43D7
:108FE000022161E7434613439B4637D04346002B9B
:108FF00000D162E1404601F0B3F903000B3B1C2BAA
:1090000000DD53E102004146083A914088461D21A7
:10901000CB1A5146D9400B0041460B439B46534661
:1090200093401A00009B25499C46604403008C46EF
:1090300063440093002137E70323B14600900C26D8
:10904000029311E7002300930133042600270293C3
:109050000AE70323C3461E43032125E701331E43CA
:109060000022012120E700239A46802300271B03CA
:10907000094A61E7802349461B03194200D1E2E017
:109080005946194200D0DEE00B431B0317001B0BAF
:10909000A246014A50E7C046FF07000001FCFFFF5F
:1090A000D0CE0000FF030000FFFFFFFEFE07000020
:1090B000FFFF0F800DFCFFFF01F8FFFFF30300002F
:1090C000D94500D9CBE000D1C6E03C004846002796
:1090D000009B013B00935B46160E1B021E431302CE
:1090E000984633041B0C9946310C0191FFF798F810
:1090F0004A4642430B04210C050019438A4207D912
:109100008919013D8E4203D88A4201D9851E8919E9
:10911000881A0199FFF784F809048C464A4621040D
:1091200064464243090C030021438A4204D9891949
:10913000013B8E4200D8F1E02D041D43AB4643466F
:10914000891A4246280C12041D0C5B46140C22009E
:109150001B041B0C5A4303946B434443029568431E
:109160001B19150CEB189C4203D980246402A446F9
:1091700060441C0C15041B042D0C20185D19814241
:1091800077D373D00C1AA24A7D1BAF42BF419446DD
:10919000009B7F426344E01B1C00864200D1DBE061
:1091A0000199FFF73DF84A4642430B04290C07009A
:1091B00019438A4207D98919013F8E4203D88A424E
:1091C00001D9871E8919881A0199FFF729F809041E
:1091D0004A46894629044D464243090C0300294367
:1091E0008A4207D98919013B8E4203D88A4201D9A4
:1091F000831E89193F04891A3A00039F1A433800D5
:1092000013041B0C584381460298150C6F434343CB
:1092100045434846000C8446DB1963449F4203D90A
:10922000802040028446654448461F0C00041B040D
:10923000000C7D191818A94200D284E000D17FE00B
:1092400001231A4357E680234A461B0313431B039B
:109250001B0BAA466F4A6FE6BA4200D935E74B4668
:10926000DC0758087B081C43FF0734E70024AF42A3
:1092700089D247444745A4415B466442A419641817
:10928000013BA6421ED2A0426DD800D1B6E0241AFE
:109290009B4678E703005A46283B9A4000279146B0
:1092A00088E6584601F05CF8203072E6030052462A
:1092B000283B9A4093460022B4E6504601F050F80D
:1092C00020309AE6A642E2D1B845DCD9341A9B4652
:1092D00059E71F2B65DC504C0099A4465C4661445D
:1092E00008008C4011008240D940501E82410C433E
:1092F00014435A46DA401300620709D00F22224075
:10930000042A05D02200141D9442894149425B1869
:109310001A0262D50122002300270DE68A4200D8F6
:109320000AE7831E891907E70F231340042B00D196
:10933000E6E5171D9742924153429B44FA08E0E547
:10934000002800D1D7E57118531EB14227D3A94296
:1093500015D358D01A0073E7002B00DC04E6012374
:1093600000229B44CDE502234744474589415B42A7
:109370009C46494289190C19E344241A03E74346E1
:109380005F0047459B41B8465B429E19023A8919E6
:10939000A94200D054E7404500D051E7ABE51A00A0
:1093A000F6E71F215F4649420C1BE740202B07D000
:1093B0001A49009B8C46634418005B4683401A435D
:1093C000501E82413A4307270023174009D00F213E
:1093D000002311401400042995D122005F075B028D
:1093E0001B0BD20817430022A6E5802359461B0316
:1093F0000B431B0317001B0B064A9DE5BD42B2D869
:109400009B460024BFE68045B9D31A00C3E7C04697
:10941000FF030000FF0700001E0400003E040000E0
:10942000F0B54F464646D6468446C0B58046194EEE
:1094300018030F034D00000B5C0082463F0B6D0DBF
:10944000C90F9146640DDB0F0120B5420AD0B4422A
:1094500003D0A54201D157450CD01CBC904699467B
:10946000A246F0BD66463E43F7D1AC42F5D1544624
:109470001443F2D10120C845EFD1994207D0002D05
:10948000EBD163461F433800471EB841E5E7002093
:10949000E3E7C046FF070000F0B54F464646D64614
:1094A0004D00C0B50E03C90F8A462C491F035C004E
:1094B0008046360B6D0D91463F0B640DDB0F8D42E0
:1094C0001ED08C4216D0002D1ED130438446002C75
:1094D00001D13A4323D06246002A1AD09A4529D0B6
:1094E000514602200139084001381CBC904699467B
:1094F000A246F0BD39001143E5D002204042F4E716
:109500003043FAD1AC420FD0002C0FD13A43E7D010
:109510000CE00122013B934318000130E5E763466C
:109520000020002BE1D0DBE73A43E6D19A45D7D1C2
:10953000A542D5DCA54205DBBE42D1D808D000202B
:10954000BE42D2D250460123013898430130CCE7C5
:10955000C845C5D80020C845F4D3C6E7FF070000BA
:10956000F0B54F464646D6464D00C0B50E03C90F6E
:109570008A462E491F035C008046360B6D0D9146CE
:109580003F0B640DDB0F8D4218D08C4211D0002DA3
:1095900018D130438446002C1ED13A431CD1634677
:1095A0000020002B30D051460220013908400138FC
:1095B0002AE039001143EAD0022025E03043FBD1F4
:1095C000AC4226D0002C26D13A4324D15146022069
:1095D00001390840013817E06246002A0FD09A4549
:1095E000E1D1A54205DBBE42DDD819D00020BE4244
:1095F0000AD25046012301389843013004E0012289
:10960000013B9343180001301CBC90469946A2468A
:10961000F0BD3A43D0D19A45C5D1A542C3DCE0E7BD
:10962000C845C0D80020C845E3D3EDE7FF070000D8
:10963000F0B55746DE464E464546E0B58346060041
:109640000F03480087B092461D003F0B400DCC0F22
:10965000002800D16FE0DE4B984238D08023FF0015
:109660001B041F43730F3B430193DA4B00279946BA
:1096700000239B46F60081442B0369001B0B5246D6
:109680009846490DED0F002900D185E0D04B994255
:1096900000D173E04346DA0080231B041343524693
:1096A000CC48520F84461343524600206144D200F6
:1096B00089442100694000918C46012149448A4631
:1096C0000F2F00D990E0C449BF00CF59BF465B4679
:1096D0003B43019300D06AE102230827002681461C
:1096E0009B46C9E732005846019B6146009102281B
:1096F00000D175E0032800D1FEE1012800D02CE163
:1097000000230027002600253F032A0D3F0BB34806
:1097100012053A4302401B051343009A5B00D10730
:109720005B080B433000190007B03CBC90469946DB
:10973000A246AB46F0BD5B463B43019300D12FE10F
:10974000002F00D1A5E1380000F00AFE03000B3B1A
:109750001C2B00DD96E11D22D31A5A460100DA4087
:109760005E4608398F4013008E403B4301939C4B6B
:1097700000271B1A994600239B467DE74146534626
:109780000B4393498C46E144002B00D01AE102229E
:109790000220174300228CE7134300D10DE143461A
:1097A000002B00D181E1404600F0DAFD02000B3AC7
:1097B0001C2A00DD72E10100434608398B409846BF
:1097C0001D239A1A5346D3401A0043461343524668
:1097D0008A404946081A824989468144002068E740
:1097E0007B4B002700268EE7140C1204120C11008C
:1097F000370C3604350C794328008C462E00604324
:109800006044834656432100300C804658467943D5
:1098100040440291844506D98846802149028C46FD
:10982000E044414602913604010C360C00048B469C
:1098300081191E0C1B041B0C0391190079438C46E3
:10984000280075436544A8465843050C45447743B2
:10985000A94203D9802149028C466744290C8C46D1
:1098600039000004000C2D042D186144AB4405910F
:109870005946049101990F043F0C080C39005143DB
:109880004243904602008C46090C8B4662437C435F
:1098900044445C44A04503D980214902884642449F
:1098A000210C884661460904090C8C46390059434D
:1098B000434370437E430F0CF6182404BE196444DE
:1098C00042448C46B34203D980235B02984640440D
:1098D000029B61469846049B370443449B46AB4534
:1098E000AD416B420D0405992D0C8C467F196744E0
:1098F000FD18A8465D462D19A542A4419346644231
:10990000A446C344DC448F42BF4198459B419345E4
:109910009241A445A4415B427F421F43360C524210
:109920006442BF192243BF18624638184302D20D61
:10993000039913436A020A43501E82416146ED0DAA
:109940002A434E023243D90100D4B3E00126500825
:1099500032400243DE0732435B08224C5444002C61
:1099600062DD510709D00F201040042805D0101DDA
:109970009042924152429B180200D90104D58024A2
:109980001948E400034054441848844200DD27E7A6
:109990005E075B02D2081F0B630516435B0DB2E640
:1099A000002399460133042700269B4664E60323DF
:1099B000019781460C279B465EE601220120174352
:1099C000002276E6032303201F43434671E6C04688
:1099D000FF07000001FCFFFF10CF0000FFFF0F801A
:1099E0000DFCFFFFFF030000FFFFFFFEFE0700006E
:1099F0000023802700933F030026434B83E6019B0F
:109A00003200A446584670E6AC466EE680270199BF
:109A10003F0339422DD03B422BD11F433F033F0B25
:109A200000951600384B6EE601252D1B382D00DD04
:109A300066E61F2D40DC35481C005044160082406D
:109A40008440EE40501E824134431443EB40620791
:109A500009D00F222240042A05D02200141D94426E
:109A6000804140421B181A023ED5012300270026E0
:109A700049E68027019B3F031F433F033F0B0094B0
:109A8000214B40E603005A46283B9A4000260192AB
:109A90006DE6584600F064FC203057E6030052465D
:109AA000283B9A401300002293E6504600F058FCF1
:109AB00020307BE6CA4650E71F201E004042041BB0
:109AC000E640202D03D0124C5444A3401A43501EAC
:109AD0008241324307260027164009D00F20002379
:109AE000104014000428B9D122005E075B021F0B4E
:109AF000D2081643002306E680273F031F433F0397
:109B00003F0B1600004BFEE5FF0700001E0400009F
:109B10003E040000F8B557464E464546DE460C006A
:109B20000903E0B5490A460F5F0031431E03DB0F0E
:109B3000760A9B46530F3343C84E6500C000E40FBE
:109B4000D2006D0DA24681467F0D9C469046B742DD
:109B500000D1B9E05B46012673409B46EE1BA3454E
:109B600000D183E0002E63DD002F00D0B1E063461A
:109B7000134300D123E1731E002B00D0BAE1861AF3
:109B80006346B04280410125C91A4042091A0B02BE
:109B900000D447E149024B0A98464346002B00D1C6
:109BA00089E1404600F0DCFB0300083B1F2B00DD91
:109BB0007CE120223000D21A4146D0409940020078
:109BC0009E400A439D4200DD6AE15D1B6B1C1F2B1A
:109BD00000DD94E1202110003500C91A8E40DA40E2
:109BE0008840DD40711E8E41110007222843002568
:109BF00006433240002A09D00F233340042B05D0FE
:109C0000331DB342B641764289191E000B0200D4BF
:109C10003DE26A1C914B55056D0D9A4200D119E148
:109C20008F4AF6080A40570752023743120B9BE04F
:109C3000002E00D0C5E06E1C7605760D012E00DCEE
:109C400048E16746861ACB1BB042BF417F42B84607
:109C50001F004346FF1A3B00B8461B0200D55FE1D8
:109C600037439AD100220024002579E0002E00DC41
:109C7000FAE0002F00D18DE0784B9D4267D0802321
:109C800067461B041F43BC46382E00DC52E1634686
:109C900013435A1E93411E188642804140420918C0
:109CA0000B0200D4BEE06D4B01359D4200D1D2E0E5
:109CB0006B4A73080A4001210E401E435108D30726
:109CC00007221E43324095E71E00164300D045E7A9
:109CD00040E7624B9D423AD0802367461B041F43F6
:109CE000BC46382E00DDEBE01F2E00DC3AE13300ED
:109CF0006746203BDF403B00202E05D04027BF1B9E
:109D00006646BE40324390464646721E96413343F5
:109D1000DAE0002B00D114E26346134300D168E17E
:109D200080234E07C008C9081B030643194208D008
:109D30006046C008184204D163460100D2085E079D
:109D40001643F3009946C900720F444D11434B4628
:109D5000DE08424B4F073743CA089D4200D16EE0F0
:109D600012036D05120B6D0D00211203130B0A0D6A
:109D700012051A433B4B2D0513402B435B00E407B0
:109D80005B082343380019003CBC90469946A24624
:109D9000AB46F8BD6346134311D0731E002B00D0B1
:109DA00007E1861886428041614440420918012536
:109DB0000B0237D502257BE73E0061469146350010
:109DC000C5E75C46002D00D0E1E00B000343F3D073
:109DD000731C00D1ACE1214B9F4200D13AE1F34327
:109DE000382B00DD6FE11F2B00DD8CE120250E00FC
:109DF000ED1AAE40B0460600AA46DE404546354361
:109E00002E005546D940A8406346451EA8415B1A1E
:109E10009C463043161AB242924163465242991A06
:109E20003D00B4E607223240002A00D0E4E60B4BA6
:109E3000F6084F073743CA089D4200D090E73B0021
:109E4000134300D1A6E180231B031A431203120B14
:109E5000024D89E715000022002785E7FF07000073
:109E6000FFFF7FFFFFFF0F80002E00D0C7E06B1CBD
:109E70005E05760D012E00DCF0E0C84DAB4200D14E
:109E8000B9E085180A008542894162444942511867
:109E90000722CE076D082E43490832401D00A9E66F
:109EA000BF49ED1A114007223240A3E6320028389C
:109EB0008240002686E6300000F052FA203073E639
:109EC000634613435A1E9341C61AB0428041404232
:109ED000091A5CE60E00674606431743002D5ED163
:109EE000002E00D0F3E0002F00D11EE15C46614659
:109EF00091462CE7A94FBE427BD01E00F1E6100030
:109F00001F3DE840202B03D04021CB1A9A40164336
:109F1000731E9E410722064332400021002583E73D
:109F2000161A6346B2428041591A40420B1A9846AB
:109F30005C4632E61F2E00DDABE02027BB1B9A46B5
:109F400063465746BB40994613004F46F3401F43B4
:109F50003B005746BA40571EBA4113436246F2408F
:109F6000891898E62027BB1B9A4663465746BB4094
:109F7000994613004F46F3401F433B005746BA40F3
:109F8000571EBA4113436246F240891A9CE7834B3D
:109F90009F425FD080252D047342294320E7002E85
:109FA0000CD1002F00D1D0E05C46614691467B4D3C
:109FB000CDE67A4FBE421CD01E0065E6002F18D0B9
:109FC000C0084E0706438020C9080003014208D09C
:109FD0006346DC08044204D12100DA46D2085E0759
:109FE0001643F300994601245346C900720F1143EA
:109FF0001C406A4DABE61D0000220027B4E6002D90
:10A0000059D10B00034300D1D6E6731C00D1B2E056
:10A01000624B9F421ED0F343382B6FDC1F2B00DDB9
:10A0200097E020250E00ED1AAE40B0460600AA4685
:10A03000DE40454635432E005546A840D940451ED2
:10A04000A8418C440643B61896429241514261445D
:10A050003D0025E63D006146914678E60B0003434E
:10A06000002D00D055E6002BF5D06346134300D1F8
:10A070006DE68618864280416144404209180022FC
:10A080000B0200D4D0E6464B01351940B2E5B1468B
:10A090005DE633006746203BDF403B00202E05D0C5
:10A0A0004027BF1B6646BE40324390464646721E5E
:10A0B00096413343EFE5394B9F42CBD080252D04A9
:10A0C00073422943A8E70843411E8841A2E6002FB6
:10A0D00000D13CE66346861ACF1AB0429B415B42F0
:10A0E000FB1A98461B024ED5161A6346B24292419D
:10A0F000591A5242891A5C4600227BE501430E0040
:10A10000711E8E419FE71D000E00203DEE40B046BF
:10A11000202B04D04025EB1A99400843814648463D
:10A120004346411E8841184374E60022002417E686
:10A13000161A6346B2429241591A5242891A3D0098
:10A1400025E561469146154D01E680220024120363
:10A1500079E61D000E00203DEE40B046202B04D0D5
:10A160004025EB1A9940084381464E464346711EEE
:10A170008E411E4367E7861896429B4161445B42CD
:10A18000C9183D008CE547463743CED007224146EB
:10A19000324049E600273A00E6E5C046FF070000E6
:10A1A000FFFF7FFF70B50C4E0D031C0349005B00E1
:10A1B0002D0B490D240B5B0DB14208D00649002040
:10A1C0008B4203D114432000441EA04170BD0543BF
:10A1D0000120002DFAD1F1E7FF07000030B5144D42
:10A1E0000A034B00120B5B0DC90F0024AB4211DDBB
:10A1F000104CA34210DC8024640322430E4CE41A6A
:10A200001F2C0CDD0D48C31ADA4013005C420029F4
:10A2100000D11C00200030BD094BCC18FAE7094DD5
:10A22000E040AC4663449A4013000343EEE7C04667
:10A23000FE0300001D0400003304000013040000AE
:10A24000FFFFFF7FEDFBFFFF70B500282DD0C31788
:10A25000C5185D40C40F280000F082F8154B1B1A8A
:10A260005B055B0D0A2815DD0B38854000222D03A8
:10A270002D0B002110002D030A0D2D0B12052A4372
:10A280000D4D1B052A4013435B00E4075B08234385
:10A29000190070BD02002900153291400A000B21FF
:10A2A000081AC5402D032D0BE3E7002400230025E9
:10A2B0000022DEE71E040000FFFF0F804100090EB0
:10A2C0004B1C70B5DBB24602750AC40F012B14DDBE
:10A2D000E0239B006D07360BCB1800210A0D2800E8
:10A2E00012051C4D32435B052A405B0813435B009B
:10A2F000E4075B082343190070BD002914D1002D29
:10A300001ED0280000F02CF80A281CDC0B232A00A1
:10A310001B1ADA40030015339D400F4B12031B1A22
:10A320005B05160B5B0DD8E7002D06D0320B80269F
:10A3300036036D071643094BCFE7084B0026CCE7E1
:10A3400000230026C9E703002A000B3B9A400025A2
:10A35000E3E7C046FFFF0F8089030000FF0700000E
:10A360001C2101231B04984201D3000C10391B0A45
:10A37000984201D3000A08391B09984201D3000909
:10A38000043902A2105C40187047C0460403020260
:10A3900001010101000000000000000030B51C00B8
:10A3A000094B05001B6885B0D868084B002A01D10D
:10A3B000074B1A000292019300912B0022000549DD
:10A3C00000F026F800F08EFD6C00002050CF000059
:10A3D0006FBE00005DCF0000014B18687047C0469B
:10A3E0006C000020084B10B50400002B02D00021A7
:10A3F00000E000BF054B1868836A002B00D0984727
:10A40000200001F045FBC046000000008CCF00009A
:10A410000EB403B5010003AB044804CB00680193FC
:10A4200000F076F802B008BC03B018476C000020BA
:10A4300070B500260C4D0D4C641BA410A64209D12A
:10A44000002601F027FB0A4D0A4C641BA410A6420B
:10A4500005D170BDB300EB5898470136EEE7B30065
:10A46000EB5898470136F2E73C0200203C020020FE
:10A470003C0200204C020020002310B59A4200D17B
:10A4800010BDCC5CC4540133F8E710B5884202D942
:10A490008B18984203D3002307E08B5C8354013A66
:10A4A000FBD210BDCC5CC45401339A42FAD1F8E718
:10A4B00003001218934200D1704719700133F9E775
:10A4C000936810B5013B9360002B04DA9469A342B2
:10A4D00007DB0A2905D01368581C106019700800A2
:10A4E00010BD00F033FC0100F9E7F8B506000F00DD
:10A4F0001400D518AC4201D1002007E021783A00C1
:10A500003000FFF7DDFF0134431CF3D1F8BD00003C
:10A51000F0B59FB002900F0016000593002805D0FB
:10A5200083690493002B01D100F0DCFD7B4B9F423B
:10A530005BD1029B5F68BB891B0762D53B69002B1F
:10A540005FD0002306AC6361203363761033A376BB
:10A5500035002B78002B01D0252B5CD1AB1B04934D
:10A560000CD0320039000298FFF7BFFF431C00D126
:10A57000C4E06269049B9446634463612B78002BBA
:10A5800000D1BBE0012200235242626002A9543292
:10A5900052186E1C2360E360A3601370A3653178CA
:10A5A00005225F4800F0BCFE751C002835D12268EA
:10A5B000D30604D5532302A95B1820211970130771
:10A5C00004D5532302A95B182B21197033782A2B49
:10A5D0002CD0350000210A20E3682A786E1C303A1E
:10A5E000092A64D900292ED026E04E4B9F4202D181
:10A5F000029B9F689FE74C4B9F429CD1029BDF6868
:10A6000099E73900029800F0F7FB002899D0012063
:10A6100040421FB0F0BD01359BE7414B2268C01A94
:10A6200001238340134323602E00B8E7059B191DC7
:10A630001B680591002B01DB099304E05B42E3609A
:10A640000223134323602B782E2B0AD16B782A2BFD
:10A6500035D1059B02351A1D1B680592002B2BDB9B
:10A660000793324E29780322300000F059FE00286B
:10A6700006D04023801B83402268013513432360AA
:10A68000297806222A486E1C217600F049FE00280F
:10A690003AD0284B002B25D10722059B0733934343
:10A6A000083305936369039A9B18636150E743433A
:10A6B00001219B18350090E701235B42D0E700237E
:10A6C0000A201A000135636029786E1C3039092987
:10A6D00003D9002BC5D00792C3E742430123521888
:10A6E0003500F1E705AB00933A00134B21000298C7
:10A6F00000E000BF0390039B0133D3D1BB895B060D
:10A7000000D584E70B9884E705AB00933A000A4B29
:10A710002100029800F080F8ECE7C046E4CF00008A
:10A7200090CF000004D00000C4CF000096CF0000FE
:10A730009ACF000000000000EBA40000F7B5150060
:10A7400001938A680B6900900C00934200DA1300B1
:10A7500022002B6043321278002A01D001332B6093
:10A7600023689B0602D52B6802332B6006272368DB
:10A770001F4027D0230043331B785A1E9341226881
:10A78000920630D42200019943320098089EB047C7
:10A79000431C25D0062320682A68E1680340002571
:10A7A000042B03D18D1AEB43DB171D40A3682269EC
:10A7B000934201DD9B1AED180027BD4220D10020F5
:10A7C00010E00137E3682A689B1ABB42D2DD220001
:10A7D0000123193201990098089EB047431CF0D11B
:10A7E00001204042FEBD3020E118433108702100B5
:10A7F0005A1C45310978A218433202331170C1E75F
:10A80000220001231A3201990098089EB047431C88
:10A81000E6D00137D1E70000F0B589B004920A0014
:10A8200043320593039002920A7E0C000E9B6E2A1F
:10A8300000D186E01FD8632A33D008D8002A00D17F
:10A840008CE0582A4DD0250042352A7030E0642A29
:10A8500001D0692AF7D1196825680A1D280629D56B
:10A8600008681A60002803DA2D23029A4042137008
:10A870006B4E0A274FE0732A74D008D86F2A1FD076
:10A88000702AE0D1202209680A43226003E0752A79
:10A8900016D0782AD7D12200782145321170614E26
:10A8A00022E025001A684235111D196013682B70CB
:10A8B000012365E008681A606906D3D500B2D1E7C4
:10A8C00019682568081D186008682E0605D5544EBD
:10A8D00008276F2A1BD00A2719E06D06F7D580B22A
:10A8E000F5E745314E4E0A7018682268011D006870
:10A8F0001960150621D5D30702D520231A432260FB
:10A900001027002803D1202322689A4322602300C5
:10A91000002243331A706368A360002B58DB0422C3
:10A92000216891432160002854D1029D002B5AD008
:10A930002500337842352B7055E05506DBD580B2C3
:10A94000D9E71A680D68101D4969186013682E064A
:10A9500001D5196002E06D06FBD519800023029D28
:10A9600023614FE01A68111D1960156800216268A3
:10A97000280000F0D5FC002801D0401B606063680F
:10A9800023610023029A13703CE023692A00049992
:10A990000398059DA847431C3ED023689B0715D408
:10A9A000079BE068984239DA180037E0220001235B
:10A9B000193204990398059EB047431C2CD00135E9
:10A9C000E368079A9B1AAB42F0DCE9E70025F7E75A
:10A9D0000028ADD0029D3900FDF722FC735C013DDB
:10A9E0002B700028F7D1082F09D12368DB0706D583
:10A9F00063682269934202DC3023013D2B70029B85
:10AA00005B1B2361059B07AA00932100049B03980D
:10AA1000FFF794FE431CB8D10120404209B0F0BDBD
:10AA2000A1CF0000B2CF00000D4B70B51C6805002F
:10AA3000A36B002B0FD1182000F056FC094BA0632C
:10AA40000360094B01224360084B83600B23838121
:10AA50000023026143610022A36B1D615A6170BD36
:10AA60006C0000200E33CDAB34126DE6ECDE050039
:10AA7000124B10B51C68A36B002B0FD1182000F0EF
:10AA800033FC0F4BA06303600E4B012243600E4B5F
:10AA900083600B238381002302614361A46B0B4A13
:10AAA000206961690A4BFDF7F7FC01220023801839
:10AAB0005941206161614800400810BD6C000020D0
:10AAC0000E33CDAB34126DE6ECDE05002D7F954CD8
:10AAD0002DF451580CB430B5164B9DB00C1E1D68AA
:10AAE00008DA8B2301202B6040421DB030BC08BC2B
:10AAF00002B01847822302A99B008B810023029099
:10AB000008619C4200D0631E8B604B6101235B4255
:10AB1000CB81209A21AB2800019300F03DFD431C1E
:10AB200001DA8B232B60002CDFD00023029A1370F4
:10AB3000DBE7C0466C0000200EB400B50B499CB0AA
:10AB40001DAB02900690079104910948094904CB76
:10AB50000591006802A9019300F01EFD0023029AEE
:10AB600013701CB008BC03B01847C046FFFFFF7F3E
:10AB70006C0000200802FFFF020010B51378541C7F
:10AB8000002B05D1CC5CD4540133002CFAD110BD7C
:10AB90002200F3E702780B78002A03D0013001315C
:10ABA0009A42F7D0D01A704703000A7801311A7020
:10ABB0000133002AF9D170470023C25C0133002A17
:10ABC000FBD1581E704730B50500002A00D130BDBA
:10ABD0000C78013A6B1C2C700131002C05D19A18AD
:10ABE0009A42F4D01C700133FAE71D00EDE710B56E
:10ABF0000378002B0FD10B785A4253415B42184027
:10AC000010BD0023CA5C002AFAD0C45C944201D172
:10AC10000133F7E701300378002BF2D11800EFE79A
:10AC2000F0B51F000E0087B00590019102920C98BC
:10AC3000347800F0EAFA082200194378751C1340B2
:10AC400036D12D2C36D1B51C74780126002F62D058
:10AC5000102F09D1302C07D120222B789343582B69
:10AC600054D110276C7802352D4B3900F318180099
:10AC70000393FDF7D5FA0491012100234942020014
:10AC80008C4618002100303909291AD80C00A74237
:10AC900023DD591C09D06346824206D302D10499B0
:10ACA000A14202DB0123784320182C780135E9E723
:10ACB0002E00BCE72B2C01D01E00C7E7B51C747812
:10ACC000FAE721004139192901D8373CDFE7210093
:10ACD0006139192901D8573CD9E75A1C08D1059A7E
:10ACE00023331360029B0398002B09D107B0F0BDFA
:10ACF000002E00D04042029A002AF7D0002B01D04B
:10AD00006B1E0193029B019A1A60EFE73024002F1B
:10AD1000AAD10827A8E7302C9ED00A27A4E7C0466E
:10AD2000FFFFFF7F37B51300064A05001068046A6D
:10AD3000002C00D1044C0A0000942900FFF770FF9A
:10AD40003EBDC0466C000020D0000020F8B50500D4
:10AD50000E001400002804D08369002B01D100F0FC
:10AD6000C1F9224B9C422DD16C68A369A360A389D1
:10AD70001B0731D52369002B2ED023682269F7B237
:10AD8000981A6369F6B2834205DC2100280000F0BE
:10AD90003BF9002826D1A3680130013BA36023685A
:10ADA0005A1C22601F706369834204D0A389DB07A9
:10ADB0001AD50A2E18D12100280000F025F9002804
:10ADC00012D00FE00A4B9C4201D1AC68CDE7094B91
:10ADD0009C42CAD1EC68C8E72100280000F00CF8BA
:10ADE0000028CAD0012676423000F8BDE4CF00002A
:10ADF00004D00000C4CF0000364B70B51D680600BB
:10AE00000C00002D05D0AB69002B02D1280000F00A
:10AE100069F9314B9C420FD16C680C23E25E93B20E
:10AE200019072DD4D90611D40923012033603733F3
:10AE30001343A381404270BD284B9C4201D1AC68B2
:10AE4000EBE7274B9C42E8D1EC68E6E75B0713D5BC
:10AE5000616B002908D023004433994202D03000AE
:10AE600000F06AFA002363632422A3899343A38139
:10AE700000236360236923600823A2891343A3810D
:10AE80002369002B0BD1A0218022A3898900920085
:10AE90000B40934203D02100300000F0E1F9012380
:10AEA000A289134011D00023A36063695B42A361B0
:10AEB000002023698342BED10C23E25E1306BAD57B
:10AEC00040231343A3810138B5E7920700D4636997
:10AED000A360EDE76C000020E4CF000004D0000088
:10AEE000C4CF000010B5062000F090FC012000F057
:10AEF000CFFD0000F7B58A8905000C00130760D468
:10AF00004B68002B04DC0B6C002B01DC0020FEBD29
:10AF1000E76A002FFAD000232E682B6080235B01A4
:10AF2000216A1A4034D0606DA3895B0706D5636837
:10AF3000C01A636B002B01D0236CC01A0200216A77
:10AF400000232800E76AB847A189431C06D12B6873
:10AF50001D2B30D82B4ADA40D3072CD50023636051
:10AF600023692360CB0405D5431C02D12B68002B39
:10AF700000D16065616B2E600029C7D02300443387
:10AF8000994202D0280000F0D7F900206063BEE7A4
:10AF900001232800B847431CC6D12B68002BC3D01F
:10AFA0001D2B01D0162B01D12E60AFE74023A289C3
:10AFB0001343A381ABE740230B430120A38140420D
:10AFC000A5E70F69002FA1D00B680F60DB1B019371
:10AFD0000023920700D14B69A360019B002B00DC8A
:10AFE00094E7019B3A00216A2800A66AB04700282E
:10AFF00003DC4023A2891343DFE7019B3F181B1AA0
:10B000000193EAE7010040200B6970B505000C00D0
:10B01000002B01D1002070BD002804D08369002BD3
:10B0200001D100F05FF80B4B9C4209D16C680C22F7
:10B03000A35E002BEED021002800FFF75BFFEAE7BC
:10B04000054B9C4201D1AC68F1E7044B9C42EED128
:10B05000EC68ECE7E4CF000004D00000C4CF0000AF
:10B06000002310B504000360436083608181436660
:10B07000C281036143618361190008225C30FFF7DC
:10B0800017FA054B24626362044BA362044BE3622C
:10B09000044B236310BDC0464DB8000075B80000D6
:10B0A000ADB80000D9B8000010B5024900F08CF826
:10B0B00010BDC04609B0000070B568254A1E554352
:10B0C0000E002900743100F081F9041E08D000211F
:10B0D0002A00016046600C30A0606832FFF7E8F992
:10B0E000200070BD836913B50400002B28D1836450
:10B0F000C3640365134B144A1B6882620193984230
:10B1000001D101238361200000F020F8606020005D
:10B1100000F01CF8A060200000F018F80022E060A9
:10B1200004216068FFF79CFF01220921A068FFF756
:10B1300097FF02221221E068FFF792FF0123A3612B
:10B1400013BDC0468CCF0000A9B00000F8B51C4B61
:10B1500007001E68B369002B02D13000FFF7C2FF61
:10B160004836B4687368013B04D53368002B07D0B8
:10B170003668F6E70C22A55E002D0DD06834F2E7A4
:10B1800004213800FFF798FF30600028F0D10C232D
:10B1900004003B602000F8BD20000A4B6566256076
:10B1A0006560A560E36025616561A56108222900ED
:10B1B0005C30FFF77DF96563A563A564E564E9E7A5
:10B1C0008CCF00000100FFFFF7B504000700002648
:10B1D00001914834002C01D13000FEBD6368A568A0
:10B1E0000093009B013B009301D52468F2E7AB89F3
:10B1F000012B08D90E22AB5E013304D029003800A0
:10B20000019B984706436835EBE7EC3000687047D0
:10B2100070B50E001D000E23C95E96B01400002903
:10B2200007DA00232B60B3891B0611D48023DB00CF
:10B230000FE06A4600F088FB0028F2DBF022019B59
:10B2400012021340054A9B185A4253412B60EDE706
:10B2500040230020236016B070BDC04600E0FFFF11
:10B26000F7B502268B8905000C00334206D0230077
:10B2700047332360236101236361F7BD01AB6A4655
:10B28000FFF7C6FF00990700280000F09FF800288C
:10B2900008D10C22A35E9A05EFD4032293431E43E8
:10B2A000A681E4E70F4BAB628023A28920601343A1
:10B2B000A381009B20616361019B002B0DD00E23B5
:10B2C000E15E280000F052FB002806D00322A3898B
:10B2D00093431A0001231343A381A0893843A0811B
:10B2E000CBE7C046A9B0000010B5034B01001868B9
:10B2F00000F06CF810BDC0466C00002082B0002940
:10B3000000D101A9101E06D0002B06D013780B60C7
:10B310001078431E984102B0704702204042FAE77D
:10B32000C9B28218904201D10020704703788B4245
:10B33000FBD00130F6E7000070B50500002910D001
:10B340000C1F2368002B00DAE418280000F034FBFF
:10B350001D4A1368002B05D163601460280000F0BB
:10B360002CFB70BDA34209D9216860188342F3D138
:10B3700018685B6841182160EEE713005A68002ADC
:10B3800001D0A242F9D919685818A0420BD12068FF
:10B390000918581819608242E0D1106852684118A3
:10B3A00019605A60DAE7A04202D90C232B60D5E776
:10B3B00021686018824203D11068526841182160E8
:10B3C00062605C60CAE7C046EC1B0020032370B5D6
:10B3D000CD1C9D43083506000C2D1ED20C25A9421C
:10B3E0001DD8300000F0E8FA254A14682100002931
:10B3F00019D1244C2368002B03D1300000F0CAF986
:10B4000020602900300000F0C5F9431C2BD10C232B
:10B410003000336000F0D1FA03E0002DDFDA0C23B6
:10B420003360002070BD0B685B1B19D40B2B03D954
:10B430000B60CC18256003E04B688C420DD1136083
:10B44000300000F0BAFA200007220B30231D904391
:10B45000C31AE7D05A42E250E4E763600C00EFE71A
:10B460000C004968C3E70323C41C9C43A042E1D0FD
:10B47000211A300000F08EF9431CDBD1C7E7C0462B
:10B48000EC1B0020F01B0020F8B507000D00160093
:10B49000002905D11100FFF799FF04002000F8BD35
:10B4A000002A03D1FFF748FF3400F7E700F086FADF
:10B4B0002C00B042F2D231003800FFF787FF041EA3
:10B4C000ECD029003200FEF7D7FF29003800FFF743
:10B4D00033FFE3E7F0B58E6885B007000C000392F8
:10B4E00001939E423CD890238A89DB001A4234D0D3
:10B4F0000325096923685B1A0293636902985D4317
:10B50000EB0F5D19019B6D1001331B18AB4200D985
:10B510001D00530532D529003800FFF757FF061EDE
:10B5200009D10C233B6040230120A28940421343F0
:10B53000A38105B0F0BD029A2169FEF79DFFA389A2
:10B54000144A1A4080231343A381029B2661F618F4
:10B5500026606561019EED1AA560019B9E4200D99F
:10B56000019E320003992068FEF78FFFA368002038
:10B570009B1BA36023689E192660DAE72A00380027
:10B58000FFF782FF061EE0D121693800FFF7D4FEE5
:10B59000C7E7C0467FFBFFFFF0B59FB00290059361
:10B5A0008B890F0016001B0611D50B69002B0ED1DD
:10B5B0004021FFF70BFF38603861002805D10C23CC
:10B5C000029A013813601FB0F0BD40237B61002355
:10B5D00006AC6361203363761033A37635002B7895
:10B5E000002B01D0252B46D1AB1B04930CD032008D
:10B5F00039000298FFF76EFF431C00D1AEE062698C
:10B60000049B9446634463612B78002B00D1A5E032
:10B61000012200235242626002A9543252186E1C69
:10B620002360E360A3601370A3653178052254485A
:10B63000FFF776FE751C00281FD12268D30604D5BB
:10B64000532302A95B1820211970130704D5532333
:10B6500002A95B182B21197033782A2B16D03500DC
:10B6600000210A20E3682A786E1C303A092A4ED954
:10B67000002918D010E00135B1E7414B2268C01A0B
:10B6800001238340134323602E00CEE7059B191D41
:10B690001B680591002B01DB099304E05B42E3602A
:10B6A0000223134323602B782E2B0AD16B782A2B8D
:10B6B00035D1059B02351A1D1B680592002B2BDB2B
:10B6C0000793304E297803223000FFF729FE002827
:10B6D00006D04023801B834022680135134323603A
:10B6E0002978062228486E1C2176FFF719FE0028CB
:10B6F0003CD0264B002B25D10722059B07339343D3
:10B70000083305936369039A9B18636166E74343B3
:10B7100001219B183500A6E701235B42D0E70023F7
:10B720000A201A000135636029786E1C3039092916
:10B7300003D9002BC5D00792C3E742430123521817
:10B740003500F1E705AB00933A00114B2100029858
:10B7500000E000BF0390039B0133D3D1BB890B985A
:10B760005B0600D42FE7012040422CE705AB009395
:10B770003A00074B21000298FFF74EF8EAE7C0466F
:10B7800090CF000096CF00009ACF0000000000008C
:10B79000D5B40000002370B5064C050008002360F6
:10B7A00000F060F9431C03D12368002B00D02B600C
:10B7B00070BDC046A42F002070B504000D001F29E5
:10B7C00004D9162303600120404270BD436C002B56
:10B7D00004D08A009B181A68002A08D1200000F0C3
:10B7E00031F82A000100200000F01AF8EDE70020EF
:10B7F000012AEAD0511C03D1162301302360E4E76B
:10B80000002428001C6090472000DEE710B5034BA1
:10B8100001001868FFF7D0FF10BDC0466C00002083
:10B82000002370B5064C050008001100236000F0ED
:10B8300001F9431C03D12368002B00D02B6070BD9D
:10B84000A42F002010B500F0E5F810BD70B50C0075
:10B850000E25495F00F0BAF8002803DB636D1B1862
:10B86000636570BDA389024A1340A381F9E7C0460E
:10B87000FFEFFFFFF8B51F008B8905000C001600D5
:10B88000DB0505D50E23C95E0022022300F080F8F7
:10B89000A389054A28001340A38132000E23E15EEC
:10B8A0003B0000F02BF8F8BDFFEFFFFF70B50C0078
:10B8B0000E25495F00F06CF8A389421C03D1054AAC
:10B8C0001340A38170BD802252011343A3816065A0
:10B8D000F8E7C046FFEFFFFF10B50E23C95E00F08A
:10B8E00021F810BD0B1E04D0FF2A04D98A2303605F
:10B8F0008B3B180070470A700123FAE770B505000A
:10B90000080011000022064C22601A0000F0B8F86E
:10B91000431C03D12368002B00D02B6070BDC046B0
:10B92000A42F0020002370B5064C050008002360FA
:10B9300000F060F8431C03D12368002B00D02B607B
:10B9400070BDC046A42F0020002370B5064C050032
:10B9500008001100236000F055F8431C03D1236850
:10B96000002B00D02B6070BDA42F0020002370B5E9
:10B97000064C05000800236000F054F8431C03D176
:10B980002368002B00D02B6070BDC046A42F002080
:10B9900070B50500080011000022064C22601A0054
:10B9A00000F050F8431C03D12368002B00D02B601B
:10B9B00070BDC046A42F0020704770470B1F1B6846
:10B9C000181F002B01DA0B58C018704770B505001E
:10B9D000080011000022064C22601A0000F03AF81C
:10B9E000431C03D12368002B00D02B6070BDC046E0
:10B9F000A42F002058220120014B40421A607047BA
:10BA0000A42F002058220120014B40421A607047A9
:10BA1000A42F002058220120014B40421A60704799
:10BA2000A42F00205822024B00201A607047C04605
:10BA3000A42F002058220120014B40421A60704779
:10BA4000A42F002058220120014B40421A60704769
:10BA5000A42F002058220120014B40421A60704759
:10BA6000A42F0020044A1368002B00D1034B1818A0
:10BA7000106018007047C046F41B0020A82F00205B
:10BA800058220120014B40421A607047A42F002029
:10BA9000FEE7C046F8B5C046F8BC08BC9E467047F5
:10BAA000F8B5C046F8BC08BC9E4670476461746136
:10BAB0000000000028BB0000EB01000031BB0000CB
:10BAC0001704000039BB00002D07000040BB000038
:10BAD0003D08000045BB0000DF02000050BB000035
:10BAE0008304000055BB0000B509000061BB0000E5
:10BAF0001B0200006BBB00003506000079BB000094
:10BB0000A105000072616E646F6D00616C6C006C69
:10BB10006173740066616C736500747275650025ED
:10BB20002E3135732E2E2E006D616B654C6973744A
:10BB3000006164644C6173740064656C65746500D5
:10BB40006A6F696E00636F707946726F6D546F0033
:10BB500066696E64006A6F696E537472696E6773AA
:10BB600000756E69636F6465417400756E69636F1B
:10BB70006465537472696E6700667265654D656DC4
:10BB80006F727900CC0F0000DC0F0000F60F000090
:10BB900074100000AC100000E21000001A11000048
:10BBA000401100007C110000BE11000014120000C2
:10BBB00058120000C41200000C13000032130000E1
:10BBC0006A130000B0130000D61300000414000034
:10BBD000361400006E140000F2140000BA150000C4
:10BBE000301600009C160000F01600001017000030
:10BBF00032170000E41700002A180000A218000005
:10BC0000CC0F0000CC0F0000D01800003819000045
:10BC1000BC190000021A00004A1A0000BC1A0000F9
:10BC20002E1B0000761B0000BC1B0000F21B000056
:10BC3000381C00007E1C0000C61C00001A1D0000FD
:10BC4000781D0000B61D0000201E0000561E0000DA
:10BC50009E1E0000E61E00002E1F0000681F000050
:10BC6000B01F0000F81F0000CC0F0000CC0F000038
:10BC7000CC0F000060200000CC0F000096200000D8
:10BC8000C2200000F820000024210000CC0F00009A
:10BC9000CC0F0000CC0F0000CC0F00005A21000098
:10BCA000A6210000CC0F0000CC0F0000EC2100000A
:10BCB0003C22000062220000CC0F0000CC0F0000EC
:10BCC000CC0F000090220000C0220000F0220000F3
:10BCD000262300005023000086230000B02300002C
:10BCE000D82300000024000030240000602400005D
:10BCF0008A240000B4240000E42400000E25000083
:10BD0000CC0F0000CC0F0000CC0F0000CC0F0000C7
:10BD1000CC0F00003E25000084250000B025000067
:10BD2000DC250000082600003E26000074260000E6
:10BD3000AA260000E02600000C270000382700009B
:10BD40006E270000CC0F0000CC0F0000CC0F0000CD
:10BD5000CC0F0000CC0F0000CC0F0000CC0F000077
:10BD6000CC0F0000CC0F0000CC0F0000CC0F000067
:10BD7000CC0F0000CC0F0000CC0F00009A27000071
:10BD8000D0270000282564206974656D206C6973D4
:10BD9000742900286F626A65637420747970653A4B
:10BDA0002025642900537461636B20756E6465728D
:10BDB000666C6F77000000000700000003000000C1
:10BDC00002BE0000B52800000ABE0000B92800002D
:10BDD00013BE0000B12800001CBE0000BD280000FA
:10BDE000000000000100000002000000030000004D
:10BDF000040000000A0000006D6963726F3A626916
:10BE00007400686173546F6E6500706C6179546F73
:10BE10006E6500686173536572766F007365745365
:10BE20006572766F00474320746F6F6B2025642026
:10BE300075736563733B20667265652025642077A2
:10BE40006F726473003C496E74656765723E003CB6
:10BE50004F626A6563743E003C4C6973743E000D2A
:10BE60000A564D2050616E69633A2025730D0A0011
:10BE70006D6973630000000088BE00007D31000022
:10BE800091BE000035310000686578546F496E74CA
:10BE90000073696E00000000E4BE0000E93100009C
:10BEA000ECBE0000ED310000F6BE00000B320000D9
:10BEB000FFBE0000153200000ABF00001F32000064
:10BEC00016BF00002932000027BF000033320000F7
:10BED0003DBF0000F731000056BF000001320000F6
:10BEE0006E657400686173576946690073746172A6
:10BEF00074576946690073746F70576946690077B3
:10BF0000696669537461747573006D794950416451
:10BF10006472657373007468696E674465736372F5
:10BF2000697074696F6E00636C6561725468696EE4
:10BF3000674465736372697074696F6E00617070D5
:10BF4000656E64546F5468696E67446573637269A3
:10BF50007074696F6E00617070656E64546F5468C0
:10BF6000696E6750726F7065727479001A1B1C03DA
:10BF7000040607090A17181900000000000808083D
:10BF800000080A4A4000000A5FEA5FEA0ED92ED391
:10BF90006E19324489330C924C924D08080000000F
:10BFA00004880808040804848488000A448A40003D
:10BFB000048EC480000000048800000EC000000051
:10BFC00000080001224488100C9252524C048C84C8
:10BFD000848E1C824C901E1EC244924C06CA525F34
:10BFE000E21FF01EC13E02448ED12E1FE244881093
:10BFF0000ED12ED12E0ED12EC488000800080000CC
:10C00000048004880244880482000EC00EC0080424
:10C010008244880ED126C0040ED135B36C0C925EDA
:10C02000D2521C925C925C0ED010100E1C92525296
:10C030005C1ED01C901E1ED01C90100ED013712EB2
:10C0400012525ED2521C8808081C1FE242524C1247
:10C0500054981492101010101E113B75B131113903
:10C0600035B3710C9252524C1C925C90100C92524F
:10C070004C861C925C92510ED00C825C1FE484842E
:10C0800084125252524C1131312A44113135BB7154
:10C0900012524C9252112A4484841EC488101E0EDF
:10C0A000C808080E10080482410EC242424E048A9B
:10C0B000400000000000001F0804800000000ED2B5
:10C0C000524F10101C925C000ED0100E02424ED245
:10C0D0004E0C925C900E06C81C88080ED24EC24CC4
:10C0E00010101C92520800080808024002424C102E
:10C0F000149814920808080806001B75B131001C3A
:10C10000925252000C92524C001C925C90000ED243
:10C110004EC2000ED010100006C8049808080EC8C1
:10C1200007001252524F0011312A4400113135BB21
:10C1300000124C8C9200112A4498001EC4881E06DE
:10C14000C48C8486080808080818080C88180000A1
:10C150000C836000000000000100000002000000ED
:10C1600003000000040000000500000006000000BD
:10C170000700000008000000090000000A0000009D
:10C180000B0000000C0000000D0000000E0000007D
:10C190000F0000001000000012000000140000005A
:10C1A00016000000180000001A0000001C0000002B
:10C1B0001E000000200000002300000026000000F8
:10C1C000290000002C0000002F00000032000000B9
:10C1D000360000003A0000003E000000420000006F
:10C1E000460000004B000000500000005500000019
:10C1F0005A00000061000000680000006F000000AD
:10C20000760000007D000000840000008B0000002C
:10C210009200000099000000A0000000A7000000AC
:10C22000AE000000B5000000BC000000C30000002C
:10C23000CA000000D1000000D8000000DF000000AC
:10C24000E6000000ED000000F4000000FB0000002C
:10C25000FF000000A4C2000059320000AFC200007D
:10C2600081370000B9C2000091340000C6C200004E
:10C27000B1340000CDC2000001350000D6C200007C
:10C2800051350000E2C200002D340000F3C200006E
:10C290009136000000C300004D37000064697370E0
:10C2A0006C6179006C696768744C6576656C006DCB
:10C2B00062446973706C6179006D62446973706C7B
:10C2C00061794F6666006D62506C6F74006D6255E7
:10C2D0006E706C6F74006D62447261775368617048
:10C2E00065006D625368617065466F724C65747469
:10C2F0006572006E656F506978656C53656E640099
:10C300006E656F506978656C53657450696E004E48
:10C310006F7420656E6F75676820726F6F6D206532
:10C3200076656E20616674657220636F6D706163FF
:10C3300074696F6E00436F6D70616374656420464D
:10C340006C61736820636F64652073746F72650A33
:10C3500025642062797465732075736564202825CF
:10C3600064252529206F66202564004261642072BF
:10C3700065636F726420666F756E642064757269A0
:10C380006E6720696E697469616C697A6174696F3E
:10C390006E002564202564202564202825642077EC
:10C3A0006F72647329002564207265636F72647311
:10C3B0002C20256420776F7264732C206D6178497E
:10C3C000442025642C20636F6D70616374696F6E07
:10C3D000206379636C657320256400526573746F04
:10C3E00072656420256420736372697074730053EE
:10C3F00074617274656400726164696F00000000AA
:10C400008EC40000494100009BC40000B9430000F5
:10C41000ABC4000059430000B9C400003945000016
:10C42000C4C4000061410000D4C40000D541000034
:10C43000E8C4000071410000F7C400001B47000081
:10C4400003C50000994600000CC500003D460000F1
:10C4500017C500008545000022C50000C145000049
:10C460002BC50000F545000034C5000085410000E3
:10C470006E756D626572006E6F6E65006F746865D3
:10C4800072007061697200737472696E670064692A
:10C490007361626C65526164696F006D657373618D
:10C4A00067655265636569766564007061636B6595
:10C4B0007452656365697665007061636B6574537A
:10C4C000656E64007265636569766564496E74655E
:10C4D0006765720072656365697665644D6573733F
:10C4E0006167655479706500726563656976656436
:10C4F000537472696E670073656E64496E74656724
:10C5000065720073656E64506169720073656E6474
:10C51000537472696E67007365744368616E6E650B
:10C520006C0073657447726F757000736574506F3B
:10C53000776572007369676E616C537472656E67BC
:10C540007468000000000000963007772C610EEE42
:10C55000BA51099919C46D078FF46A7035A563E95A
:10C56000A395649E3288DB0EA4B8DC791EE9D5E081
:10C5700088D9D2972B4CB609BD7CB17E072DB8E780
:10C58000911DBF906410B71DF220B06A4871B9F3D5
:10C59000DE41BE847DD4DA1AEBE4DD6D51B5D4F40E
:10C5A000C785D38356986C13C0A86B647AF962FD73
:10C5B000ECC9658A4F5C0114D96C0663633D0FFAC0
:10C5C000F50D088DC8206E3B5E10694CE44160D5C6
:10C5D000727167A2D1E4033C47D4044BFD850DD2B0
:10C5E0006BB50AA5FAA8B5356C98B242D6C9BBDBC3
:10C5F00040F9BCACE36CD832755CDF45CF0DD6DCBE
:10C60000593DD1ABAC30D9263A00DE518051D7C864
:10C610001661D0BFB5F4B42123C4B3569995BACFEF
:10C620000FA5BDB89EB802280888055FB2D90CC610
:10C6300024E90BB1877C6F2F114C6858AB1D61C189
:10C640003D2D66B69041DC760671DB01BC20D298A8
:10C650002A10D5EF8985B1711FB5B606A5E4BF9F35
:10C6600033D4B8E8A2C9077834F9000F8EA8099628
:10C6700018980EE1BB0D6A7F2D3D6D08976C649193
:10C68000015C63E6F4516B6B62616C1CD8306585AC
:10C690004E0062F2ED95066C7BA5011BC1F4088289
:10C6A00057C40FF5C6D9B06550E9B712EAB8BE8BCA
:10C6B0007C88B9FCDF1DDD62492DDA15F37CD38C53
:10C6C000654CD4FB5861B24DCE51B53A7400BCA351
:10C6D000E230BBD441A5DF4AD795D83D6DC4D1A483
:10C6E000FBF4D6D36AE96943FCD96E34468867AD5A
:10C6F000D0B860DA732D0444E51D03335F4C0AAAF9
:10C70000C97C0DDD3C710550AA41022710100BBEFB
:10C7100086200CC925B56857B3856F2009D466B942
:10C720009FE461CE0EF9DE5E98C9D9292298D0B077
:10C73000B4A8D7C7173DB359810DB42E3B5CBDB724
:10C74000AD6CBAC02083B8EDB6B3BF9A0CE2B603A5
:10C750009AD2B1743947D5EAAF77D29D1526DB045A
:10C760008316DC73120B63E3843B64943E6A6D0DA5
:10C77000A85A6A7A0BCF0EE49DFF099327AE000AF0
:10C78000B19E077D44930FF0D2A3088768F2011E83
:10C79000FEC206695D5762F7CB67658071366C191A
:10C7A000E7066B6E761BD4FEE02BD3895A7ADA103B
:10C7B000CC4ADD676FDFB9F9F9EFBE8E43BEB7171C
:10C7C000D58EB060E8A3D6D67E93D1A1C4C2D838A6
:10C7D00052F2DF4FF167BBD16757BCA6DD06B53F0C
:10C7E0004B36B248DA2B0DD84C1B0AAFF64A03364B
:10C7F000607A0441C3EF60DF55DF67A8EF8E6E31CA
:10C8000079BE69468CB361CB1A8366BCA0D26F2512
:10C8100036E2685295770CCC03470BBBB91602225F
:10C820002F260555BE3BBAC5280BBDB2925AB42B74
:10C83000046AB35CA7FFD7C231CFD0B58B9ED92C89
:10C840001DAEDE5BB0C2649B26F263EC9CA36A75EE
:10C850000A936D02A906099C3F360EEB85670772A5
:10C8600013570005824ABF95147AB8E2AE2BB17B0C
:10C87000381BB60C9B8ED2920DBED5E5B7EFDC7C93
:10C8800021DFDB0BD4D2D38642E2D4F1F8B3DD68EA
:10C890006E83DA1FCD16BE815B26B9F6E177B06FE5
:10C8A0007747B718E65A0888706A0FFFCA3B0666D2
:10C8B0005C0B0111FF9E658F69AE62F8D3FF6B615F
:10C8C00045CF6C1678E20AA0EED20DD75483044E01
:10C8D000C2B30339612667A7F71660D04D4769498F
:10C8E000DB776E3E4A6AD1AEDC5AD6D9660BDF40A2
:10C8F000F03BD83753AEBCA9C59EBBDE7FCFB24755
:10C90000E9FFB5301CF2BDBD8AC2BACA3093B35339
:10C91000A6A3B4240536D0BA9306D7CD2957DE5442
:10C92000BF67D9232E7A66B3B84A61C4021B685D1B
:10C93000942B6F2A37BE0BB4A18E0CC31BDF055A94
:10C940008DEF022D416C6C207461736B73207374D6
:10C950006F707065640076303732002025732025B3
:10C9600073004D656D6F727920636C6561726564EB
:10C97000004E6F2066726565207461736B20656E72
:10C980007472696573000000D0C90000ED590000A1
:10C99000DDC9000085560000E9C90000235A0000E7
:10C9A000EFC90000335A0000F5C90000435A0000E7
:10C9B000FBC90000B956000005CA0000555A000026
:10C9C0000DCA0000F957000073656E736F72730033
:10C9D000616363656C65726174696F6E0074656D27
:10C9E00070657261747572650074696C7458007456
:10C9F000696C74590074696C745A00746F7563685B
:10CA00005265616400693263526561640069326332
:10CA100057726974650000008CCA0000D55A000086
:10CA20009ACA0000D95A0000A3CA0000E55A0000C3
:10CA3000ADCA0000E95A0000B6CA0000ED5A000075
:10CA4000BBCA0000F15A0000C0CA0000F55A00003D
:10CA5000CCCA0000F95A0000D3CA0000FD5A0000F9
:10CA6000DCCA0000015B0000E1CA0000055B0000B9
:10CA7000ECCA0000095B0000F6CA0000DD5A0000A5
:10CA800000CB0000E15A000074667400656E6162BC
:10CA90006C65446973706C6179006765745769648B
:10CAA00074680067657448656967687400736574C5
:10CAB000506978656C006C696E650072656374001E
:10CAC000726F756E64656452656374006369726346
:10CAD0006C6500747269616E676C6500746578746A
:10CAE00000746674546F756368656400746674548A
:10CAF0006F7563685800746674546F756368590085
:10CB0000746674546F75636850726573737572657B
:10CB10000057656C636F6D6520746F204D6963729B
:10CB20006F426C6F636B732100705F7370692021BB
:10CB30003D204E554C4C002F686F6D652F62726F13
:10CB40006D61676F73612F2E706C6174666F726DAB
:10CB5000696F2F7061636B616765732F6672616DBA
:10CB600065776F726B2D61726475696E6F6E6F722F
:10CB70006469636E7266352F6C6962726172696591
:10CB8000732F5350492F5350492E637070005350E8
:10CB900049436C6173733A3A535049436C61737300
:10CBA000284E52465F5350495F547970652A2C20B5
:10CBB00075696E74385F742C2075696E74385F7493
:10CBC0002C2075696E74385F742900000000000025
:10CBD000000000000D5D0000C95C0000EF5C00007B
:10CBE000F95C0000035D0000ED5C00000300000044
:10CBF0000200000001000000040000000500000029
:10CC0000110000000C0000000B00000012000000EA
:10CC10000A000000060000001A00000014000000D6
:10CC200017000000160000001500000010000000B2
:10CC3000FFFFFFFFFFFFFFFF000000001E000000DE
:10CC400019000000180000000700000008000000A4
:10CC5000090000000D0000000E0000000F000000A1
:10CC60001C0000001B0000001D000000130000005D
:10CC70000000000000000000BD610000ED68000041
:10CC80003D6200005162000047620000B96100008F
:10CC9000AD6100005D620000D9610000A961000083
:10CCA000000000000000304300000000000030C31E
:10CCB0007371727400000000FB21F93FFB210940F1
:10CCC0007CD91240FB2119407A6A1F407CD922404E
:10CCD000BBFD2540FB2129403A462C407A6A2F4073
:10CCE0005C4731407CD932409C6B3440BBFD3540C1
:10CCF000DB8F3740FB2139401BB43A403A463C4079
:10CD00005AD83D407A6A3F404C7E40405C474140A3
:10CD10006C1042407CD942408CA243409C6B444002
:10CD2000AC344540BBFD4540CBC64640DB8F474059
:10CD3000EB584840FB21494083F9A200444E6E0065
:10CD4000FC291500D1572700DD34F50062DBC00057
:10CD50003C999500419043006351FE00BBDEAB005F
:10CD6000B761C5003A6E2400D24D42004906E0008A
:10CD700009EA2E001C92D100EB1DFE0029B11C0017
:10CD8000E83EA700F535820044BB2E009CE98400F4
:10CD9000B4267000417E5F00D6913900538339007C
:10CDA0009CF439008B5F840028F9BD00F81F3B001C
:10CDB000DEFF97000F980500112FEF000A5A8B0035
:10CDC0006D1F6D00CF7E360009CB2700464FB700A0
:10CDD0009E663F002DEA5F00BA277500E5EBC700AD
:10CDE0003D7BF100F739070092528A00FB6BEA00A5
:10CDF0001FB15F00085D8D00300356007BFC4600CC
:10CE0000F0AB6B0020BCCF0036F49A00E3A91D0004
:10CE10005E619100081BE60085996500A0145F0023
:10CE20008D40680080D8FF0027734D000606310052
:10CE3000CA561500C9A873007BE260006B8CC00065
:10CE400000000040FB21F93F000000002D44743E2B
:10CE5000000000809846F83C0000006051CC783B10
:10CE600000000080831BF0390000004020257A3844
:10CE7000000000802282E336000000001DF36935C7
:10CE80000200000003000000040000000600000093
:10CE9000E48500008E8500008E850000BC860000C1
:10CEA0008A8500008A850000B2860000BC860000EA
:10CEB0008A850000B28600008A850000BC860000DA
:10CEC000C0860000C0860000C0860000C886000042
:10CED000C0900000328F0000768F0000DA8E0000D4
:10CEE000768F000066900000768F0000DA8E0000DA
:10CEF000328F0000328F000066900000DA8E000052
:10CF0000D28E0000D28E0000D28E000074900000FD
:10CF1000E8970000EA960000EA960000089A0000F0
:10CF2000E4960000E4960000F0990000089A0000E2
:10CF3000E4960000F0990000E4960000089A0000D2
:10CF4000FE990000FE990000FE9900000C9A000076
:10CF50002C2066756E6374696F6E3A20006173737E
:10CF6000657274696F6E2022257322206661696C78
:10CF700065643A2066696C6520222573222C206C3A
:10CF8000696E65202564257325730A0070000020F2
:10CF9000232D302B2000686C4C00656667454647A2
:10CFA0000030313233343536373839414243444525
:10CFB0004600303132333435363738396162636494
:10CFC0006566000000000000000000000000000096
:10CFD0000000000000000000000000000000000051
:10CFE0000000000000000000000000000000000041
:10CFF0000000000000000000000000000000000031
:10D000000000000000000000000000000000000020
:10D010000000000000000000000000000000000010
:10D02000000000004300504F5349580000202020CA
:10D0300020202020202028282828282020202020C8
:10D040002020202020202020202020202088101098
:10D0500010101010101010101010101010040404F4
:10D0600004040404040404101010101010104141B2
:10D0700041414141010101010101010101010101A0
:10D0800001010101010101011010101010104242B4
:10D090004242424202020202020202020202020270
:10D0A0000202020202020202101010102000000010
:10D0B0000000000000000000000000000000000070
:10D0C0000000000000000000000000000000000060
:10D0D0000000000000000000000000000000000050
:10D0E0000000000000000000000000000000000040
:10D0F0000000000000000000000000000000000030
:10D10000000000000000000000000000000000001F
:10D11000000000000000000000000000000000000F
:10D1200000000000000000000000000000000000FF
:04D1300000000000FB
:08D13400D42FFF7F0100000071
:10D13C00FFFFFFFF40060000010000001800000088
:10D14C0019FCFFFFFFFFFFFFFF00000002000000C3
:10D15C0003000000FFFFFFFF0000000001000000C3
:10D16C000000020001000000FFFFFFFF00000000B4
:10D17C00020000000000040002000000FFFFFFFF9F
:10D18C000000000003000000000008000300000085
:10D19C000A000000080000000100000070000020E0
:10D1AC0000000000E4CF000004D00000C4CF000059
:10D1BC000000000000000000000000000000000063
:10D1CC000000000000000000000000000000000053
:10D1DC000000000000000000000000000000000043
:10D1EC000000000000000000000000000000000033
:10D1FC000000000000000000000000000000000023
:10D20C0043000000000000000000000000000000CF
:10D21C000000000000000000000000000000000002
:10D22C0043000000000000000000000000000000AF
:10D23C0000000000000000000000000000000000E2
:10D24C00430000000000000000000000000000008F
:10D25C0000000000000000000000000000000000C2
:10D26C00430000000000000000000000000000006F
:10D27C0000000000000000000000000000000000A2
:10D28C00430000000000000000000000000000004F
:10D29C000000000000000000000000000000000082
:10D2AC00430000000000000000000000000000002F
:10D2BC000000000000000000000000000000000062
:10D2CC00430000000000000000000000000000000F
:10D2DC000000000000000000000000000000000042
:10D2EC00E5B80000FDB20000000000002CD00000EA
:10D2FC0026BB00006FBE00006FBE00006FBE0000BA
:10D30C006FBE00006FBE00006FBE00006FBE00005D
:10D31C006FBE00006FBE0000FFFFFFFFFFFFFFFFAF
:10D32C00FFFFFFFFFFFF000001004153434949008D
:10D33C0000000000000000000000000000000000E1
:10D34C000000000000000000000041534349490068
:10D35C0000000000000000000000000000000000C1
:10D36C00000000000000000000000000E9000000C8
:10D37C00995C0000E15F000009650000C10000003D
:040000030000607D1C
:00000001FF
